:020000040800F2
:1000000000060020E10100086D0E0008ED0D00085B
:10001000450E0008ED0D0008190E0008E301000868
:10002000E3010008E3010008E301000841210008A2
:10003000E3010008E3010008E3010008E301000810
:10004000E3010008E3010008E3010008E301000800
:10005000E3010008E3010008093200083532000816
:10006000613200088D320008B9320008E30100084F
:10007000E3010008E3010008E3010008E3010008D0
:10008000E3010008E3010008E3010008E3010008C0
:10009000E3010008E3010008E3010008E53200087D
:1000A000E3010008E3010008E3010008E3010008A0
:1000B0007D300008E3010008E3010008E3010008C7
:1000C000E3010008E3010008E3010008E301000880
:1000D000E3010008E3010008E3010008E301000870
:1000E0004D330008E3010008E3010008E3010008C4
:1000F000E3010008E3010008E3010008E301000850
:10010000E3010008E3010008E3010008E30100083F
:10011000E3010008E3010008E3010008E30100082F
:10012000E3010008E3010008E3010008E30100081F
:10013000E3010008E3010008E3010008E30100080F
:10014000E3010008E3010008E30100087928000842
:10015000E3010008E3010008E3010008E3010008EF
:10016000E3010008E3010008E3010008E3010008DF
:10017000E3010008E3010008E3010008E3010008CF
:10018000E3010008E3010008E3010008E3010008BF
:10019000E3010008E3010008E3010008E3010008AF
:1001A000E3010008E3010008E3010008E30100089F
:1001B000E3010008E3010008E3010008E30100088F
:1001C000E3010008E3010008E3010008E30100087F
:1001D000E3010008E3010008E3010008E30100086F
:1001E00002E000F000F8FEE772B63A4880F30888B3
:1001F000394880F3098839484EF60851CEF200019B
:10020000086040F20000CCF200004EF63471CEF2ED
:1002100000010860BFF34F8FBFF36F8F40F2000003
:10022000C0F2F0004EF68851CEF200010860BFF334
:100230004F8FBFF36F8F4FF00000E1EE100A4EF6C4
:100240003C71CEF200010860062080F31488BFF3F1
:100250006F8F01F0F5FF01F0D1FF02F073FE4FF058
:1002600055301F491B4A91423CBF41F8040BFAE745
:100270001C49194A91423CBF41F8040BFAE71A495C
:100280001A4A1B4B9A423EBF51F8040B42F8040B2A
:10029000F8E700201749184A91423CBF41F8040B87
:1002A000FAE701F0AFFF02F0A1FE144C144DAC428E
:1002B00003DA54F8041B8847F9E700F041F8114CC1
:1002C000114DAC4203DA54F8041B8847F9E701F0FA
:1002D00097BF000000060020002200200000000858
:1002E00000000020000600207837000800220020CF
:1002F0004022002040220020A82D0020E00100081C
:10030000E0010008E0010008E00100082DE9F04FDD
:100310002DED108AC1F80CD0C3689D46BDEC108A43
:10032000BDE8F08F002383F311882846A047002002
:1003300001F012FBFEE701F08DFA00DFFEE700009E
:1003400038B501F0CDFE054601F0F0FE0446D8B9FF
:100350000F4B9D421AD001339D4218BF044641F213
:10036000883504BF01240025002001F0C3FE0CB134
:1003700000F076F800F010FD00F09EFB284600F03B
:10038000BFF800F06DF8F9E70025EDE70546EBE76B
:10039000010007B008B500F061FBA0F1200358424E
:1003A000584108BD07B541F21203022101A8ADF87A
:1003B000043000F071FB03B05DF804FB38B5202376
:1003C00083F311881748C3680BB101F04BFB164A41
:1003D000144800234FF47A7101F008FB002383F3E3
:1003E0001188124C236813B12368013B23606368B2
:1003F00013B16368013B63600D4D2B7833B96368BB
:100400007BB9022000F042FC322363602B78032B7F
:1004100007D163682BB9022000F038FC4FF47A73DF
:10042000636038BD40220020BD0300085C2300202B
:1004300054220020084B187003280CD8DFE800F085
:1004400008050208022000F017BC022000F00ABCD8
:10045000024B00225A607047542200205C23002087
:10046000234B244A10B51C46196801313FD0043390
:100470009342F9D16268A24239D31F4B9B6803F1C2
:10048000006303F540439A4231D2002000F02EFB76
:100490000220FFF7CFFF194B1A6C00221A64196E65
:1004A0001A66196E596C5A64596E5A665A6E5A69B0
:1004B00042F080025A615A6922F080025A615A69F8
:1004C0001A6942F000521A611A6922F000521A6148
:1004D0001B6972B64FF0E0232021C3F8084DD4E920
:1004E000003281F311889D4683F30888104710BDC0
:1004F00000C0000820C00008002200200038024090
:100500002DE9F04F93B0A94B00902022FF210AA8BB
:100510009D6800F0EBFBA64A1378A3B9A54801211A
:10052000C3601170202383F31188C3680BB101F0FD
:1005300099FAA14A9F4800234FF47A7101F056FAC4
:10054000002383F31188009B13B19C4B009A1A601F
:100550009B4A009C1378032B1EBF00231370974AFD
:100560004FF0000A18BF5360D3465646D1460120CB
:1005700000F082FB24B1914B1B68002B00F00F822E
:10058000002000F06BFA0390039B002BF2DB0120AC
:1005900000F068FB039B213B162BE8D801A252F820
:1005A00023F000BF0106000829060008BD06000868
:1005B0006F0500086F0500086F0500084507000873
:1005C000130900082D0800088F080008B708000864
:1005D000DD0800086F050008EF0800086F05000837
:1005E00061090008A10600086F050008A5090008B8
:1005F0000D060008A10600086F0500088F08000816
:100600000220FFF7C7FE002840F0F381009B022183
:10061000BAF1000F08BF1C4605A841F21233ADF82D
:10062000143000F039FAA2E74FF47A7000F016FAAD
:10063000071EEBDB0220FFF7ADFE0028E6D0013FEE
:10064000052F00F2D881DFE807F0030A0D101336FA
:1006500005230593042105A800F01EFA17E053486E
:100660000421F9E757480421F6E757480421F3E746
:100670004FF01C08404600F03BFA08F104080590D2
:10068000042105A800F008FAB8F12C0FF2D10120DE
:1006900000FA07F747EA0B0B5FFA8BFB4FF00009F4
:1006A00000F070FB26B10BF00B030B2B08BF0024EE
:1006B000FFF778FE5BE745480421CDE7002EA5D083
:1006C0000BF00B030B2BA1D10220FFF763FE0746B3
:1006D00000289BD0012000F009FA0220FFF7AAFEB3
:1006E00000265FFA86F8404600F010FA044688B10A
:1006F000404600F01BFA01360028F2D1BA46044603
:1007000041F21213022105A8ADF814303E4600F064
:10071000C3F92CE70120FFF78DFE2546234B9B688C
:10072000AB4207D9284600F0E3F9013040F066817A
:100730000435F3E7224B00251D70204BBA465D605F
:100740003E46ADE7002E3FF461AF0BF00B030B2BE1
:100750007FF45CAF0220FFF76DFE322000F07EF9DF
:10076000B0F10008FFF652AF18F003077FF44EAF68
:100770000E4A926808EB050393423FF647AFB8F57F
:10078000807F3FF743AF124B0193B84522DD4FF412
:100790007A7000F063F90390039A002AFFF636AFEF
:1007A000019B039A03F8012B0137EDE7002200209B
:1007B0005823002040220020BD0300085C230020B5
:1007C0005422002004220020082200200C220020B5
:1007D00058220020C820FFF7DDFD074600283FF41F
:1007E00015AF1F2D11D8C5F1200242450AAB25F0E7
:1007F000030028BF424683490192184400F050FA92
:10080000019A8048FF2100F071FA4FEAA8037D4960
:100810000193C8F38702284600F070FA06460028C4
:100820003FF46EAF019B05EB830539E70220FFF72C
:10083000B1FD00283FF4EAAE00F0A2F900283FF431
:10084000E5AE0027B846704B9B68BB4218D91F2FF6
:1008500011D80A9B01330ED027F0030312AA1344C8
:1008600053F8203C05934046042205A900F000FB04
:1008700004378046E7E7384600F03AF90590F2E79A
:10088000CDF81480042105A800F006F908E700233C
:10089000642104A8049300F0F5F800287FF4B6AEB4
:1008A0000220FFF777FD00283FF4B0AE049800F077
:1008B0004FF90590E6E70023642104A8049300F0B3
:1008C000E1F800287FF4A2AE0220FFF763FD0028C4
:1008D0003FF49CAE049800F04BF9EAE70220FFF7E2
:1008E00059FD00283FF492AE00F05AF9E1E70220EA
:1008F000FFF750FD00283FF489AE05A9142000F051
:1009000055F904210746049004A800F0C5F83946BB
:10091000B9E7322000F0A2F8071EFFF677AEBB075A
:100920007FF474AE384A926807EB090393423FF6AE
:100930006DAE0220FFF72EFD00283FF467AE27F0D2
:1009400003074F44B9453FF4ABAE484600F0D0F83A
:100950000421059005A800F09FF809F10409F1E7CA
:100960004FF47A70FFF716FD00283FF44FAE00F009
:1009700007F9002844D00A9B01330BD008220AA9AA
:10098000002000F0BBF900283AD02022FF210AA85D
:1009900000F0ACF9FFF706FD1C4800F0E3FF13B0D0
:1009A000BDE8F08F002E3FF431AE0BF00B030B2BA4
:1009B0007FF42CAE0023642105A8059300F062F8B3
:1009C000074600287FF422AE0220FFF7E3FC8046B2
:1009D00000283FF41BAEFFF7E5FC41F2883000F041
:1009E000C1FF059800F000FA464600F0CBF93C46FE
:1009F000BDE5064654E64FF0000907E6BA467FE635
:100A000037467DE65822002000220020A086010003
:100A100070B50F4B1B780133DBB2012B0C4611D89C
:100A20000C4D29684FF47A730E6AA2FB033201461B
:100A300022462846B047844204D1074B00221A7050
:100A4000012070BD4FF4FA7000F08CFF0020F8E731
:100A500010220020502500209023002007B50023FD
:100A6000024601210DF107008DF80730FFF7D0FF96
:100A700020B19DF8070003B05DF804FB4FF0FF3094
:100A8000F9E700000A4608B50421FFF7C1FF80F02E
:100A90000100C0B2404208BD30B4054C2368DD6996
:100AA000044B0A46AC460146204630BC604700BFB6
:100AB00050250020A086010070B501F003FA094E10
:100AC000094D3080002428683388834208D901F01A
:100AD000F3F92B6804440133B4F5404F2B60F2D393
:100AE00070BD00BF922300206423002001F0ACBA47
:100AF00000F1006000F540400068704700F10060C0
:100B0000920000F5404001F02BBA0000054B1A6836
:100B1000054B1B889B1A834202D9104401F0CCB9C3
:100B200000207047642300209223002038B5074D31
:100B300004462868204401F0C7F928B928682044F1
:100B4000BDE8384001F0D8B938BD00BF64230020AB
:100B500010F003030AD1B0F5047F05D200F1005074
:100B6000A0F51040D0F80038184670470023FBE786
:100B700000F10050A0F51040D0F8100A70470000B6
:100B8000064991F8243033B10023086A81F82430F3
:100B90000822FFF7B3BF0120704700BF6823002081
:100BA000014B1868704700BF002004E070B52A4B65
:100BB0001B68C3F30B0204461B0C62B140F21340E6
:100BC000824230D040F2194082422ED040F2214081
:100BD00082422CD10322214D0C2000FB0252556889
:100BE00042F20102934224D0B3F5805F23D041F258
:100BF0000102934221D041F2030293421FD041F2FD
:100C00000702934214BF3F233123013C0C44013DB2
:100C10000A46A24215D215F9016F501C9EB100F888
:100C2000016C0246F5E70122D5E70222D3E70C4D1D
:100C3000D6E73323E9E74123E7E75A23E5E75923DA
:100C4000E3E7104605E02C258442157001D9901C7D
:100C50005370401A70BD00BF002004E078340008D3
:100C60004C340008022802BF024B4FF080729A6198
:100C7000704700BF00080240022802BF024B4FF439
:100C800080729A61704700BF00080240022801BFCD
:100C9000024A536983F4807353617047000802402D
:100CA00010B50023934203D0CC5CC4540133F9E760
:100CB00010BD000010B5013810F9013F3BB191F9AA
:100CC00000409C4203D11AB10131013AF4E71AB154
:100CD00091F90020981A10BD1046FCE70346024621
:100CE000D01A12F9011B0029FAD1704702440346B9
:100CF000934202D003F8011BFAE770472DE9F8434D
:100D00001F4D144695F824200746884652BBDFF84D
:100D100070909CB395F824302BB92022FF214846CF
:100D20002F62FFF7E3FF95F82400C0F10802A2420A
:100D300028BF2246D6B24146920005EB8000FFF75D
:100D4000AFFF95F82430A41B1E44F6B2082E1744BA
:100D50009044E4B285F82460DBD1FFF711FF00284E
:100D6000D7D108E02B6A03EB82038342CFD0FFF791
:100D700007FF0028CBD10020BDE8F8830120FBE766
:100D800068230020024B1A78024B1A70704700BF8C
:100D9000902300201022002010B50F4C0F4800F0C7
:100DA000F7F821460D4800F01FF924680C48626DE1
:100DB000D2F8043843F00203C2F8043800F0D2FD40
:100DC0000849204600F016FA626DD2F8043823F084
:100DD0000203C2F8043810BD6C350008502500200D
:100DE00040420F00743500087047000000B59BB00A
:100DF000EFF3098168226846FFF752FFEFF305839E
:100E0000044B9A6BDA6A9A6A9A6A9A6A9A6A9A6A36
:100E10009B6AFEE700ED00E000B59BB0EFF30981AF
:100E200068226846FFF73CFFEFF30583044B9A6B9B
:100E30009A6A9A6A9A6A9A6A9A6A9B6AFEE700BFF5
:100E400000ED00E000B59BB0EFF309816822684631
:100E5000FFF726FFEFF30583034B5A6B9A6A9A6AF2
:100E60009A6A9A6A9B6AFEE700ED00E0FEE70000DE
:100E700030B5094D0A4491420DD011F8013B58405C
:100E8000082340F30004013B2C4013F0FF0384EAE5
:100E90005000F6D1EFE730BD2083B8ED026843681B
:100EA0001143016003B118477047000013B5446B4C
:100EB000D4F894341A681178042915D1217C0229B8
:100EC00012D11979128901238B4013420CD101A947
:100ED00004F14C0001F03CFFD4F89444019B2179CB
:100EE0000246206800F0CEF902B010BD143001F0C7
:100EF000BFBE00004FF0FF33143001F0B9BE000058
:100F00004C3001F091BF00004FF0FF334C3001F046
:100F10008BBF0000143001F08DBE00004FF0FF3198
:100F2000143001F087BE00004C3001F05DBF0000BE
:100F30004FF0FF324C3001F057BF000000207047E7
:100F400010B5D0F894341A6811780429044617D1E2
:100F5000017C022914D15979528901238B40134213
:100F60000ED1143001F020FE024648B1D4F894446A
:100F70004FF4807361792068BDE8104000F070B9CB
:100F800010BD0000406BFFF7DBBF000070470000A2
:100F90007FB5124B036000234360C0E90233012593
:100FA00002260F4B057404460290019300F184025F
:100FB000294600964FF48073143001F0D1FD094B9F
:100FC0000294CDE9006304F523724FF4807329463F
:100FD00004F14C0001F098FE04B070BDA834000884
:100FE000850F0008AD0E00080B68202282F31188DF
:100FF0000A7903EB820290614A79093243F82200B0
:101000008A7912B103EB8203986102230374C0F85A
:101010009414002383F311887047000038B5037FD0
:10102000044613B190F85430ABB9201D01250221BC
:10103000FFF734FF04F1140025776FF0010100F091
:10104000B9FC84F8545004F14C006FF00101BDE884
:10105000384000F0AFBC38BD10B501210446043063
:10106000FFF71CFF0023237784F8543010BD0000E5
:1010700038B504460025143001F08AFD04F14C0017
:10108000257701F059FE201D84F854500121FFF707
:1010900005FF2046BDE83840FFF752BF90F84430C6
:1010A00003F06003202B07D190F84520212A4FF050
:1010B000000303D81F2A06D800207047222AFBD13C
:1010C000C0E90E3303E0034A82630722C26303646C
:1010D000012070471122002037B5D0F894341A68E7
:1010E0001178042904461AD1017C022917D11979F3
:1010F000128901238B40134211D100F14C0528467F
:1011000001F0DAFE58B101A9284601F021FED4F819
:101110009444019B21790246206800F0B3F803B0A3
:1011200030BD0000F0B500EB810385B09E69044638
:101130000D46FEB1202383F3118804EB8507301D93
:101140000821FFF7ABFEFB685B691B6806F14C00EA
:101150001BB1019001F00AFE019803A901F0F8FD0E
:10116000024648B1039B2946204600F08BF8002335
:1011700083F3118805B0F0BDFB685A691268002A34
:10118000F5D01B8A013B1340F1D104F14402EAE798
:10119000093138B550F82140DCB1202383F31188A0
:1011A000D4F894241368527903EB8203DB689B69BB
:1011B0005D6845B104216018FFF770FE294604F10F
:1011C000140001F0FBFC2046FFF7BAFE002383F376
:1011D000118838BD7047000001F0A8B801230370E2
:1011E0000023C0E90133C36183620362C3624362C7
:1011F0000363704738B50446202383F31188002524
:10120000C0E90355C0E90555416001F09FF802238C
:10121000237085F3118838BD70B500EB8103054656
:101220005069DA600E46144618B110220021FFF70B
:101230005DFDA06918B110220021FFF757FD31466E
:101240002846BDE8704001F04BB90000826802F00A
:10125000011282600022C0E90422826101F0CCB94F
:10126000F0B400EB81044789E4680125A4698D404E
:101270003D43458123600023A2606360F0BC01F020
:10128000E7B90000F0B400EB81040789E4680125A8
:1012900064698D403D43058123600023A260636043
:1012A000F0BC01F061BA000070B5022300250446CD
:1012B0000370C0E90255C0E90455C564856180F832
:1012C000345001F0A9F863681B6823B12946204611
:1012D000BDE87040184770BD037880F85030052392
:1012E000037043681B6810B504460BB1042198478E
:1012F0000023A36010BD000090F8502043680270E6
:101300001B680BB1052118477047000070B590F8B5
:101310003430044613B1002380F8343004F1440221
:10132000204601F08BF963689B68B3B994F84430A8
:1013300013F0600535D00021204601F0DDFB0021CF
:10134000204601F0CFFB63681B6813B106212046DD
:101350009847062384F8343070BD2046984700280B
:10136000E4D0B4F84A30E26B9A4288BFE36394F960
:101370004430E56B002B4FF0200380F20381002DF9
:1013800000F0F280092284F8342083F311880021D0
:10139000D4E90E232046FFF775FF002383F311885D
:1013A000DAE794F8452003F07F0343EA022340F292
:1013B0000232934200F0C58021D8B3F5807F48D037
:1013C0000DD8012B3FD0022B00F09380002BB2D11F
:1013D00004F14C02A2630222E2632364C1E7B3F585
:1013E000817F00F09B80B3F5407FA4D194F8463014
:1013F000012BA0D1B4F84C3043F0020332E0B3F536
:10140000006F4DD017D8B3F5A06F31D0A3F5C063EE
:10141000012B90D8636894F846205E6894F84710D2
:10142000B4F848302046B047002884D04368A3630E
:101430000368E3631AE0B3F5106F36D040F602425A
:1014400093427FF478AF5C4BA3630223E3630023F2
:10145000C3E794F84630012B7FF46DAFB4F84C30FD
:1014600023F00203C4E90E55A4F84C30256478E754
:10147000B4F84430B3F5A06F0ED194F8463084F838
:101480004E30204601F020F863681B6813B101213B
:1014900020469847032323700023C4E90E339CE7BA
:1014A00004F14F03A3630123C3E72378042B10D176
:1014B000202383F311882046FFF7C8FE85F31188A7
:1014C0000321636884F84F5021701B680BB12046DC
:1014D000984794F84630002BDED084F84F30042330
:1014E000237063681B68002BD6D0022120469847E2
:1014F000D2E794F848301D0603F00F0120460AD5C4
:1015000001F08EF8012804D002287FF414AF2B4B91
:101510009AE72B4B98E701F075F8F3E794F846301B
:10152000002B7FF408AF94F8483013F00F01B3D0CC
:101530001A06204602D501F0F3FAADE701F0E6FA0B
:10154000AAE794F84630002B7FF4F5AE94F84830C3
:1015500013F00F01A0D01B06204602D501F0CCFAF3
:101560009AE701F0BFFA97E7142284F8342083F356
:1015700011882B462A4629462046FFF771FE85F33F
:101580001188E9E65DB1152284F8342083F31188CF
:101590000021D4E90E232046FFF762FEFDE60B2270
:1015A00084F8342083F311882B462A4629462046A6
:1015B000FFF768FEE3E700BFD8340008D034000826
:1015C000D434000838B590F834300446002B3ED0AF
:1015D000063BDAB20F2A34D80F2B32D8DFE803F0FB
:1015E0003731310822323131313131313131373710
:1015F000C56BB0F84A309D4214D2C3681B8AB5FB54
:10160000F3F203FB12556DB9202383F311882B46A7
:101610002A462946FFF736FE85F311880A2384F807
:1016200034300EE0142384F83430202383F31188FF
:1016300000231A4619462046FFF712FE002383F3C3
:10164000118838BD036C03B198470023E7E70021F8
:10165000204601F051FA0021204601F043FA636868
:101660001B6813B10621204698470623D7E70000E0
:1016700010B590F83430142B044629D017D8062B17
:1016800005D001D81BB110BD093B022BFBD80021AE
:10169000204601F031FA0021204601F023FA636868
:1016A0001B6813B1062120469847062319E0152B25
:1016B000E9D10B2380F83430202383F311880023F1
:1016C0001A461946FFF7DEFD002383F31188DAE797
:1016D000C3689B695B68002BD5D1036C03B1984745
:1016E000002384F83430CEE7024B0022C3E90033F4
:1016F0009A60704794230020002303748268054B8E
:101700001B6899689142FBD25A680360426010607E
:10171000586070479423002008B5202383F3118874
:10172000037C032B05D0042B0DD02BB983F3118838
:1017300008BD436900221A604FF0FF334361FFF791
:10174000DBFF0023F2E7D0E9003213605A60F3E7D1
:10175000002303748268054B1B6899689142FBD88B
:101760005A680360426010605860704794230020FC
:10177000054B19690874186802681A60536018618B
:1017800001230374FEF7C2BD9423002030B54B1C27
:101790000B4D87B0044610D02B690A4A01A800F00F
:1017A00025F92046FFF7E4FF049B13B101A800F0E0
:1017B00059F92B69586907B030BDFFF7D9FFF8E731
:1017C000942300201917000838B50C4D41612B698E
:1017D00081689A689142044603D8BDE83840FFF713
:1017E0008BBF1846FFF7B4FF01232C610146237419
:1017F0002046BDE83840FEF789BD00BF9423002095
:10180000044B1A681B6990689B68984294BF00203B
:10181000012070479423002010B5084C23682069EC
:101820001A6822605460012223611A74FFF790FF46
:1018300001462069BDE81040FEF768BD94230020F2
:1018400008B5FFF7DDFF18B1BDE80840FFF7E4BFBA
:1018500008BD0000FFF7E0BFFEE7000010B50C4C2C
:10186000FFF742FF00F0B4F80A498022204600F05A
:101870003BF8012344F8180C037400F071FC0023BA
:1018800083F3118862B60448BDE8104000F04CB8FC
:10189000BC230020DC340008EC34000800F01CB944
:1018A000EFF3118020B9EFF30583202282F3118832
:1018B0007047000010B530B9EFF30584C4F3080495
:1018C00014B180F3118810BDFFF7BAFF84F31188BB
:1018D000F9E70000034A516853685B1A9842FBD845
:1018E000704700BF001000E0826002220282704751
:1018F0008368A3F17C0243F80C2C026943F83C2C6A
:10190000426943F8382C074A43F81C2CC26843F854
:10191000102C022203F8082C002203F8072CA3F154
:10192000180070472503000810B5202383F31188A1
:10193000FFF7DEFF00210446FFF746FF002383F395
:101940001188204610BD0000024B1B6958610F2012
:10195000FFF70EBF94230020202383F31188FFF7A5
:10196000F3BF000008B50146202383F31188082047
:10197000FFF70CFF002383F3118808BD49B1064B24
:1019800042681B6918605A60136043600420FFF7C7
:10199000FDBE4FF0FF30704794230020036898424B
:1019A00006D01A680260506059611846FFF7A4BE5D
:1019B0007047000038B504460D462068844200D1C7
:1019C00038BD036823605C604561FFF795FEF4E76E
:1019D000054B03F11402C3E905224FF0FF31002249
:1019E000C3E90712704700BF9423002070B51C4E56
:1019F000C0E9032305460C4601F090FA334653F83C
:101A0000142F9A420DD13062C5E901242A600A2CB4
:101A10002CBF00190A30C6E90555BDE8704001F039
:101A20006BBA316A431AE31838BF1C469368A34265
:101A300002D9081901F06EFA73699A6894420CD8B9
:101A40005A68AC602B606A6015609A685D60121B12
:101A50009A604FF0FF33F36170BD1B68A41AECE786
:101A60009423002038B51B4C636998420DD0D0E90F
:101A7000003213605A6000228168C2609A680A448A
:101A80009A604FF0FF33E36138BD2246036842F8A5
:101A9000143F002193425A60C16003D1BDE8384031
:101AA00001F032BA9A688168256A0A449A6001F0A6
:101AB00035FA63699A68411B8A42E5D9AB181D1A49
:101AC000092D206A98BF01F10A02BDE83840104490
:101AD00001F020BA942300202DE9F041184C002792
:101AE00004F11406656901F019FA236AAA68C11A9B
:101AF0008A4215D813442362D5E9003213605A6034
:101B00006369D5F80C80EF60B34201D101F0FCF9B4
:101B100087F311882869C047202383F31188E1E700
:101B20006169B14209D013441B1ABDE8F0410A2B88
:101B30002CBFC0180A3001F0EDB9BDE8F08100BF3C
:101B40009423002000207047FEE70000704700004B
:101B50004FF0FF307047000002290CD0032904D059
:101B60000129074818BF00207047032A05D80548F7
:101B700000EBC2007047044870470020704700BF68
:101B8000D0350008202200208435000870B59AB0B6
:101B90000546084601A9144600F0C2F801A8FFF75F
:101BA0009DF8431C5B00C5E9003400222370032329
:101BB0006370C6B201AB02341046D1B28E4204F15A
:101BC000020401D81AB070BD13F8011B04F8021CFE
:101BD00004F8010C0132F0E708B5202383F31188E3
:101BE0000348FFF779FA002383F3118808BD00BF8B
:101BF0005025002090F8443003F01F02012A07D13D
:101C000090F845200B2A03D10023C0E90E3315E0DC
:101C100003F06003202B08D1B0F848302BB990F8BE
:101C20004520212A03D81F2A04D8FFF737BA222AD1
:101C3000EBD0FAE7034A82630722C2630364012000
:101C4000704700BF1822002007B5052917D8DFE824
:101C500001F0191603191920202383F31188104A63
:101C600001900121FFF7D8FA01980E4A0221FFF7EF
:101C7000D3FA0D48FFF7FCF9002383F3118803B072
:101C80005DF804FB202383F311880748FFF7C6F9AA
:101C9000F2E7202383F311880348FFF7DDF9EBE730
:101CA00024350008483500085025002038B50C4D73
:101CB0000C4C0D492A4604F10800FFF767FF05F1B7
:101CC000CA0204F110000949FFF760FF05F5CA7266
:101CD00004F118000649BDE83840FFF757BF00BFC0
:101CE000182A002020220020043500080E350008A4
:101CF0001935000870B5044608460D46FEF7EEFF9C
:101D0000C6B22046013403780BB9184670BD32467E
:101D10002946FEF7CFFF0028F3D10120F6E70000A7
:101D20002DE9F04705460C46FEF7D8FF2B49C6B211
:101D30002846FFF7DFFF08B10636F6B228492846E5
:101D4000FFF7D8FF08B11036F6B2632E0BD8DFF8D4
:101D50008C80DFF88C90234FDFF894A02E7846B962
:101D60002670BDE8F08729462046BDE8F04701F01F
:101D700065BB252E2ED1072241462846FEF79AFF45
:101D800070B9194B224603F10C0153F8040B42F8C9
:101D9000040B8B42F9D11B78137007350D34DDE746
:101DA000082249462846FEF785FF98B90F4BA21C2A
:101DB000197809090232C95D02F8041C13F8011BE5
:101DC00001F00F015345C95D02F8031CF0D118342E
:101DD0000835C3E704F8016B0135BFE7F0350008AB
:101DE0001935000806360008F8350008107AFF1F7C
:101DF0001C7AFF1FBFF34F8F024AD368DB03FCD46A
:101E0000704700BF003C024008B5094B1B7873B90E
:101E1000FFF7F0FF074B1A69002ABFBF064A5A6056
:101E200002F188325A601A6822F480621A6008BD92
:101E3000762C0020003C02402301674508B50B4B7F
:101E40001B7893B9FFF7D6FF094B1A6942F000429D
:101E50001A611A6842F480521A601A6822F4805299
:101E60001A601A6842F480621A6008BD762C00205D
:101E7000003C02400B28F0B516D80C4C0C492378D6
:101E80007BB90C4D0E460C234FF0006255F8047BD5
:101E900046F8042B013B13F0FF033A44F6D101232B
:101EA000237051F82000F0BD0020FCE7A82C002092
:101EB000782C002018360008014B53F8200070479A
:101EC000183600080C2070470B2810B5044601D9BD
:101ED000002010BDFFF7CEFF064B53F82430184406
:101EE000C21A0BB90120F4E712680132F0D1043BA9
:101EF000F6E700BF183600080B2838B5044628D886
:101F0000FFF7CEFCFFF776FFFFF77EFF124AF323C1
:101F1000D360E300DBB243F4007343F002031361C8
:101F2000136943F48033136105462046FFF762FFCF
:101F3000FFF7A0FF094B53F8241000F0E9F82846FA
:101F4000FFF77CFFFFF7B6FC2046BDE83840FFF7FF
:101F5000BBBF002038BD00BF003C0240183600085F
:101F600012F001032DE9F04105460E4614464BD10F
:101F70008218B2F1016F61D8314B1B6813F0010375
:101F80005CD0304FFFF78CFCFFF73EFFF323FB6084
:101F9000FFF730FF314640F20128032C18D824F017
:101FA0000104284E0C446D1A40F20118A142336915
:101FB00005EB01072AD123F001033361FFF73EFF50
:101FC000FFF778FC0120BDE8F081043C0435E4E72C
:101FD000AB07E4D13B6923F440733B613B6943EABF
:101FE00008033B6151F8046B2E60BFF34F8FFFF77E
:101FF00001FF2B689E42E8D03B6923F001033B615F
:10200000FFF71CFFFFF756FC0020DCE723F44073CA
:102010003361336943EA080333610B883B80BFF3C4
:102020004F8FFFF7E7FE3F8831F8023BBFB2BB425C
:10203000BCD0336923F001033361E1E71846C2E7FE
:1020400000380240003C0240084908B50B7828B12E
:102050001BB9FFF7D9FE01230B7008BD002BFCD084
:10206000BDE808400870FFF7E9BE00BF762C0020ED
:1020700010B50244064BD2B2904200D110BD441CB0
:1020800000B253F8200041F8040BE0B2F4E700BFBF
:10209000502800400F4B30B51C6F240407D41C6F30
:1020A00044F400741C671C6F44F400441C670A4C21
:1020B000236843F4807323600244084BD2B29042F9
:1020C00000D130BD441C00B251F8045B43F82050ED
:1020D000E0B2F4E7003802400070004050280040B1
:1020E00007B5012201A90020FFF7C2FF019803B044
:1020F0005DF804FB13B50446FFF7F2FFA04205D0DC
:10210000012201A900200194FFF7C4FF02B010BD15
:1021100070470000034B1A681AB9034AD2F87428B2
:102120001A607047AC2C00200030024008B5FFF761
:10213000F1FF024B1868C0F3407008BDAC2C0020C2
:10214000EFF3098305494A6B22F001024A636833C1
:1021500083F30988002383F31188704700EF00E0C0
:10216000202080F3118862B60C4B0D4AD96821F407
:10217000E0610904090C0A43DA60D3F8FC2009493C
:1021800042F08072C3F8FC200A6842F001020A6043
:102190001022DA7783F82200704700BF00ED00E0DC
:1021A0000003FA05001000E010B5202383F3118826
:1021B0000E4B5B6813F4006314D0F1EE103AEFF3AA
:1021C0000984683C4FF08073E361094BDB6B236645
:1021D00084F30988FFF714FB10B1064BA36110BD0F
:1021E000054BFBE783F31188F9E700BF00ED00E042
:1021F00000EF00E0370300083A03000870470000D2
:10220000FEE700000A4B0B480B4A90420BD30B4BE6
:10221000DA1C121AC11E22F003028B4238BF0022C0
:102220000021FEF763BD53F8041B40F8041BECE7E4
:10223000B8370008A82D0020A82D0020A82D0020C8
:102240007047000070B5D0E915439E6800224FF03A
:10225000FF3504EB42135101D3F800090028BEBF3B
:10226000D3F8000940F08040C3F80009D3F8000B10
:102270000028BEBFD3F8000B40F08040C3F8000B2D
:10228000013263189642C3F80859C3F8085BE0D2DC
:102290004FF00113C4F81C3870BD00001D4B03EB58
:1022A00080022DE9F043D2F80CC05D6DDCF81420FB
:1022B000461CD2F800E005EB063605EB40185168E5
:1022C00071450AD3D5F83438012202FA00F023EA26
:1022D0000000C5F83408BDE8F083BCF81040AEEB50
:1022E0000103A34228BF2346D8F81849A4B2B3EB90
:1022F000840FF0D89468A4F1040959F8047F37607A
:10230000A4EB09071F44042FF7D81C440B44946026
:102310005360D4E7B02C0020890141F02001016115
:1023200003699B06FCD41220FFF7D4BA10B5054C04
:102330002046FEF753FF4FF0A0436365024BA365B1
:1023400010BD00BFB02C00206C36000870B50378BB
:10235000012B054650D12A4B446D98421BD1294B85
:102360005A6B42F080025A635A6D42F080025A65FD
:102370005A6D5A6942F080025A615A6922F080020D
:102380005A610E2143205B6900F0D4FB1E4BE360D1
:102390001E4BC4F800380023C4F8003EC02323605D
:1023A0006E6D4FF40413A3633369002BFCDA012331
:1023B00033610C20FFF78EFA3369DB07FCD412205F
:1023C000FFF788FA3369002BFCDA0026A66028465E
:1023D000FFF738FF6B68C4F81068DB68C4F814684E
:1023E000C4F81C684BB90A4BA3614FF0FF3363611B
:1023F000A36843F00103A36070BD064BF4E700BF80
:10240000B02C00200038024040140040030020029D
:10241000003C30C0083C30C0F8B5446D0546002192
:102420002046FFF779FFA96D00234FF001128F6856
:10243000C4F834384FF00066C4F81C284FF0FF3061
:1024400004EB431201339F42C2F80069C2F8006BEB
:10245000C2F80809C2F8080BF2D20B686A6DEB6586
:10246000636210231361166916F01006FBD1122067
:10247000FFF730FAD4F8003823F4FE63C4F80038CC
:10248000A36943F4402343F01003A3610923C4F874
:102490001038C4F814380A4BEB604FF0C043C4F84E
:1024A000103B084BC4F8003BC4F81069C4F800396D
:1024B000EB6D03F1100243F48013EA65A362F8BDEB
:1024C0004836000840800010426D90F84E10D2F857
:1024D000003823F4FE6343EA0113C2F80038704762
:1024E0002DE9F84300EB8103456DDA68166806F0C4
:1024F0000306731E022B05EB41130C4680460FFAB0
:1025000081F94FEA41104FF00001C3F8101B4FF062
:10251000010104F1100398BFB60401FA03F39169B5
:102520008EBF334E06F1805606F5004600293AD09C
:10253000578A04F15801490137436F50D5F81C18E8
:102540000B43C5F81C382B180021C3F81019536928
:102550000127611EA7409BB3138A928B9B08012A17
:1025600088BF5343D8F85C20981842EA034301F12E
:10257000400205EB8202C8F85C0021465360284601
:10258000FFF7CAFE08EB8900C3681B8A43EA84533D
:10259000483464011E432E51D5F81C381F43C5F83A
:1025A0001C78BDE8F88305EB4917D7F8001B21F428
:1025B0000041C7F8001BD5F81C1821EA0303C0E747
:1025C00004F13F0305EB83030A4A5A60284621467B
:1025D000FFF7A2FE05EB4910D0F8003923F40043C1
:1025E000C0F80039D5F81C3823EA0707D7E700BF41
:1025F0000080001000040002826D1268C265FFF7BF
:1026000021BE00005831436D49015B5813F400406E
:1026100004D013F4001F0CBF0220012070470000FB
:102620004831436D49015B5813F4004004D013F462
:10263000001F0CBF022001207047000000EB810149
:10264000CB68196A0B6813604B68536070470000D1
:1026500000EB810330B5DD68AA691368D36019B94E
:10266000402B84BF402313606B8A1468426D1C4466
:10267000013CB4FBF3F46343033323F0030302EBA5
:10268000411043EAC44343F0C043C0F8103B2B68F9
:1026900003F00303012B09B20ED1D2F8083802EB84
:1026A000411013F4807FD0F8003B14BF43F08053F7
:1026B00043F00053C0F8003B02EB4112D2F8003B5C
:1026C00043F00443C2F8003B30BD00002DE9F04167
:1026D000244D6E6D06EB40130446D3F8087BC3F817
:1026E000087B38070AD5D6F81438190706D505EB44
:1026F00084032146DB6828465B689847FA071FD5A4
:10270000D6F81438DB071BD505EB8403D968CCB9A0
:102710008B69488A5A68B2FBF0F600FB16228AB928
:102720001868DA6890420DD2121AC3E900242023F7
:1027300083F311880B482146FFF78AFF84F3118841
:10274000BDE8F081012303FA04F26B8923EA020356
:102750006B81CB68002BF3D021460248BDE8F041E5
:10276000184700BFB02C002000EB810370B5DD6876
:10277000436D6C692668E6604A0156BB1A444FF403
:102780000020C2F810092A6802F00302012A0AB2E6
:102790000ED1D3F8080803EB421410F4807FD4F86C
:1027A000000914BF40F0805040F00050C4F8000908
:1027B00003EB4212D2F8000940F00440C2F80009CD
:1027C000D3F83408012202FA01F10143C3F83418A6
:1027D00070BD19B9402E84BF4020206020682E8A29
:1027E0008419013CB4FBF6F440EAC44040F00050C8
:1027F0001A44C6E7F8B504461E48456D05EB441378
:10280000D3F80869C3F80869F10717D5D5F8103867
:10281000DA0713D500EB8403D9684B691F68DA68BF
:10282000974218D2D21B00271A605F60202383F3DF
:1028300011882146FFF798FF87F31188330617D5D3
:10284000D5F834280123A340134211D02046BDE817
:10285000F840FFF723BD012303FA04F2038923EABA
:10286000020303818B68002BE8D021469847E5E7F7
:10287000F8BD00BFB02C00202DE9F74F984C666DD5
:102880007569B3691D4015F48058756107D02046FD
:10289000FEF70AFD03B0BDE8F04FFFF785BC002D41
:1028A00012DAD6F8003E8E489F071EBFD6F8003ECB
:1028B00023F00303C6F8003ED6F8043823F00103E2
:1028C000C6F80438FEF718FD280505D58448FFF73B
:1028D000B9FC8348FEF700FDA9040CD5D6F80838EA
:1028E00013F0060FF36823F470530CBF43F4105336
:1028F00043F4A053F3602A0704D56368DB680BB187
:1029000077489847EB0274D4AF0227D5D4F8549097
:10291000DFF8CCB100274FF0010A09EB4712D2F8DB
:10292000003B03F44023B3F5802F11D1D2F8003BD4
:10293000002B0DDA62890AFA07F322EA03036381A6
:1029400004EB8703DB68DB6813B1394658469847C8
:10295000A36D01379B68FFB29F42DED9E80617D509
:10296000676D3A6AC2F30A1002F00F0302F4F01224
:10297000B2F5802F00F08880B2F5402F08D104EB2B
:1029800083030022DB681B6A07F5805790426DD1F4
:102990002903D6F8184813D5E20302D50020FFF723
:1029A00095FEA30302D50120FFF790FE670302D531
:1029B0000220FFF78BFE260302D50320FFF786FED9
:1029C0006D037FF567AFE00702D50020FFF712FF28
:1029D000A10702D50120FFF70DFF620702D50220F3
:1029E000FFF708FF23077FF555AF0320FFF702FF2E
:1029F00050E7636DDFF8E8B0019300274FF0010A5C
:102A0000A36D9B685FFA87F999453FF67DAF019BFF
:102A100003EB4913D3F8002902F44022B2F5802FCA
:102A200022D1D3F80029002A1EDAD3F8002942F077
:102A30009042C3F80029D3F80029002AFBDB606D1F
:102A40004946FFF769FC22890AFA09F322EA0303DF
:102A5000238104EB8903DB689B6813B14946584620
:102A600098474846FFF71AFC0137C9E7910708BFA6
:102A7000D7F80080072A98BF03F8018B02F1010202
:102A800098BF4FEA182881E7023304EB830207F569
:102A900080575268D2F818C0DCF80820DCE9001C26
:102AA000A1EB0C0C002188420AD104EB830463687B
:102AB0009B699A6802449A605A6802445A6067E7C0
:102AC00011F0030F08BFD7F800808C4588BF02F8CB
:102AD000018B01F1010188BF4FEA1828E3E700BF2D
:102AE000B02C0020436D03EB4111D1F8003B43F4BF
:102AF0000013C1F8003B7047436D03EB4111D1F85F
:102B0000003943F40013C1F800397047436D03EBFB
:102B10004111D1F8003B23F40013C1F8003B70478A
:102B2000436D03EB4111D1F8003923F40013C1F8D0
:102B30000039704700F1604303F561430901C9B2F0
:102B400083F80013012200F01F039A4043099B0001
:102B500003F1604303F56143C3F880211A607047B5
:102B600030B5039C0172043304FB0325C0E906530E
:102B7000049B03630021059BC160C0E90000C0E91C
:102B80000422C0E90842C0E90A11436330BD0000D5
:102B9000416A0022C0E90411C0E90A22C2606FF054
:102BA0000101FEF707BF0000D0E90432934201D1D2
:102BB000C2680AB9181D7047002070470369196080
:102BC000C2680132C260C2691344826903619342E0
:102BD00024BF436A03610021FEF7E0BE38B5044616
:102BE0000D46E3683BB16269131D1268A36213448A
:102BF000E362002007E0237A33B929462046FEF736
:102C0000BDFE0028EDDA38BD6FF00100FBE70000E3
:102C1000C368C269013BC36043691344826943616D
:102C2000934224BF436A436100238362036B03B171
:102C30001847704770B52023044683F31188866ACD
:102C40003EB9FFF7CBFF054618B186F31188284639
:102C500070BDA36AE26A13F8015BA362934202D3D8
:102C60002046FFF7D5FF002383F31188EFE700002C
:102C70002DE9F84F04460E46174698464FF02009B6
:102C800089F311880025AA46D4F828B0BBF1000FBB
:102C900009D141462046FFF7A1FF20B18BF31188EF
:102CA0002846BDE8F88FD4E90A12A7EB050B521AA3
:102CB000934528BF9346BBF1400F1BD9334601F122
:102CC000400251F8040B43F8040B9142F9D1A36A76
:102CD00040334036A3624035D4E90A239A4202D3F6
:102CE0002046FFF795FF8AF31188BD42D8D289F3B9
:102CF0001188C9E730465A46FDF7D2FFA36A5B4404
:102D00005E44A3625D44E7E710B5029C01720433A0
:102D100004FB0321C0E906130023C0E90A33039B27
:102D20000363049BC460C0E90000C0E90422C0E959
:102D30000842436310BD0000026AC260426AC0E9F3
:102D400004220022C0E90A226FF00101FEF732BE20
:102D5000D0E904239A4201D1C26822B9184650F83A
:102D6000043B0B607047002070470000C368C269D5
:102D70000133C3604369134482694361934224BFB2
:102D8000436A43610021FEF709BE000038B50446DE
:102D90000D46E3683BB123691A1DA262E269134440
:102DA000E362002007E0237A33B929462046FEF784
:102DB000E5FD0028EDDA38BD6FF00100FBE700000B
:102DC00003691960C268013AC260C269134482692A
:102DD0000361934224BF436A036100238362036B50
:102DE00003B118477047000070B520230D46044614
:102DF000114683F31188866A2EB9FFF7C7FF10B119
:102E000086F3118870BDA36A1D70A36AE26A01335C
:102E10009342A36204D3E16920460439FFF7D0FF4F
:102E2000002080F31188EDE72DE9F84F04460D46A8
:102E3000904699464FF0200A8AF311880026B3463F
:102E4000A76A4FB949462046FFF7A0FF20B187F394
:102E500011883046BDE8F88FD4E90A073A1AA8EB82
:102E60000607974228BF1746402F1BD905F140039C
:102E700055F8042B40F8042B9D42F9D1A36A403346
:102E8000A3624036D4E90A239A4204D3E16920467A
:102E90000439FFF795FF8BF311884645D9D28AF3A1
:102EA0001188CDE729463A46FDF7FAFEA36A3B446E
:102EB0003D44A3623E44E5E7D0E904239A4217D19A
:102EC000C3689BB1836A8BB1043B9B1A0ED013601D
:102ED000C368013BC360C3691A44836902619A42B3
:102EE00024BF436A036100238362012318467047AD
:102EF0000023FBE700F088B84FF0804300225863BE
:102F00001A610222DA6070474FF080430022DA60D3
:102F1000704700004FF08043586370474FF0804384
:102F2000586A70474B6843608B688360CB68C360A6
:102F30000B6943614B6903628B6943620B680360F1
:102F40007047000008B5264B26481A6940F2FF1169
:102F50000A431A611A6922F4FF7222F001021A610F
:102F60001A691A6B0A431A631A6D0A431A651E4AD4
:102F70001B6D1146FFF7D6FF02F11C0100F58060C2
:102F8000FFF7D0FF02F1380100F58060FFF7CAFFBC
:102F900002F1540100F58060FFF7C4FF02F17001F7
:102FA00000F58060FFF7BEFF02F18C0100F5806044
:102FB000FFF7B8FF02F1A80100F58060FFF7B2FF4C
:102FC00002F1C40100F58060FFF7ACFF02F1E001FF
:102FD00000F58060FFF7A6FFBDE8084000F09AB852
:102FE00000380240000002407836000808B500F0C2
:102FF00007FAFEF733FCFFF78DF8BDE80840FEF74F
:1030000055BE000070470000104B1A6C42F00102E0
:103010001A641A6E42F001021A660D4A1B6E93681A
:1030200043F0010393604FF0804353229A624FF0C4
:10303000FF32DA6200229A615A63DA605A60012232
:103040005A6108211A601C20FFF774BD0038024045
:10305000002004E04FF0804208B51169D3680B40AE
:10306000D9B2C9439B07116107D5202383F3118887
:10307000FEF714FC002383F3118808BD08B5FFF7A1
:10308000E9FFBDE80840FFF78FB800001F4B1A6941
:103090006FEAC2526FEAD2521A611A69C2F3080289
:1030A0001A614FF0FF301A695A69586100215A6954
:1030B00059615A691A6A62F080521A621A6A02F0F9
:1030C00080521A621A6A5A6A58625A6A59625A6A6D
:1030D0001A6C42F080521A641A6E42F080521A66DC
:1030E0001A6E0B4A106840F480701060186F00F47C
:1030F0004070B0F5007F1EBF4FF48030186719672D
:10310000536823F40073536000F05AB9003802404A
:1031100000700040334B4FF080521A64324A4FF433
:10312000404111601A6842F001021A601A68910762
:10313000FCD59A6822F003029A602A4B9A6812F032
:103140000C02FBD1196801F0F90119609A601A6844
:1031500042F480321A601A689203FCD55A6F42F02A
:1031600001025A671F4B5A6F9007FCD51F4A5A60DD
:103170001A6842F080721A601B4A53685904FCD5E1
:10318000184B1A689201FCD5194A9A60194B1A68B3
:10319000194B9A42194B21D1194A1168194A914287
:1031A0001CD140F205121A60144A136803F00F0391
:1031B000052BFAD10B4B9A6842F002029A609A688A
:1031C00002F00C02082AFAD15A6C42F480425A6486
:1031D0005A6E42F480425A665B6E704740F2057246
:1031E000E1E700BF0038024000700040085440078B
:1031F00000948838002004E011640020003C024064
:1032000000ED00E041C20F41084A08B5516913685A
:103210000B4003F00103536123B1054A13680BB15E
:1032200050689847BDE80840FEF7BEBF003C01402B
:10323000282D0020084A08B5516913680B4003F097
:103240000203536123B1054A93680BB1D0689847D4
:10325000BDE80840FEF7A8BF003C0140282D002033
:10326000084A08B5516913680B4003F00403536121
:1032700023B1054A13690BB150699847BDE808406E
:10328000FEF792BF003C0140282D0020084A08B5F7
:10329000516913680B4003F00803536123B1054AD9
:1032A00093690BB1D0699847BDE80840FEF77CBF31
:1032B000003C0140282D0020084A08B551691368D8
:1032C0000B4003F01003536123B1054A136A0BB19D
:1032D000506A9847BDE80840FEF766BF003C0140D1
:1032E000282D0020174B10B55A691C68144004F4AF
:1032F00078725A61A30604D5134A936A0BB1D06A57
:103300009847600604D5104A136B0BB1506B984771
:10331000210604D50C4A936B0BB1D06B9847E2059C
:1033200004D5094A136C0BB1506C9847A30504D51A
:10333000054A936C0BB1D06C9847BDE81040FEF77E
:1033400033BF00BF003C0140282D00201A4B10B5B0
:103350005A691C68144004F47C425A61620504D521
:10336000164A136D0BB1506D9847230504D5134AC7
:10337000936D0BB1D06D9847E00404D50F4A136EDE
:103380000BB1506E9847A10404D50C4A936E0BB153
:10339000D06E9847620404D5084A136F0BB1506F82
:1033A0009847230404D5054A936F0BB1D06F984713
:1033B000BDE81040FEF7F8BE003C0140282D00207B
:1033C000062108B50846FFF7B5FB06210720FFF7E1
:1033D000B1FB06210820FFF7ADFB06210920FFF70E
:1033E000A9FB06210A20FFF7A5FB06211720FFF7FE
:1033F000A1FBBDE8084006212820FFF79BBB000089
:1034000008B5FFF743FE00F00BF8FDF7E5FEFDF70A
:10341000BDFDFFF7F7FDBDE80840FFF76BBD0000FD
:103420000023054A19460133102BC2E9001102F1AD
:103430000802F8D1704700BF282D0020034611F87C
:10344000012B03F8012B002AF9D1704753544D3357
:1034500032463F3F3F00000053544D333246343034
:10346000780053544D3332463432780053544D3340
:103470003246343436585800000000004C340008FE
:103480003F00000013040000583400083F00000013
:1034900019040000623400083F000000210400000D
:1034A0006C3400083F00000000000000090F000815
:1034B000F50E0008310F00081D0F0008290F000845
:1034C000150F0008010F0008ED0E00083D0F000861
:1034D0000000000001000000000000006D61696E46
:1034E0000000000069646C6500000000E43400081E
:1034F000D8230020502500200100000059180008A2
:10350000000000004172647550696C6F74002542C0
:103510004F415244252D424C002553455249414CC0
:103520002500000002000000000000002511000836
:103530009111000840004000E8290020F8290020EF
:103540000200000000000000030000000000000076
:10355000D51100080000000010000000082A00201B
:10356000000000000100000000000000B02C00205E
:1035700001010200491C0008591B0008F51B000846
:10358000D91B0008430000008C35000809024300E5
:10359000020100C0320904000001020201000524FA
:1035A0000010010524010001042402020524060084
:1035B00001070582030800FF09040100020A000058
:1035C00000070501024000000705810240000000DD
:1035D00012000000D835000812011001020000405E
:1035E000091241570002010203010000040309040B
:1035F00025424F41524425007370656564796265C8
:103600006566347633003031323334353637383905
:103610004142434445460000004000000040000095
:103620000040000000400000000001000000020017
:103630000000020000000200000002000000020082
:103640000000020000000200000000000D1300084E
:10365000C51500087116000840004000102D00201C
:10366000102D002001000000202D0020800000000F
:103670004001000003000000000180420000000043
:10368000AAAAAAAA00010040FFFF00000000000053
:1036900000A00A000000000100000000AAAAAAAAD7
:1036A00000000001FFFF000000000000000000001B
:1036B0000000010000000000AAAAAAAA0000000061
:1036C000FFFE0000000000000000000000000000FD
:1036D00000000000AAAAAAAA00000000FFFF000044
:1036E00000000000000000000000000000000000DA
:1036F000AAAAAAAA00000000FFFF00000000000024
:10370000000000000000000000000000AAAAAAAA11
:1037100000000000FFFF00000000000000000000AB
:103720000000000000000000AAAAAAAA00000000F1
:10373000FFFF00000000000000000000000000008B
:10374000000000000A00000000000000030000006C
:103750000000000000000000000000000000000069
:103760000000000000000000000000000000000059
:1037700000000000000000003A040000000000000B
:1037800000400F0000000000FF009600000000084D
:10379000009600000000080004000000EC3500085E
:1037A0000000000000000000000000000000000019
:1037B0000000000000000000FFFFFFFFFFFFFFFF11
:1037C000FFFFFFFFFFFFFFFFFFFFFFFFFFFFFFFF09
:1037D000FFFFFFFFFFFFFFFFFFFFFFFFFFFFFFFFF9
:1037E000FFFFFFFFFFFFFFFFFFFFFFFFFFFFFFFFE9
:1037F000FFFFFFFFFFFFFFFFFFFFFFFFFFFFFFFFD9
:10C000000006002099D20008C577080821770808A3
:10C010008D77080821770808597708089BD200080F
:10C020009BD200089BD200089BD200086DA90A0889
:10C030009BD200089BD200089BD200089BD200082C
:10C040009BD200089BD200089BD200089BD200081C
:10C050009BD200089BD2000805B50A082DB50A0836
:10C0600055B50A087DB50A08A5B50A08055E0A088F
:10C070002D5E0A08595E0A08855E0A08B15E0A0844
:10C08000D95E0A08055F0A08895D0A089BD2000884
:10C090009BD200089BD200089BD20008CDB50A08AD
:10C0A0009BD200089BD200089BD200089BD20008BC
:10C0B0009BD2000819B70A082DB70A089BD20008BE
:10C0C0009BD2000891640A0839660A089BD20008CE
:10C0D0009BD20008A1B60A08B5B60A08C9B60A0874
:10C0E00031B60A089BD200089BD2000851B70A0853
:10C0F00055B70A0869B70A086DB70A08315F0A0818
:10C100009BD200089BD2000841B70A089BD20008C6
:10C11000DDB60A08F1B60A089BD200089BD20008D7
:10C120005D5F0A08855F0A08B15F0A08DD5F0A08DB
:10C1300009600A089BD200089BD200089BD2000825
:10C140009BD200089BD200089BD2000899B00A0835
:10C1500031600A085D600A0889600A0805B70A08A4
:10C160009BD200089BD200089BD200089BD20008FB
:10C170009BD200089BD200089BD200089BD20008EB
:10C180009BD200089BD200089BD200089BD20008DB
:10C190009BD200089BD200089BD200089BD20008CB
:10C1A0009BD200089BD200089BD200089BD20008BB
:10C1B0009BD200089BD200089BD200089BD20008AB
:10C1C0009BD200089BD200089BD200089BD200089B
:10C1D0009BD200089BD200089BD200089BD200088B
:10C1E00049020108B5DD0108914303088DF10408F7
:10C1F00095F7040829660508C1C6050885CE050817
:10C20000BDD1050871320608DD51060801E40608B3
:10C21000514E0708A95B07088D6908084D6E08088C
:10C220007D49090895AA0908ADD0090855DB090818
:10C2300065070A082D0D0A08000000000000000034
:10C2400081F0004102E000BF83F0004330B54FEAC7
:10C2500041044FEA430594EA050F08BF90EA020F34
:10C260001FBF54EA000C55EA020C7FEA645C7FEAC7
:10C27000655C00F0E2804FEA5454D4EB5555B8BFEA
:10C280006D420CDD2C4480EA020281EA030382EA5B
:10C29000000083EA010180EA020281EA0303362DED
:10C2A00088BF30BD11F0004F4FEA01314FF4801CC0
:10C2B0004CEA113102D0404261EB410113F0004FD2
:10C2C0004FEA03334CEA133302D0524263EB430389
:10C2D00094EA050F00F0A780A4F10104D5F1200E27
:10C2E0000DDB02FA0EFC22FA05F2801841F1000182
:10C2F00003FA0EF2801843FA05F359410EE0A5F156
:10C3000020050EF1200E012A03FA0EFC28BF4CF086
:10C31000020C43FA05F3C01851EBE37101F000453C
:10C3200007D54FF0000EDCF1000C7EEB00006EEB49
:10C330000101B1F5801F1BD3B1F5001F0CD34908D3
:10C340005FEA30004FEA3C0C04F101044FEA44522A
:10C3500012F5800F80F09A80BCF1004F08BF5FEAB1
:10C36000500C50F1000041EB045141EA050130BD91
:10C370005FEA4C0C404141EB0101013C28BFB1F5A3
:10C38000801FE9D291F0000F04BF01460020B1FAEE
:10C3900081F308BF2033A3F10B03B3F120020CDAC1
:10C3A0000C3208DD02F1140CC2F10C0201FA0CF09F
:10C3B00021FA02F10CE002F11402D8BFC2F1200C04
:10C3C00001FA02F120FA0CFCDCBF41EA0C019040BA
:10C3D000E41AA2BF01EB0451294330BD6FEA040403
:10C3E0001F3C1CDA0C340EDC04F11404C4F12002EE
:10C3F00020FA04F001FA02F340EA030021FA04F300
:10C4000045EA030130BDC4F10C04C4F1200220FA56
:10C4100002F001FA04F340EA0300294630BD21FA94
:10C4200004F0294630BD94F0000F83F4801306BF5A
:10C4300081F480110134013D4EE77FEA645C18BF4E
:10C440007FEA655C29D094EA050F08BF90EA020FE5
:10C4500005D054EA000C04BF1946104630BD91EADD
:10C46000030F1EBF0021002030BD5FEA545C05D1E0
:10C470004000494128BF41F0004130BD14F580041F
:10C480003CBF01F5801130BD01F0004545F0FE4193
:10C4900041F470014FF0000030BD7FEA645C1ABFC8
:10C4A000194610467FEA655C1CBF0B46024650EAFF
:10C4B000013406BF52EA033591EA030F41F400212B
:10C4C00030BD00BF90F0000F04BF0021704730B5B1
:10C4D0004FF4806404F132044FF000054FF0000186
:10C4E00050E700BF90F0000F04BF0021704730B547
:10C4F0004FF4806404F1320410F0004548BF40421C
:10C500004FF000013EE700BF42004FEAE2014FEA70
:10C5100031014FEA02701FBF12F07F4393F07F4F4B
:10C5200081F06051704732F07F4208BF704793F04E
:10C530007F4F04BF41F40021704730B54FF4607461
:10C5400001F0004521F000411CE700BF50EA010264
:10C5500008BF704730B54FF000050AE050EA01020D
:10C5600008BF704730B511F0004502D5404261EB7D
:10C5700041014FF4806404F132045FEA915C3FF4BE
:10C58000D8AE4FF003025FEADC0C18BF03325FEA5B
:10C59000DC0C18BF033202EBDC02C2F1200300FA0C
:10C5A00003FC20FA02F001FA03FE40EA0E0021FA31
:10C5B00002F11444BDE600BF70B54FF0FF0C4CF41F
:10C5C000E06C1CEA11541DBF1CEA135594EA0C0FD1
:10C5D00095EA0C0F00F0DEF82C4481EA030621EA0C
:10C5E0004C5123EA4C5350EA013518BF52EA033547
:10C5F00041F4801143F4801338D0A0FB02CE4FF0F9
:10C600000005E1FB02E506F00042E0FB03E54FF028
:10C610000006E1FB03569CF0000F18BF4EF0010E20
:10C62000A4F1FF04B6F5007F64F5407404D25FEA1C
:10C630004E0E6D4146EB060642EAC62141EA5551CF
:10C640004FEAC52040EA5E504FEACE2EB4F1FD0C11
:10C6500088BFBCF5E06F1ED8BEF1004F08BF5FEA8F
:10C66000500E50F1000041EB045170BD06F0004641
:10C6700046EA010140EA020081EA0301B4EB5C04EE
:10C68000C2BFD4EB0C0541EA045170BD41F48011E6
:10C690004FF0000E013C00F3AB8014F1360FDEBF0B
:10C6A000002001F0004170BDC4F10004203C35DAE7
:10C6B0000C341BDC04F11404C4F1200500FA05F36A
:10C6C00020FA04F001FA05F240EA020001F000420B
:10C6D00021F0004110EBD37021FA04F642EB060181
:10C6E0005EEA430E08BF20EAD37070BDC4F10C04AB
:10C6F000C4F1200500FA04F320FA05F001FA04F26F
:10C7000040EA020001F0004110EBD37041F100015A
:10C710005EEA430E08BF20EAD37070BDC4F1200565
:10C7200000FA05F24EEA020E20FA04F301FA05F2CD
:10C7300043EA020321FA04F001F0004121FA04F275
:10C7400020EA020000EBD3705EEA430E08BF20EA45
:10C75000D37070BD94F0000F0FD101F0004640007F
:10C7600041EB010111F4801F08BF013CF7D041EA01
:10C77000060195F0000F18BF704703F00046520005
:10C7800043EB030313F4801F08BF013DF7D043EAD6
:10C790000603704794EA0C0F0CEA135518BF95EA8C
:10C7A0000C0F0CD050EA410618BF52EA4306D1D113
:10C7B00081EA030101F000414FF0000070BD50EA32
:10C7C000410606BF1046194652EA430619D094EABC
:10C7D0000C0F02D150EA013613D195EA0C0F05D1A6
:10C7E00052EA03361CBF104619460AD181EA0301FA
:10C7F00001F0004141F0FE4141F470014FF00000B2
:10C8000070BD41F0FE4141F4780170BD70B54FF04C
:10C81000FF0C4CF4E06C1CEA11541DBF1CEA1355CC
:10C8200094EA0C0F95EA0C0F00F0A7F8A4EB0504AE
:10C8300081EA030E52EA03354FEA013100F08880A5
:10C840004FEA03334FF0805545EA131343EA12636E
:10C850004FEA022245EA111545EA10654FEA002623
:10C860000EF000419D4208BF964244F1FD0404F5DC
:10C87000407402D25B084FEA3202B61A65EB030538
:10C880005B084FEA32024FF480104FF4002CB6EBF5
:10C89000020E75EB030E22BFB61A754640EA0C0075
:10C8A0005B084FEA3202B6EB020E75EB030E22BFB5
:10C8B000B61A754640EA5C005B084FEA3202B6EBF6
:10C8C000020E75EB030E22BFB61A754640EA9C00B5
:10C8D0005B084FEA3202B6EB020E75EB030E22BF85
:10C8E000B61A754640EADC0055EA060E18D04FEA43
:10C8F000051545EA16754FEA06164FEAC30343EAE3
:10C9000052734FEAC2025FEA1C1CC0D111F4801FAF
:10C910000BD141EA00014FF000004FF0004CB6E7A8
:10C9200011F4801F04BF01430020B4F1FD0C88BF47
:10C93000BCF5E06F3FF6AFAEB5EB030C04BFB6EB52
:10C94000020C5FEA500C50F1000041EB045170BD45
:10C950000EF0004E4EEA113114EB5C04C2BFD4EB72
:10C960000C0541EA045170BD41F480114FF0000EF6
:10C97000013C90E645EA060E8DE60CEA135594EA72
:10C980000C0F08BF95EA0C0F3FF43BAF94EA0C0F75
:10C990000AD150EA01347FF434AF95EA0C0F7FF4EA
:10C9A00025AF104619462CE795EA0C0F06D152EA3E
:10C9B00003353FF4FDAE1046194622E750EA410622
:10C9C00018BF52EA43067FF4C5AE50EA41047FF433
:10C9D0000DAF52EA43057FF4EBAE12E74FF0FF3C98
:10C9E00006E000BF4FF0010C02E000BF4FF0010C69
:10C9F0004DF804CD4FEA410C7FEA6C5C4FEA430CE2
:10CA000018BF7FEA6C5C1BD001B050EA410C0CBF30
:10CA100052EA430C91EA030F02BF90EA020F002092
:10CA2000704710F1000F91EA030F58BF994208BFF9
:10CA300090422CBFD8176FEAE37040F001007047B6
:10CA40004FEA410C7FEA6C5C02D150EA013C07D10D
:10CA50004FEA430C7FEA6C5CD6D152EA033CD3D058
:10CA60005DF8040B704700BF8446104662468C4652
:10CA70001946634600E000BF01B5FFF7B7FF002885
:10CA800048BF10F1000F01BD4DF808EDFFF7F4FFAE
:10CA90000CBF012000205DF808FB00BF4DF808ED39
:10CAA000FFF7EAFF34BF012000205DF808FB00BF5C
:10CAB0004DF808EDFFF7E0FF94BF012000205DF87E
:10CAC00008FB00BF4DF808EDFFF7CEFF94BF012033
:10CAD00000205DF808FB00BF4DF808EDFFF7C4FF2C
:10CAE00034BF012000205DF808FB00BF4FEA410C75
:10CAF0007FEA6C5C02D150EA013C0AD14FEA430C58
:10CB00007FEA6C5C02D152EA033C02D14FF0000094
:10CB100070474FF0010070474FEA410212F50012D2
:10CB200015D211D56FF47873B3EB625212D94FEA74
:10CB3000C12343F0004343EA505311F0004F23FA5E
:10CB400002F018BF404270474FF00000704750EAB3
:10CB5000013005D111F0004008BF6FF00040704770
:10CB60004FF00000704700BF4A0011D212F50012CA
:10CB700011D20DD56FF47873B3EB62520ED44FEA35
:10CB8000C12343F0004343EA505323FA02F07047B5
:10CB90004FF00000704750EA013002D14FF0FF30F3
:10CBA00070474FF0000070474FEA4102B2F1E04396
:10CBB00024BFB3F5001CDCF1FE5C0DD901F0004C84
:10CBC0004FEAC0024CEA5070B2F1004F40EB8300D4
:10CBD00008BF20F00100704711F0804F21D113F100
:10CBE0003872BCBF01F00040704741F480114FEA39
:10CBF0005252C2F11802C2F1200C10FA0CF320FAC2
:10CC000002F018BF40F001004FEAC1234FEAD323DE
:10CC100003FA0CFC40EA0C0023FA02F34FEA430348
:10CC2000CCE77FEA625307D150EA01331EBF4FF0D1
:10CC3000FE4040F44000704701F0004040F0FE40EC
:10CC400040F40000704700BF80F0004002E000BFE9
:10CC500081F0004142001FBF5FEA410392EA030FE7
:10CC60007FEA226C7FEA236C6AD04FEA1262D2EB31
:10CC70001363C1BFD218414048404140B8BF5B4236
:10CC8000192B88BF704710F0004F40F4000020F0CF
:10CC90007F4018BF404211F0004F41F4000121F0E5
:10CCA0007F4118BF494292EA030F3FD0A2F101022F
:10CCB00041FA03FC10EB0C00C3F1200301FA03F16D
:10CCC00000F0004302D5494260EB4000B0F5000F90
:10CCD00013D3B0F1807F06D340084FEA310102F14F
:10CCE0000102FE2A51D2B1F1004F40EBC25008BF01
:10CCF00020F0010040EA03007047490040EB0000CB
:10CD0000013A28BFB0F5000FEDD2B0FA80FCACF1CB
:10CD1000080CB2EB0C0200FA0CF0AABF00EBC250F8
:10CD200052421843BCBFD0401843704792F0000FE6
:10CD300081F4000106BF80F400000132013BB5E739
:10CD40004FEA41037FEA226C18BF7FEA236C21D0AF
:10CD500092EA030F04D092F0000F08BF0846704714
:10CD600090EA010F1CBF0020704712F07F4F04D1E2
:10CD7000400028BF40F00040704712F100723CBFF5
:10CD800000F50000704700F0004343F0FE4040F41F
:10CD9000000070477FEA226216BF08467FEA2363DD
:10CDA0000146420206BF5FEA412390EA010F40F4C8
:10CDB000800070474FF0000304E000BF10F0004314
:10CDC00048BF40425FEA000C08BF704743F09643FB
:10CDD00001464FF000001CE050EA010208BF704716
:10CDE0004FF000030AE000BF50EA010208BF70479D
:10CDF00011F0004302D5404261EB41015FEA010CB2
:10CE000002BF84460146002043F0B64308BFA3F1A9
:10CE10008053A3F50003BCFA8CF2083AA3EBC2538B
:10CE200010DB01FA02FC634400FA02FCC2F12002AA
:10CE3000BCF1004F20FA02F243EB020008BF20F0E1
:10CE40000100704702F1200201FA02FCC2F1200247
:10CE500050EA4C0021FA02F243EB020008BF20EA3C
:10CE6000DC7070477BB972B90029BEBF00204FF05B
:10CE7000004106E008BF00281CBF6FF000414FF0E2
:10CE8000FF3000F007BAADF1080C6DE904CE0029BF
:10CE900009DB002B1ADB00F095F8DDF804E0DDE992
:10CEA000022304B07047404261EB4101002B1BDBC1
:10CEB00000F088F8DDF804E0DDE9022304B0404228
:10CEC00061EB4101524263EB43037047524263EB13
:10CED000430300F077F8DDF804E0DDE9022304B055
:10CEE000404261EB41017047524263EB430300F063
:10CEF00069F8DDF804E0DDE9022304B0524263EB97
:10CF00004303704753B94AB9002908BF00281CBF22
:10CF10004FF0FF314FF0FF3000F0BCB9ADF1080C1D
:10CF20006DE904CE00F04EF8DDF804E0DDE90223FF
:10CF300004B07047430803F05533C01A830803F068
:10CF4000333300F03330184400EB101000F00F3092
:10CF500000EB002000EB0040000E704707EE900A47
:10CF6000F5EEC07AF1EE10FA01D400F00BB8F1EE54
:10CF7000677A08B517EE900A00F004F8404261EBBA
:10CF8000410108BDD0B5FFF7BFFA0C4B00220646A1
:10CF90000F46FFF711FBFFF7E7FD0446FFF792FA94
:10CFA000074B0022FFF708FB02460B463046394686
:10CFB000FFF74AF9FFF7D8FD2146D0BD0000F03D4C
:10CFC0000000F0412DE9F047089D04468E46002BF5
:10CFD0004DD18A42944669D9B2FA82F252B101FA2D
:10CFE00002F3C2F1200120FA01F10CFA02FC41EA3D
:10CFF000030E94404FEA1C48210CBEFBF8F61FFAC2
:10D000008CF708FB16E341EA034306FB07F199425C
:10D010000AD91CEB030306F1FF3080F01F8199420F
:10D0200040F21C81023E63445B1AA4B2B3FBF8F0E9
:10D0300008FB103344EA034400FB07F7A7420AD970
:10D040001CEB040400F1FF3380F00A81A74240F298
:10D0500007816444023840EA0640E41B00261DB103
:10D06000D4400023C5E900433146BDE8F0878B4238
:10D0700009D9002D00F0EF800026C5E900013046F7
:10D080003146BDE8F087B3FA83F6002E4AD18B42D1
:10D0900002D3824200F2F980841A61EB030301207B
:10D0A0009E46002DE0D0C5E9004EDDE702B9FFDE67
:10D0B000B2FA82F2002A40F09280A1EB0C014FEA12
:10D0C0001C471FFA8CFE0126200CB1FBF7F307FB6F
:10D0D000131140EA01410EFB03F0884208D91CEB12
:10D0E000010103F1FF3802D2884200F2CB804346AF
:10D0F000091AA4B2B1FBF7F007FB101144EA01448E
:10D100000EFB00FEA64508D91CEB040400F1FF311C
:10D1100002D2A64500F2BB800846A4EB0E0440EA0A
:10D1200003409CE7C6F12007B34022FA07FC4CEA13
:10D13000030C20FA07F401FA06F31C43F9404FEA06
:10D140001C4900FA06F3B1FBF9F8200C1FFA8CFE1B
:10D1500009FB181140EA014108FB0EF0884202FA6F
:10D1600006F20BD91CEB010108F1FF3A80F0888030
:10D17000884240F28580A8F102086144091AA4B2ED
:10D18000B1FBF9F009FB101144EA014100FB0EFE6E
:10D190008E4508D91CEB010100F1FF346CD28E459D
:10D1A0006AD90238614440EA0840A0FB0294A1EB2E
:10D1B0000E01A142C846A64656D353D05DB1B3EB8B
:10D1C000080261EB0E0101FA07F722FA06F3F140BB
:10D1D0001F43C5E9007100263146BDE8F087C2F162
:10D1E0002003D8400CFA02FC21FA03F391400143DA
:10D1F0004FEA1C471FFA8CFEB3FBF7F007FB103613
:10D200000B0C43EA064300FB0EF69E4204FA02F4BE
:10D2100008D91CEB030300F1FF382FD29E422DD911
:10D22000023863449B1B89B2B3FBF7F607FB163346
:10D2300041EA034106FB0EF38B4208D91CEB0101C6
:10D2400006F1FF3816D28B4214D9023E6144C91A46
:10D2500046EA004638E72E46284605E70646E3E656
:10D260001846F8E64B45A9D2B9EB020864EB0C0E60
:10D270000138A3E74646EAE7204694E74046D1E76F
:10D28000D0467BE7023B614432E7304609E764441D
:10D29000023842E7704700BF02E000F000F8FEE706
:10D2A00072B6374880F30888364880F309883648D4
:10D2B0003649086040F20000CCF200004EF63471AE
:10D2C000CEF200010860BFF34F8FBFF36F8F40F2C3
:10D2D0000000C0F2F0004EF68851CEF20001086066
:10D2E000BFF34F8FBFF36F8F4FF00000E1EE100AD6
:10D2F0004EF63C71CEF200010860062080F31488DF
:10D30000BFF36F8F9DF090FB9CF068FC4FF05530A1
:10D310001F491B4A91423CBF41F8040BFAE71D49E3
:10D32000184A91423CBF41F8040BFAE71A491B4ADC
:10D330001B4B9A423EBF51F8040B42F8040BF8E72E
:10D3400000201849184A91423CBF41F8040BFAE703
:10D350009DF06EFB9CF096FC144C154DAC4203DA2C
:10D3600054F8041B8847F9E702F05EFF114C124D98
:10D37000AC4203DA54F8041B8847F9E79DF056BB2A
:10D38000000600200022002000C0000808ED00E098
:10D39000000000200006002040030D0800220020AD
:10D3A0006C2600207026002060520120E0C1000899
:10D3B00038C2000838C2000838C200082DE9F04F12
:10D3C0002DED108AC1F80CD0C3689D46BDEC108AC3
:10D3D000BDE8F08F002383F311882846A047002082
:10D3E0009CF082F9FEE79BF0EFFF00DFFEE7000014
:10D3F00001F0FF01102A2BDB10F0070F08D010F806
:10D40000013B013A8B422DD010F0070F42B3F6D109
:10D41000F0B441EA012141EA014122F007047FF022
:10D4200000070023F0E80256083C85EA010586EA79
:10D43000010685FA47F5A3FA87F586FA47F6A5FAB5
:10D4400087F68EB9EED1F0BC01F0FF0102F00702C1
:10D4500032B110F8013B013A83EA010313B1F8D16C
:10D460000020704701387047002D06BF354603384D
:10D47000073815F0010F07D1013015F4807F02BF86
:10D48000013015F4C03F0130F0BC0138704700BFD7
:10D4900010F8012B11F8013B012A28BF9A42F7D05E
:10D4A000D01A7047034613F8012B002AFBD1181A33
:10D4B0000138704738B50022002304460D46FFF7B7
:10D4C000EDFA28B920462946BDE8384000F00AB8F0
:10D4D000204605F1004100F005F8404261EB4101B2
:10D4E00038BD00BFD0B50C4B002206460F46FFF7F3
:10D4F00063F8FFF739FB0446FEF7E4FF074B002211
:10D50000FFF75AF802460B4630463946FEF79CFEB6
:10D51000FFF72AFB2146D0BD0000F03D0000F0419E
:10D52000036800221B68184770B50D4B1C68E56A3C
:10D530002B681E6872F0B6F9014630B1E06A0368E4
:10D54000DB699847411E18BF01212846B0474BF0C0
:10D550000DF8E36ABDE8704093F89C104AF006B8F5
:10D560007826002013B501912021044672F0A6F917
:10D5700090B10A4BDFED0A7A93EDC87A019AB4EEC6
:10D58000E77AF1EE10FA05DA2046064B202172F018
:10D590009DF9002002B010BD0120FBE7805600205D
:10D5A00000000034642D0B0837B5094B0191054686
:10D5B000D3F8500603689B6998470199044618B947
:10D5C000044A284672F08AFB204603B030BD00BFF3
:10D5D00080760020782D0B0830B585B00446039185
:10D5E000402172F06BF990B31A49039AD1F8083EC2
:10D5F000D1F80C1EB3F90A5040F21450854214DCE5
:10D60000B3F90E5040F2A3639D421ADDB1F90A50FE
:10D61000854214DCB1F90E10994216DD1146204600
:10D6200005B0BDE8304072F0ABB90B4B00930B4B2B
:10D630002046402172F04AF9002005B030BD084B69
:10D64000F4E7054B0093074BF2E7054BFAE701209F
:10D65000F3E700BF805600205C2D0B088C2D0B08D3
:10D66000B07A0B08A22D0B082DE9F041DFF8A48059
:10D670000546D8F8500603688EB05B6A0E46984798
:10D68000F0B13146284672F04DFA044600B30AF074
:10D6900041FD002704462E22394602A80197A1F039
:10D6A000E5F82046322301AA01210AF09BF804463E
:10D6B00090B9144A01AB3146284672F00FFB07E0DF
:10D6C000D8F8500603689B6A98470028D9D10124EE
:10D6D00020460EB0BDE8F08198F8683633B10A4AAA
:10D6E0003146284672F0FAFA3C46F1E7074803F063
:10D6F000ADF804460028EAD1054A3146284672F0C2
:10D70000EDFAE5E7B82D0B08C12D0B0880260020A7
:10D71000CE2D0B0880760020A7B5C57F0191074666
:10D7200065B91F4B1B68986A03685B6B9847019942
:10D73000054630B91B4A384672F0D0FA284603B085
:10D74000A0BDBB6833B93B685B6B384603B0BDE82E
:10D75000A0401847144890F9483B002B09DD00F51C
:10D760001270019176F0EAFD0199054608B90F4A59
:10D77000E1E73846019173F015F9019905460C4827
:10D7800077F06AFE019905403846FFF7EBFEEDB2EF
:10D79000054001993846FFF707FF0540CEE700BF77
:10D7A00078260020E82D0B0880560020FF2D0B085E
:10D7B0005052002083680BB172F0EEBD012070471B
:10D7C00038B5054673F0A8F9044630B90C4A137809
:10D7D00043F001031370204638BD0121094876F05B
:10D7E000ADF8094806F004FB084876F039FE2846F3
:10D7F000FFF79AFE0649284673F0A8F8EBE700BF4A
:10D80000D48700201857002090860020C858002098
:10D81000202E0B0838B5054673F034FA044688B15B
:10D820000948D0F8502600F648539A4203D000F534
:10D83000586026F037FB2846FFF776FE0349284656
:10D8400073F084F8204638BD80760020302E0B0817
:10D8500008B5064BD3F8500603681B69984720B1FA
:10D86000BDE80840024872F01DB808BD807600206F
:10D870000C65002030B52DED028B85B00D46B0EE65
:10D88000408AFFF7E5FF0446C8B10AF043FC294689
:10D8900009F0BCF9B4EE488AF1EE10FAF0EE400A55
:10D8A00074BF9FED090A9FED090A09487EBF28EE63
:10D8B000008A9FED080A28EE000A05F061FD204667
:10D8C00005B0BDEC028B30BDE02E654200000000CB
:10D8D000508300200000C842014802F06DB800BF2C
:10D8E0008026002001485FF095B900BF2047002046
:10D8F000704700007047000000207047002070470C
:10D90000012070477047000000207047C820704712
:10D9100001207047012070470820704790F8903030
:10D920008B4286BF00EB8100D0F894000020704746
:10D9300090F890308B4286BF00EB8100D0F89400C5
:10D940000020704708B5034BD3F8500603681B68E6
:10D95000984708BD80760020044BD3ED007AFDEE99
:10D96000E77A17EE903A18B2704700BF785200205D
:10D97000014B93F8AC01704780460020034B93F9AC
:10D98000E001003818BF0120704700BF804600202A
:10D99000014B93F9AE01704780460020044BD3F849
:10D9A000500603F53F63C01A18BF0120704700BF3F
:10D9B00080760020704700007047000008B50448DA
:10D9C00007F044FE00280CBF0A200B2008BD00BF52
:10D9D0008026002038B5154DD5F850060368DB6960
:10D9E00098470028D5F850060368DB680CBF01246F
:10D9F0004124984708B144F008040D4BD5F850264F
:10DA000093F91833002B0B4B0ADD9A420AD044F0ED
:10DA10004004094871F046FF20B144F0800401E061
:10DA20009A42F6D144F0010038BD00BF8076002054
:10DA300080560020708200200C65002000B513EE97
:10DA4000103A8DB06222CDF8253013EE903ACDF821
:10DA500029302123CDE900328DF82410192303AA9F
:10DA6000C2218DED030ACDED040A8DED051ACDED31
:10DA7000061A8DED072ACDED082A4EF0E5FC0DB013
:10DA80005DF804FB2DE9F0412DED028B1D4F9FED5C
:10DA90001E8A002484B005462646F0EE488A07F523
:10DAA000516897F8903FE1B28B4216D9404642F058
:10DAB00037F880B1436836B1D3ED007AF4EEE78AE7
:10DAC000F1EE10FA07DDD3ED008ADB8808EE103A9C
:10DAD000B8EE488A01260134E3E76EB108235322E9
:10DAE000CDE90032287CCDED028A0DEB0302AD2199
:10DAF0008DED038A4EF0A8FC04B0BDEC028BBDE8AE
:10DB0000F08100BF8026002000000000F8B5B54D70
:10DB1000B5F8BC31DA07044639D505F6FC4CDCED26
:10DB2000000ADFEDB17A05F6F84C9CED000A05F528
:10DB3000516305F6045205F61C5605F60C5005F621
:10DB4000085105F6185796ED003AD0ED002A91EDF0
:10DB5000002A93ED001AD7ED003AD2ED001A207C8E
:10DB600060EEA70A20EE270A0521FFF767FF207C59
:10DB70004EF000FC0646207C4FF000FB00F1210334
:10DB80009E4204D2207CBDE8F8404DF049BEB5F875
:10DB9000BC319B072DD505F67471D1ED001A934960
:10DBA00005F6687305F6887C05F66C7205F67C76DA
:10DBB00005F6787005F68C77D6ED002A90ED002AF0
:10DBC00091ED001A93ED000ADCED003A97ED003A72
:10DBD000D2ED000A207C0421FFF730FF207C4EF0BC
:10DBE000C9FB0646207C4FF0C9FA00F121039E4292
:10DBF000C8D3B5F8BC315F0734D505F6CC6CDCED85
:10DC0000000ADFED797A05F6C86C9CED000A05F58F
:10DC10006E6305F6D46205F6EC6605F6DC6005F683
:10DC2000D86105F6E86796ED003AD0ED002A91ED4F
:10DC3000002A93ED001AD7ED003AD2ED001A207CAD
:10DC400060EEA70A20EE270A0221FFF7F7FE207CEC
:10DC50004EF090FB0646207C4FF090FA00F1210335
:10DC60009E428FD3B5F8BC311E0723D500216048F2
:10DC700070F03CF90721D0ED2D3A90ED2E3AD0ED21
:10DC80002A2A90ED292AD0ED281A90ED2B1AD0EDF2
:10DC9000260A90ED250A207CFFF7D0FE207C4EF06E
:10DCA00069FB0646207C4FF069FA00F121039E4291
:10DCB000FFF468AFB5F8BC31D80623D501214C4834
:10DCC00070F014F90821D0ED2D3A90ED2E3AD0EDF8
:10DCD0002A2A90ED292AD0ED281A90ED2B1AD0EDA2
:10DCE000260A90ED250A207CFFF7A8FE207C4EF046
:10DCF00041FB0646207C4FF041FA00F121039E4291
:10DD0000FFF440AFB5F8BC31990620D5394B207CE3
:10DD1000D3ED163A93ED173AD3ED132A93ED122A69
:10DD2000D3ED111A93ED141AD3ED0F0A93ED0E0AE9
:10DD30000921FFF783FE207C4EF01CFB0646207C69
:10DD40004FF01CFA00F121039E42FFF41BAFB5F81F
:10DD5000BC315A0620D5284B207CD3ED003A93EDF8
:10DD6000013A53ED032A13ED042A53ED051A13ED7E
:10DD7000021A53ED070A13ED080A0A21FFF75EFEA7
:10DD8000207C4EF0F7FA0646207C4FF0F7F900F1C0
:10DD900021039E42FFF4F6AEB5F8BC311B0620D538
:10DDA000164B207CD3ED003A93ED013A53ED032A54
:10DDB00013ED042A53ED051A13ED021A53ED070A69
:10DDC00013ED080A0B21FFF739FE207C4EF0D2FA42
:10DDD0000546207C4FF0D2F900F121039D42FFF46B
:10DDE000D1AEF8BD80460020E02E654200560020EE
:10DDF000405000208056002094620020C062002025
:10DE000038B5C5780B46352D044628BF3525352253
:10DE100000211846A0F02AFD2A4604F10C01BDE8B5
:10DE20003840A0F0D9BC000037B504460D4606487E
:10DE30000192114676F006FA019A2946204603B06F
:10DE4000BDE8304053F010B9185800202DE9FF41CB
:10DE50004FF00008CDE900289FED0F0A0F4F8DED20
:10DE6000030A0C46064615464FF47A73B1F90220B0
:10DE7000D7F8081E53F0D2FBCDE900589DED030AF8
:10DE8000B4F90420D7F80C1E4FF47A73304653F0DF
:10DE9000C5FB04B0BDE8F0810000FA4480560020C4
:10DEA00008B54FF061FD40F4E67040F0010008BD98
:10DEB00013B54FF44470CDE900210FF081FF044603
:10DEC00028B1DDE9002154F06FF9024B23602046B0
:10DED00002B010BD6C300B0810B504460FF078FF8F
:10DEE000204610BD0B4B93F860267AB993F868264C
:10DEF00062B9D3F8500603F53F62904208D003F6AA
:10DF00002843984214BF042003207047052070471F
:10DF1000022070478076002008B54B69012B07D19D
:10DF2000084876F0A7FA08B1002008BD0420FCE7F5
:10DF3000022B03D1034876F0A9FAF4E7BDE80840C4
:10DF40004FF0F8BDC858002010B594B0044603A89F
:10DF50000FF0D4FB1A4BD3F85006036803A91B6CCF
:10DF6000984750B3247C79F063FC059BDDED047A7F
:10DF70000893069B09930023F8EEE77A9FED117A48
:10DF80000B930C930D930E930F9310931193129385
:10DF90004FF6F853ADF84C300023962267EE877A9F
:10DFA0008DF84E303323CDE90032079007AA572170
:10DFB0002046CDED0A7A4EF047FA14B010BD00BFEE
:10DFC000807600200AD7233CF0B52DED028B2C4C37
:10DFD0000546D4F8500603688BB0DB6898470028E4
:10DFE00049D0D4F8504627482F7CDFED278A73F0BC
:10DFF0007DF8236820461B6B60EE288A9847BDEEAB
:10E00000C00A204610EE103A1EB22368DB6A984719
:10E01000BDEEC00A204610EE103A1DB22368DB6B3D
:10E020009847DFED1A7A2368B4EEE70AB0EE408A2B
:10E03000F1EE10FA5B6B58BFB0EE678A2046984746
:10E04000BCEEC88A002303930593069318EE103A9A
:10E05000B722ADF824301A23CDE900323E2103AABD
:10E060003846CDED048A8DED070AADF82060ADF895
:10E0700022504EF0E9F90BB0BDEC028BF0BD00BFB1
:10E0800080760020DC520020E02E654200FF7F47B2
:10E0900070B52DED048B044688B02948DFED298A40
:10E0A00077F016F9D8B3492056F0AEFC9FED269ACA
:10E0B00020EE090A4A2020EE288A56F0A5FC20EE20
:10E0C000090A60EE288A267C79F0B2FB05462046D4
:10E0D00053F0DCFCBDEEC88AFDEEE88A18EE103A7B
:10E0E00018EE902AADF80C300023CDE90533ADF8D9
:10E0F0000E30ADF81020ADF812308DF81C30ED2246
:10E100001623CDE900328DF81D0002AA22213046E7
:10E1100002954EF099F908B0BDEC048B70BD1A2041
:10E1200056F072FCDFED097A80EE278A462056F021
:10E130006BFCDFED077A28EE288A20EE270AC0E77D
:10E140005052002000401C466F12833A00A08C45BC
:10E150000AD7233C2DE9F047044692B0007C4EF0EC
:10E1600009F90546207C4FF009F800F126039D428D
:10E1700005D2207C12B0BDE8F0474DF051BB4248BB
:10E1800007F064FA002878D0404B1F68002F74D045
:10E190001921384641F048FD00286ED009F0BAFF39
:10E1A000064604A80FF0AAFA04A9304609F074FD47
:10E1B0004FF0000A97F88082D1465FFA8AF39845BB
:10E1C0005BD994F80F330133DBB2434534BF84F895
:10E1D0000F3384F80F9394F80F13384641F0A0FCE6
:10E1E000054600284CD0836893F92130192B47D17C
:10E1F00042F094FB002843D02B6803A91B6A2846F1
:10E20000984708B900230393284642F07DFB94F811
:10E210001080074679F00CFB6A68DDED057A94F80A
:10E220000F3312689FED1A7A8DF84430F8EEE77AD2
:10E230003B1F5F4208900F920698039AD6F80C1283
:10E2400009905F410798109267EE877A2F22262364
:10E25000D6F804C2D6F808420A90CDE900320E91F1
:10E2600008AA42F61E314046CDED0B7ACDF830C0FB
:10E270000D948DF845704EF0E7F812B0BDE8F087C8
:10E280000AF1010A99E700BF802600205C8800207F
:10E290000AD7233C2DE9F04300F50057C7B097F8A3
:10E2A000B05904460E46002D35D07022002106A834
:10E2B00004F5A044A0F0DAFA04F53D631868FEF70F
:10E2C00023F9012D8046894628D004F6D4342068ED
:10E2D000FEF71AF904460D4679F0AAFA4FF47A725D
:10E2E0005043002297F8B0392290239202A980224D
:10E2F00024A88DF81031CDE90289CDE90445A0F0BC
:10E300006BFA71228923CDE9003242F2283122AA28
:10E3100030464EF099F847B0BDE8F0830024002560
:10E32000DAE700003C2938B5054620D008D81B297B
:10E3300011D0242926D02846BDE8384053F0A0BC8F
:10E340004D29F8D126214DF07DFA044640B12846EA
:10E35000FFF700FF05E016214DF074FA044610B9EE
:10E360000024204638BD2846FFF792FEF9E78921B0
:10E370004DF068FA04460028F2D0297C0748FFF7E0
:10E3800089FFEEE70C214DF05DFA04460028E7D046
:10E39000297C034876F086F8E3E700BF802600205A
:10E3A000C858002030B52DED028BCD7891B0272DC7
:10E3B0000C464FF027024FF0000106A828BF272582
:10E3C000A0F054FA04F10C012E4C2A4606A8A0F045
:10E3D00003FAD4F8500603681B69984700284CD00C
:10E3E0009DF83E5015F04001019146D1FFEE000A24
:10E3F00040F28F30B7EE001A9DED0E0ADFED228A53
:10E400001FF006FF0199D4F850068DED0E0AB0EE0C
:10E41000408A02F0A1FF15F0040F68EE000A9FED9C
:10E420001B8A1BD0079B0293089B0393099B0493B1
:10E4300002A80A9BCDED010A059322F037F820EEE1
:10E44000280ADDED010A20EE080A04F54D6011B03E
:10E45000BDEC028BBDE8304004F066BF9DED0D0AB7
:10E4600020EE280A04F54D6020EE080A11B0BDEC3C
:10E47000028BBDE8304004F083BF11B0BDEC028BCD
:10E4800030BD00BF80760020E02E65420000C8420B
:10E4900070B50E4ED6F85006036886B01B690C4660
:10E4A000984780B102AD28460FF028F906AB13E972
:10E4B00003008DE8030004F1080195E80C0006F55F
:10E4C0004D6005F043F906B070BD00BF80760020B6
:10E4D00070B5304D2DED028B0646D5F8500691ED06
:10E4E000018A03688AB01B690C46984750B9BDEE93
:10E4F000C88A18EE103ADB0704D402200AB0BDEC3B
:10E50000028B70BDD4E9040120F09EFC0028F4D0F9
:10E51000236913B96369002BEFD002A80FF0EEF85E
:10E5200002AA2146304652F0E9FF0028E5D0D5F88E
:10E53000500603681B699847D0B194ED000ADFEDDF
:10E54000167AB4EEE70AF1EE10FA1ADA06AC2046B3
:10E550000FF0D4F80AAB13E903008DE803000F486D
:10E5600094E80C0002A905F0F1F840B10020C5E7DD
:10E570000B4802220F2106F047FF0028DDD10420BE
:10E58000BCE7D5F850060368DB6C98470028DDD15E
:10E59000F5E700BF807600200000003450830020A3
:10E5A0008026002030B58C8BC22C85B005460B46EA
:10E5B0003AD00CD8B22C26D0C02C30D0142C42D05B
:10E5C0001946284605B0BDE8304054F0F1B9D12CC9
:10E5D0003FD0B4F5967FF3D1D1ED007A9FED2D7A3F
:10E5E000F0EEE77AF4EEC77AF1EE10FA50D5D1EDFD
:10E5F000017AF0EEE77AF4EEC77AF1EE10FA47D539
:10E600002549022221E0254A91ED010AD2F850065F
:10E610000268D26C9047A0B9042005B030BD05B0A7
:10E62000BDE83040FFF754BF1C4A91ED000AD2F814
:10E630005046F7EE000A1FF0E7FC0146204602F0C4
:10E640009FFE0020E9E716490222164806F066FE02
:10E65000E1E7D1ED017AFCEEE77ACDED027AD1ED7A
:10E66000007A9DF80830FCEEE77ACDED037AD1ED23
:10E67000027AFDEEE77A17EE902A12B2009291ED3F
:10E68000030A9DF80C200146064805F097FEC4E7F2
:10E690000220C2E700000034C883002080760020FA
:10E6A00018860020802600202DE9F04F2DED028BEA
:10E6B000934F9FB0084610A9FFF7A2FBD7F850066A
:10E6C00003681B699847002800F0118104A80FF027
:10E6D00015F804A9A7F5755009F022FB002800F0F1
:10E6E00006819DF874C0BCF1010F04D0ACF10703A2
:10E6F000022B00F2FC8007F2BC530FCBBDF8705028
:10E7000008AC15F0030984E80F0005F0180B05F0BC
:10E71000C00A05F4806805F400661ED1BCF1070F3D
:10E720009DED110ADDED120A14D0ACF1080CBCF11C
:10E73000010F00F2A480734B93ED037AD3ED007ABE
:10E7400060EEC76A67EEA00AE0EE276AE0EE070A0D
:10E75000B0EE660A20460FF003FBBBF1000F40F05D
:10E7600093805946D7F8500602F0F6FDDDED157A94
:10E770009DED147A8DED030A27EEA70AA7EE070A8E
:10E780001FF076FC9DED031A40F2E330F1EE410AF2
:10E790001FF03EFDDDED140AB0EE408A9DED150A36
:10E7A0009DF06AFEDFED587A9DF8743060EE277AAE
:10E7B000083B9FED560A012B67EE807A0CD8544B2C
:10E7C00003F5986393ED000AB8EEC00A30EE270A0D
:10E7D0001FF0C8FCF0EE407AB8F1000F1BD19FED9E
:10E7E0004A0ADDED1A7A9DF8743067EE807A083BAC
:10E7F0009FED460A012B67EE807A0CD8444B03F557
:10E80000986393ED000AB8EEC00A30EE270A1FF0B5
:10E81000A9FCF0EE407A002E3BD19FED3B0A9DED26
:10E820001B7A27EE007A9FED390A27EE000ABBF12A
:10E83000000F4BD105F44065B5F5406F5CD09FEDFE
:10E84000357ADDED146AF4EEC76AF1EE10FAFFEEE8
:10E85000000AB7EE007A88BFF0EE470AB9F1000F60
:10E8600037D0BAF1000F42D0B5F5406F14D168EE41
:10E87000200A2948B0EE670A04F056FD37E004ABE1
:10E880000FCB84E80F0065E7DFED247AB0EE678AEE
:10E89000A2E79FED220ACAE7B8F1000F06D036BB07
:10E8A00068EE200A1C4804F06BFD20E0FEB1DEE7B4
:10E8B000BAF1000F1BD0B8F1000F03D1BEB1DFEDEC
:10E8C000170AD6E79EB9DFED150AEBE7B9F1000F9D
:10E8D000EED10CAD28460EF011FFDDE90E018DE8FA
:10E8E00003000D4895E80C00214604F02FFF1FB0EF
:10E8F000BDEC028BBDE8F08FF7EE000AAEE700BF7B
:10E9000080760020903B0020E02E65420000C84247
:10E9100080360020000000B450830020000000007A
:10E920002DE9F04F2DED028BDFF8D0B19BB00846FA
:10E930000CA9FFF765FADBF8500603681B699847D6
:10E94000002800F095809DF864300B2B00F2908039
:10E95000DFE803F0068E8E068E06068E8E8E060685
:10E960000BF2BC530FCBBDF8604004AD14F00309AB
:10E9700085E80F0004F0180804F0C00A04F480676A
:10E9800004F4006609D1DDE90D0120F05DFA0028EC
:10E990006ED00D9B06930E9B0793B8F1000F6CD1C0
:10E9A0004146DBF8500602F0D7FCDDED117A9DED13
:10E9B000107A8DED030A27EEA70AA7EE070A1FF0CB
:10E9C00057FB9DED031A4FF48A60F1EE410A1FF0E8
:10E9D0001FFCDDED100AB0EE408A9DED110A9DF09E
:10E9E0004BFDDFED417A60EE277A9FED400A67EE3E
:10E9F000807A4FB99FED3C0ADDED167A67EE807A9A
:10EA00009FED3A0A67EE807A002E3BD19FED360AE1
:10EA10009DED177A27EE007A9FED340A27EE000A63
:10EA2000B8F1000F53D104F44064B4F5406F4BD0FB
:10EA30009FED2F7ADDED106AF4EEC76AF1EE10FA61
:10EA4000FFEE000AB7EE007A88BFF0EE470AB9F190
:10EA5000000F1AD108AC20460EF050FEDDE90A0185
:10EA60008DE80300234894E80C00294604F06EFE6C
:10EA70001BB0BDEC028BBDE8F08FDFED1F7AB0EE6E
:10EA8000678AB6E79FED1C0ACAE7BAF1000FEFD01C
:10EA9000B4F5406F07D168EE200A1648B0EE670A59
:10EAA00004F042FCE4E73FB1002EE1D168EE200A19
:10EAB000104804F065FCDBE7002ED9D0EBE7002E10
:10EAC000D6D1DFED0D0AF3E7F7EE000ABFE7B9F1A3
:10EAD000000FBFD0BAF1000FCAD0002FEFD1002E27
:10EAE000C6D0DFED050AD8E7E02E65420000C84237
:10EAF000000000B450830020000000008076002059
:10EB000010B44B7A8C7ACA7A43EA042343EA02436C
:10EB1000542B07D0562B09D0522B0BD15DF8044B48
:10EB2000FFF740BC5DF8044BFFF7BEBD5DF8044B3A
:10EB3000FFF7F6BE5DF8044B52F0D2BD014B93F8DF
:10EB4000AA01704780460020074B084AD3F85016A8
:10EB5000914201BFA3F5005393F94402B0FA80F04B
:10EB6000400918BF00207047807600209086002062
:10EB7000074B084AD3F85016914207D1A3F500532A
:10EB800093F94402431E5842584170470020704791
:10EB9000807600209086002038B5036A1D4D43F42E
:10EBA000B84303620446D5F8500603681B6A9847C9
:10EBB00038B1D4E9092342F4406243F4406362620D
:10EBC000A362D5F850060368DB68984738B1D4E9EA
:10EBD000092342F4A04243F4A0436262A3620E4BB5
:10EBE0001868A8B190F8803293B1236A43F4807317
:10EBF0002362636A43F480736362002140F090FFF4
:10EC000030B141F08BFE18B1A36A43F48073A36264
:10EC100038BD00BF807600205C8800207FB500F5FD
:10EC200031561C360446304672F060FADFED1D7A2C
:10EC300020EE270A002301A904F5965001938DEDDB
:10EC4000020A039307F094FC09F064FA09F00EF845
:10EC500004F57C6504F5335238326D21284648F0BE
:10EC60002DFB284606F543726C2148F027FB204611
:10EC700001F05EFB30B104F53B5208326A212846B0
:10EC800048F01CFB04F5405393F9483B002B06DD8C
:10EC900004F5405238326921284648F00FFB04B091
:10ECA00070BD00BFE02E65422DE9F04F054695B0DE
:10ECB000344806F0CBFC002860D005F551691921D5
:10ECC000484640F0B1FF002858D010A80EF016FDBD
:10ECD00010A905F5965008F0DFFFDFF8BCB000275B
:10ECE00095F8903FFEB2B34248D93146484640F0CD
:10ECF00017FF044600283FD0836893F92130192B71
:10ED00003AD141F00BFE002836D063681A6905EB52
:10ED1000860303F5A043D3F8701691422CD0C3F8B4
:10ED2000702623680FA91B6A2046984708B900235C
:10ED30000F9378F085FD0D900F988A46FDF7E4FB60
:10ED4000CDE90A0161680868FDF7DEFBCDE908013D
:10ED500013990D9A0C4B06911299019305F57C6855
:10ED60000A4B0093CDE90461CDE9022A0849094A1A
:10ED70005B46404649F016F80137B1E715B0BDE8EB
:10ED8000F08F00BF80260020A3310B08AA310B08AA
:10ED90009E310B087F310B0878310B08F0B58BB032
:10EDA000154606460F462422002101A81C469FF066
:10EDB0005DFDA3238DF8043095238DF805300323E2
:10EDC0008DF8063078F03CFD2B6804936B68059352
:10EDD000AB680693236807936368CDF80700CDF806
:10EDE0000B1008932422A3688DF80F7001A906F573
:10EDF0007C60099348F0D6FB0BB0F0BD30B589B00C
:10EE00001D220446002168469FF030FDA3238DF8A3
:10EE1000003095238DF8013001238DF8023078F011
:10EE20000FFD04F5A045CDF80300D5F85006CDF848
:10EE300007100368DB6B984710EE103AD5F85006C0
:10EE4000CDF80B300368DB6A984710EE103AD5F81E
:10EE50005006CDF80F3003681B6B984710EE103A40
:10EE6000CDF8133004F58053D5F85006D3F8C034EC
:10EE7000ADF8173003685B6B984710EE103A1D220F
:10EE8000694604F57C60CDF8193048F08BFB09B079
:10EE900030BD00002DE9F04F2DED068B00F54055FB
:10EEA00091B095F9483B002B06464ADD00F57C6998
:10EEB00000F54950083075F041FA0446002845D065
:10EEC00095EDA58ADFED237A95F8084328EE278A89
:10EED00078F0B6FC06F52F558046686D0F46FDF7B5
:10EEE00013FB8246A86D8B46FDF70EFB41EC190B18
:10EEF000E86DFDF709FB41EC1A0B06F56D50083083
:10EF000005F086FD10EE100AFDF7FEFACDE90E01C0
:10EF100018EE100A8DED0CAB8DED0A9BCDE908AB18
:10EF2000FDF7F2FA0C4B01930C4B0093CDE906016F
:10EF3000CDE902870A4B0B4A0B490494484648F036
:10EF400031FF11B0BDEC068BBDE8F08F9FED078A55
:10EF5000BEE700BFE02E6542F4310B08FC310B0820
:10EF6000B4310B08BC310B08EF310B085241C07FA4
:10EF700030B52DED028B00F531558BB01C350446B4
:10EF80002C4B00936946284672F0A0F921220021FB
:10EF900001A89FF06BFCA3238DF8043095238DF816
:10EFA000053002238DF8063078F04AFC04F5405312
:10EFB000CDF80B10D3F8083ECDF80700B3F90830B0
:10EFC000ADF80F3004F52F5310339FED1B8A5B6AA9
:10EFD000CDF8113004F5A043D3F8500603689B6BBD
:10EFE000984710EE103A2846CDF81530009BCDF822
:10EFF000193071F06BFF20EE080A04F5AF5110EEE6
:10F00000103A04F5AE5018311430CDF81D3022F00E
:10F01000A5F820EE080A212210EE103A01A904F505
:10F020007C60CDF8213048F0BDFA0BB0BDEC028B0E
:10F0300030BD00BF5241C07FE02E654270B590F8F0
:10F04000AB2B00F698030C2101FB023300F5315580
:10F050008AB01C350446D3F888611C4B019301A982
:10F06000284672F0C5F81D22002102A89FF0FEFB81
:10F07000A3238DF8083095238DF8093078F0E0FB54
:10F0800004F54053CDF80B00D3F80C3ECDF80F102B
:10F09000B3F90830ADF8133004F52F531033284678
:10F0A0009B6ACDF8153072F08BFA10EE103A1D22E3
:10F0B000CDF8193002A9019BCDF81D3004F57C6014
:10F0C000CDF8216048F06EFA0AB070BD5241C07FA1
:10F0D00013B5044604F5805400F57C60019047F0B8
:10F0E0005BFD019847F0F2FD94F9D430019823B10B
:10F0F00002B0BDE8104047F091BE02B010BD000064
:10F1000010B500F5A0430446D3F8500603681B6809
:10F11000984704F50053014693F85C2104F57C60A0
:10F1200048F000FC04F5965009F0EAF904F59070F7
:10F13000BDE8104016F0F6BF992070472DE9F34165
:10F140000446043054F046F93E4E3F4B636054256C
:10F15000601954F0F5FA66513035B5F5557FF7D1A1
:10F1600004F5557055F014FF04F25C7104F5FC656C
:10F17000084601916EF090FC019928466EF0FAFD68
:10F1800004F67C27294604F51F6075F09BFF38467E
:10F1900071F0B2FD002104F6B86074F003F904F5D3
:10F1A00077605FF069FB04F6B87074F047FE04F511
:10F1B000825004F58058103040F098F904F5CD568F
:10F1C000224BC8F8503004F5835004F589551C359E
:10F1D0001836083075F068F832463946284672F01D
:10F1E000C5FF1B4BC8F83C3104F5C8500EF086FA39
:10F1F00005F2D4700EF082FA04F5C9500EF07EFAD2
:10F2000005F2F4700EF07AFA04F5CA500EF076FAB0
:10F2100005F614000EF072FA04F5CB50083005F034
:10F2200087FA3946304672F08BFB04F5DC50083023
:10F2300003F084FC204607493FF004FA204602B060
:10F24000BDE8F0818C740B08A0740B089C2E0B0891
:10F2500050C40C08F46B0B08F0B500F50651B5B0BE
:10F2600010222031044646F0CFFD574800222B21C2
:10F270003EF062FD3FF0ECFB544A13881A2143F044
:10F2800002030020138055F00DFE0220462155F0A8
:10F2900009FE204601F04CF840B104F546501E230B
:10F2A00014A910308DF850303FF0EAFF484D55F06A
:10F2B00003FC95E80F0004AE86E80F0002A9304673
:10F2C0003EF042FCF0B105F1100314AA183518689D
:10F2D0005968164603C60833AB423246F7D1186860
:10F2E0001B79306033719DF808300C2B0AD834AA92
:10F2F0001344079813F8803C00EE103AB8EE400A29
:10F300003FF048FD334D95E80F0008AE103586E814
:10F310000F0095E80F000CAF87E80F0003A93046F7
:10F320003EF012FC0146002849D00021B7EE000A49
:10F3300030463EF055FC04F507552749802214A8B5
:10F340009FF04AFA2035082114A800223EF0F4FC70
:10F3500010A928463EF078FA00282ED01F490B68E5
:10F36000D8070ED41E4B04F5F75208321A6004F584
:10F3700002522032DA6004F5015208329A61012308
:10F380000B6028461649032201253EF02BFD154A45
:10F390000095002304F57C61FD203EF0D1FC124B6A
:10F3A0001A68D20705D4114A1D6004F58F54083439
:10F3B00014600E4801213EF031FD35B0F0BDB7EECE
:10F3C000000A3846B5E700BF44690B0840880020B2
:10F3D000F02A0B08102B0B08302B0B08702600208E
:10F3E0000022002044140C0874260020242200204F
:10F3F0000069C0F3401070470F299DBF302303FB05
:10F400000100503000207047014B93F9D401704740
:10F4100080460020024B93F8580600F00100704728
:10F420008076002008B503689B68984780F001004B
:10F43000C0B208BD014BD3F8080E704780560020BB
:10F4400000290DDB074890F8242ECBB29A4207D34F
:10F45000D0F8203E0122595CA0F5405005F0D4BF01
:10F46000704700BF8056002008B53AB1022A10D17B
:10F47000BDE808400748352205F050BF064AD2F8DB
:10F4800050268A4205D154F025F9BDE8084054F0D1
:10F49000ABB808BD802600208076002030B589B04A
:10F4A0001C220021104D03AC01A89FF0DFF920467B
:10F4B0000EF024F905F2BC530FCB84E80F001023A3
:10F4C00001A905F55860ADF8063022F06BFD40B19A
:10F4D000064BB5F8B42D1B680549986903681B688D
:10F4E000984709B030BD00BF807600207826002004
:10F4F000A4720B0801290A4603D0022900D019B9C9
:10F500000122024805F0F0BA704700BFC861002030
:10F510004A2910B40B4604462FD026DC3F2921DCB3
:10F52000292913DC04390C2918D9204619465DF81D
:10F53000044B54F0BBBEA3F1C9000121814040F24D
:10F5400043400142F1D05DF8044B70472A39012055
:10F5500088400C4901400029E7D0F4E701200A491E
:10F560009840F7E74829E0D1EDE7D329DDDCC82949
:10F57000E1DC6129E7D09B29F5E75DF8044B1146F2
:10F58000FFF7B8BF01FF2200900001000B464A2B95
:10F59000F7B5064611465FDC292B0FDC072B70D030
:10F5A00056DC002B5DD0042B00F0AC800A463046C0
:10F5B000194603B0BDE8F04054F03CBCA3F12A0268
:10F5C000202AF3D801A050F822F000BF09F7000864
:10F5D000ADF50008ADF50008ADF50008ADF5000883
:10F5E000ADF50008ADF50008ADF50008DBF6000844
:10F5F000E7F60008F3F60008F9F60008FFF6000841
:10F600000FF7000815F70008ADF50008ADF5000884
:10F610001BF70008ADF50008ADF50008ADF50008D2
:10F6200027F70008ADF50008ADF50008ADF50008B6
:10F63000ADF50008ADF50008ADF50008ADF5000822
:10F64000ADF5000821F70008ADF5000835F7000812
:10F65000102BABD14D4949E09B2B6FD003DC612BC4
:10F66000A4D101240AE0A3F1C9050A2D9ED80124E2
:10F6700004FA05F540F24342154297D0204603B004
:10F68000F0BD022AEDD1424DD5F8503605F6485767
:10F69000BB42E6D03F4870F005F9044678B905F55D
:10F6A000586022F03DFA52F061FD3B4A05214BF0D3
:10F6B000ADFE2146A5F5A04000F042FED1E7D5F809
:10F6C0005036BB42CDD0B5F9B43D13B93046FFF743
:10F6D000E5FE3046FFF7E2FED0E70229C1D12F4810
:10F6E00000F0CCFFBDE70A462D493046FFF7BCFECF
:10F6F000B7E70A462B49F8E70A462B49F5E70A46D9
:10F700002A49F2E72A49F1E70A462A49EDE70A467B
:10F710002949EAE70A462949E7E70A462849E4E78A
:10F720000A462849E1E71A4BD3F8500603685B6D97
:10F73000984796E73046FFF7DDFE92E722480192B0
:10F7400075F0C6FD00288CD1124870F0ABF8044665
:10F75000002886D00E4BD3F8502603F57160824204
:10F760003FF47FAF03F628439A423FF47AAF019902
:10F7700002297FF476AF1A2055F018FB52F0F6FC00
:10F78000124A01994BF042FE78E700BFC88300207F
:10F79000807600200C650020B8720B0880260020BF
:10F7A000E082002018830020DC850020A882002051
:10F7B0001886002054860020508300209085002069
:10F7C00090860020E863002050520020D1720B0880
:10F7D00000207047002070470020704700207047CD
:10F7E00000207047002070470020704700207047BD
:10F7F00008B50368DB68984780F00100C0B208BD17
:10F8000001207047012070479FED010A704700BF3B
:10F810000000000000207047012070470020704762
:10F82000704700001020704700487047BC740B08F8
:10F83000704700000020704701207047002070478B
:10F840000020704700F5065024307047004870478C
:10F85000B4550B0800F5A040D0F8500603681B68AB
:10F860001847000000F5A04300F5BA40D3F8503621
:10F8700048301B1A5842584170470000034808603E
:10F880002021117008221A60704700BF54770B08BE
:10F8900003685B681847000000F09ABF00F0FABDEB
:10F8A00056F0C6BB45F0BEBC1CF030BC47F0E0BF14
:10F8B00005F09EBB04F010BB01F09CB801F030BA1B
:10F8C0000CF0E8B855F05ABF58F094B90BF046BCAC
:10F8D00053F04EBE53F054BB51F018BD05F084BB3D
:10F8E00005F0A0BB74F0B8BE0AF0A8BD17F072BB5B
:10F8F00000F0C2BC05F03EBC04F0F6BE01F0DEB97B
:10F9000010B50368DB680446984728B120460021FB
:10F91000BDE8104001F034BD10BD000003F022B876
:10F9200002F05CBD02F0A0BA70B50A4B0446D3F8F1
:10F9300050060368DB680E469847054640B104F55B
:10F94000A044D4F850060368DB6B984786ED000AA4
:10F95000284670BD8076002070B50A4B0446D3F867
:10F9600050060368DB680E469847054640B104F52B
:10F97000A044D4F850060368DB6A984786ED000A75
:10F98000284670BD8076002070B50A4B0446D3F837
:10F9900050060368DB680E469847054640B104F5FB
:10F9A000A044D4F8500603685B6B984786ED000AC4
:10F9B000284670BD8076002070B500F5A04304464F
:10F9C000D3F85006036886B01B690D46984780B18E
:10F9D00002AE30460DF092FE06AB13E903008DE84F
:10F9E000030004F5B94096E80C002946503003F0B6
:10F9F000ADFE06B070BD000070B51F4B036000F592
:10FA0000A0430446D3F850051C4AC3F8A02308B10C
:10FA10000EF0E2F91A4B236004F5805393F8842E1C
:10FA200042B9D3F8805E2DB128461BF06DFA284606
:10FA30000EF0CEF904F58E500C306FF077FA04F525
:10FA40008650143056F0CEF804F6C44504F66446E9
:10FA5000B54204D0183D28461AF0AAFEF8E7094B33
:10FA6000C4F8983804F694104AF018FF04F51060B2
:10FA70004AF014FF204670BDE4790B08842E0C0870
:10FA8000240D0C0878D40B0838B5474B044640F8D1
:10FA9000043B56F0EDFB04F110000BF085FC04F183
:10FAA000680045F04DF904F5907015F01DFF04F560
:10FAB00086600AF033FB04F254500EF08FF904F61E
:10FAC00098001CF0D7F904F5446056F0AFF904F53E
:10FAD00051603FF0CFFF04F57C6047F097FC04F5E0
:10FAE0008650143056F066F804F5885010300CF04B
:10FAF0006FFF04F58E500C306FF004FA04F58F5050
:10FB0000083045F0DFFC04F591501C3057F092FDB1
:10FB100004F5805304F593520025104683F8605293
:10FB2000224B10301A603BF0D9FB294604F5965061
:10FB300006F072FE04F5C850103067F081FD04F540
:10FB4000E85014306BF0C6FE04F5F1500C306EF046
:10FB500033FB04F5F45010306EF068FF04F5F750F5
:10FB6000083005F07BFD04F50150083068F0C6F957
:10FB700004F5025020305CF07BFD04F5005304F5E1
:10FB8000055083F85C510A4D34306FF08FFD2B68BF
:10FB900013B1084877F01AFE204607493EF052FD9F
:10FBA0002C60204638BD00BF240D0C083091002089
:10FBB00094880020C4740B084C0C0C08F8B504465B
:10FBC000254601F03DFA214B45F8383B204B646552
:10FBD000C4E916341F4BC4E918341F4BA36604F163
:10FBE0007C000DF08BFD04F198000DF087FD04F111
:10FBF000B4000DF083FD4FF6FF76184BC4F8C83003
:10FC0000A4F8CC6004F1D0000DF078FD4FF0FF3780
:10FC1000134B1449C4F82C7128461D603EF012FDA8
:10FC2000A4F87470A4F8906004F5A2700DF066FD5D
:10FC300004F5BE700DF062FD04F5CC700DF05EFDB4
:10FC400004F5DA700DF05AFD2046F8BDF47D0B087E
:10FC50001DF9000821F9000825F900080000FFFF40
:10FC600084870020C0E10B082DE9F041044686B0EE
:10FC7000FFF70AFF864B2360864B8748186004F520
:10FC800006521C32002314269DB206FB05010133E7
:10FC9000097C0029F8D1814B1D80814B196811B175
:10FCA000804877F093FD04F5075020301A60FFF785
:10FCB00045FA04F5785071F005F804F5405504F55F
:10FCC00007531533C5F8203E04F57850062385F810
:10FCD000243E283055F080FB04F57A500C306FF04C
:10FCE000A1FD714BC5F88C3E04F57B5004306FF0DC
:10FCF00083FD6E4BC5F8C43E04F57B50083004F517
:10FD0000A04504F5A74760F031F92037684BC5F8E6
:10FD1000A03307F1080076F0C7FC04F5A74604F508
:10FD2000A8484C3608F13008304614364FF0E2FC53
:10FD3000B045F9D10723C5F854350023A5F8583547
:10FD40004FF4CB700EF042F8C5F8500504F5AA4008
:10FD50005C3076F0A9FC04F5AB40203076F0A4FCD2
:10FD6000544B1A6802B91F60534BC5F8A03304F511
:10FD7000AB403C300DF0C2FC04F5AB404FF4805179
:10FD80004C300BF00DFC04F5B7464C4B0593703628
:10FD90004B4BC5F850660494009304F5AD4006AB98
:10FDA00013E90C004FF400711C300AF065FE304678
:10FDB00001F046F9434BC5F8F03B04F5B840283054
:10FDC00001F03EF9404BC5F8283C04F5B8406030DE
:10FDD00001F036F93D4BC5F8603C04F5B9401830E8
:10FDE00001F02EF93A4BC5F8983C04F5B940503073
:10FDF00001F026F9374BC5F8D03C04F5BA4038304D
:10FE00000DF07CFC04F5BE4604F5BA4010364830CF
:10FE1000FFF7D4FE304601F013F92F4BC5F8103F21
:10FE200006F138000DF06AFC04F5BE405C3001F0CC
:10FE300007F92A4BC5F85C3F04F5BF40183001F0C4
:10FE4000FFF8274BC5F8983F04F5BF40543001F048
:10FE5000F7F8244BC5F8D43F04F5C040103001F04A
:10FE6000EFF804F5C0431D461F4A1A6150354FF0A4
:10FE7000804603A9284603964AF0B8FF02A905F177
:10FE80000C0002964AF0B2FF204606B0BDE8F081B1
:10FE9000E4790B0850880020446E0B084E8800203F
:10FEA0000C880020D8740B084C2E0B088C2E0B08E5
:10FEB000842E0C08B08B002040310B08FDF80008A0
:10FEC000D4790B08FC740B0840800B0828810B08C0
:10FED000147C0B08D47F0B08B4800B0818830B0824
:10FEE000A8810B08AC820B081C820B08F0B50446F5
:10FEF00000F57A5085B00C30FDF716FB04F59656E8
:10FF0000204605F04BF90021304608F089F804F549
:10FF1000AB413C31304607F0BFFE04F5A04504F587
:10FF2000805785F86C0697F83C1511F0010103D154
:10FF3000236820469B6C9847002301A93046019313
:10FF40000293039307F0F8FE28B301A820F09AFD6E
:10FF500005F5D36585ED000A0121204605F072FB09
:10FF600028B12046FEF75AFE2046FEF793FF802177
:10FF7000204605F067FB18B11DF042FC1BF04AFE5D
:10FF80004FF48011204605F05DFB10B1304606F0BD
:10FF9000C9FB05B0F0BD94F8E433B02202FB034383
:10FFA00094F8282493F8C131002AD5D1022B81BFBF
:10FFB00007F2C46705F5D3653B682B60CCE700000A
:10FFC000FFF794BF70B500F50053044693F9CC31A8
:10FFD00033B300F5A043D3F84C550DB377F028FCAC
:10FFE00004F5755393ED090ADFED0E7A9FED0E1AB5
:10FFF000DFED0E0A451B20EE270A40F269101EF0C5
:020000040801F1
:1000000007F9FCEEC07A204617EE903A9D42084A66
:10001000BDE8704034BF00230123022100F092BDEF
:1000200070BD00BF00007A440000804F0000000057
:10003000DA670B08FFF7C6BF37B50221044605F0A3
:1000400001FB50B10121204605F0FCFA28B92046F9
:10005000FEF7E4FD2046FEF71DFF1021204605F0C7
:10006000F1FA10B12046FEF7E9FF2021204605F005
:10007000E9FA00B304F56E5520461835FEF7BEFECA
:10008000284671F0A1FCB0B1284671F095FD04F549
:100090007C6004F56E54343404F140026E2101900A
:1000A00047F00CF9019804F16C026F2103B0BDE830
:1000B000304047F003B903B030BD0000FFF7BCBFCC
:1000C00010B54FF40051044605F0BCFA10B12046BB
:1000D000FEF74EFF4FF48041204605F0B3FA38B1E9
:1000E0002046FEF7F5FF04F524503C306DF0D0FDBE
:1000F0008021204605F0A6FA28B11DF081FBBDE85D
:1001000010401BF0ABBD10BDFFF7DABF73B503683D
:10011000354D9B6D044604F57A5698470C3655F0DC
:1001200057F854F03FFD00213046FDF7F5FAA8716D
:1001300030462E4E0123EB716FF0B4FB336828710B
:10014000DB6A2B4A93F89C306B7104F50055B5F8C7
:10015000AA11117013B9204600F06EF93368DB6AFA
:1001600093F89C6036B195F85E311BB977F060FB6F
:10017000C5F8600185F85E6104F5405604F52F5519
:1001800096ED240A103528468DED010A75F0A0F889
:10019000014604F54C509DED010A1C3072F028F91F
:1001A00096ED240A28468DED010A75F091F8014676
:1001B00004F56E509DED010A183071F045FC45F0D4
:1001C000E7F844F04FFD04F527506DF095FE67F019
:1001D00099FF0446284676F09FF90146204602B072
:1001E000BDE8704067F06ABFB58700207826002020
:1001F000AC230020FFF78ABF10B5094B1B780446DB
:1002000023B100F531501C3071F08AFB04F5A04495
:10021000D4F850060368BDE810409B68184700BF3B
:10022000E48B0020FFF7E8BF38B5054B1C68236856
:100230000A461D68034B01462046A847002038BDEA
:10024000782600208026002010B576F0FBFD064CB5
:10025000064B18602046FFF707FD2046044A054973
:10026000BDE810409BF0C0BD80260020782600200D
:1002700060E90020F9F9000813B500F5A043044631
:1002800093F8ED3B23B102B0BDE8104003F0CABFC4
:1002900000F53150002301A91C30019370F0A8FF34
:1002A00004F57A500C306FF0FDFA014604F52F503A
:1002B000D4ED460A9DED010A103076F0D9F802B06F
:1002C00010BD000010B500F54053D1ED007A9FED50
:1002D000157AD3ED630A93EDC50A90ED461A00F541
:1002E000005367EEC77A9FED107A93F8D03B67EE24
:1002F000A07A20EE070A13F00C0F00F531500C46DF
:10030000A7EE870A14BF0121002160EE870A1C3086
:1003100070F00AFEDFED057A20EE270A84ED000A70
:1003200010BD00BF0AD7233C35FA8E3C0000C842FE
:1003300000F5405090F94C01C31E58425841704797
:100340007FB5044604F5965668460D460DF0D6F97D
:10035000304606F0EDFD18B90025284604B070BD02
:100360006946304607F098FC0028F5D023682A46F5
:10037000DB6C69462046984705460028ECD004F51A
:1003800042500121183073F0D9FAE6E7F0B52DEDAF
:10039000028B044687B000F596500D46174607F0CD
:1003A00069FB064600283CD03FB104F5805292F824
:1003B0003C3543F0020382F83C3504F5BB4021F0A4
:1003C00011FED5ED017A9FED197A9FED198AF8EEAD
:1003D000E77A04F5A74467EE877A203417EE900A8F
:1003E000FCF792F8D5ED037AF8EEE77ACDE904014F
:1003F00067EE887A17EE900AFCF786F8D5ED027A58
:10040000F8EEE77ACDE9020167EE887A17EE900AF6
:10041000FCF77AF8074ACDE90001062120464AF0A8
:10042000F5FF304607B0BDEC028BF0BD0AD7233C88
:1004300095BFD633507A0B087FB500F58056044639
:1004400096F83C359A0715D4684604F596550DF094
:1004500055F96946284607F01FFC58B104F5866037
:1004600009F030FF96F83C35DB0705D4694628468D
:1004700007F000FB04B070BD05F51B7168460DF078
:10048000FFFBF6EE007AB4EEE70AF1EE10FAEDD5D6
:10049000F0E70000F8B500F57A560C360446304611
:1004A0006FF000FA054618B9504B00221A80F8BDCB
:1004B00004F5005797F9CD31002BF5D004F5A04392
:1004C000D3F850060368DB68984720B92046FFF749
:1004D0002FFF0028E8D004F5405393F99031002B0A
:1004E00042D007EE903A9FED427AF8EEE77A04F5B3
:1004F000805303F5996267EE877A92ED007AB0EE49
:10050000C77AB4EEE77AF1EE10FA0CDC03F2C443DA
:1005100093ED007AB0EEC77AB4EEE77AF1EE10FA16
:10052000CCBF012500252046FFF702FFF0B1002DCA
:10053000BDD048F01BF80C21012247F0CFFD20462A
:10054000FFF7F6FE04F5A7432033014600283CD010
:10055000284A002118464AF059FF30460122BDE8DA
:10056000F8400C21FDF756B91D46DCE72DBB04F51C
:10057000805303F2C4629FED207AD2ED007AF4EE4C
:10058000C77AF1EE10FA8FDA03F2D453D3ED027A80
:10059000F0EEE77AF4EEC77AF1EE10FA84DA07F5B6
:1005A0003D63D3ED0A7AB1EE047AF0EEE77AF4EE29
:1005B000C77AF1EE10FA3FF577AF0C4A1388013392
:1005C0009BB2132B1380B2D9B3E718460B4A4AF0FB
:1005D0001DFF04F5B84113222831204604F09EFE89
:1005E00097F9CD31022B7FF462AFB6E7F886002091
:1005F00035FA8E3C707A0B080AD7A33D817A0B0836
:100600002DE9F04D88B0044647F0B0FF054677F07D
:1006100017F904F5C04307469B6E04F5C040B3F1DB
:10062000000800F1500018BF4FF001080E464AF0D4
:100630007BFB0068FBF768FF824604F5C0405C3036
:100640008B464AF071FB0068FBF75EFFCDE904AB17
:10065000CDE90601CDE90076054B064A0649CDF8FD
:100660000880284647F0AEFB08B0BDE8F08D00BF1B
:10067000987A0B089D7A0B08B97A0B0873B5044673
:1006800000F57A500C306FF00DF904F5A7452035D0
:1006900004F5C04640B90023154AB3660221284636
:1006A0004AF0B4FE02B070BD04F5315069461C300A
:1006B00070F09EFD0028EED004F5C0406946503031
:1006C0004AF034FB04F52F53103304F5C0409B6A05
:1006D000019301A95C304AF029FB77F0A9F80023C7
:1006E000B066F3662046FFF78BFF024AD6E700BFED
:1006F000C07A0B08DC7A0B0870B52DED028B00F583
:10070000C04686B0B36E0446002B4FD030465C30F6
:100710004AF00AFB90ED008A304650304AF004FB64
:10072000B2EE047AD0ED007AB4EEC78A04F5A7459C
:10073000F1EE10FACDED057A05F120053ADB9FEDDB
:10074000207AB4EEC78AF1EE10FA33D89FED1D7A05
:10075000F4EEC77AF1EE10FA2CDBFDEEC87A04F560
:10076000065017EE903A0DF113013E308DF813301C
:100770003EF0B4FD04F5065005A930303EF044FDCE
:1007800004F5005292F9BE31D2F8B0010393FBF7A1
:10079000BBFE039B0C4ACDE90001022128464AF02A
:1007A00035FE0023B3662046FFF72AFF06B0BDECF6
:1007B000028B70BD054A022128464AF027FEF0E769
:1007C0000000C84200000034F47A0B08177B0B08C5
:1007D0007FB500F5C0450446AB6E83B300F53150DC
:1007E00001A91C3070F004FD48B32846154E03964D
:1007F00003AA01A950304AF007FB04F52F53103328
:1008000028469B6A029303AA02A95C3003964AF029
:10081000FBFAEB6E0C4A5343B3F1333F02D8204648
:10082000FFF7EEFEEB6E0133EB6677F001F8AB6E8F
:10083000C01AB0F5FA6F02D32046FFF75DFF04B08F
:1008400070BD00BF0AD7A33CCDCCCCCC13B50446B9
:1008500000F5965006F06CFBD8B101A9134806F0DC
:1008600025FE04F57A500C306FF01CF89DF804302A
:1008700088B9DC06C3F300100BD49DF8052091075E
:10088000C2F3400005D41C07C3F3C00001D402F03A
:10089000010002B010BDD90603D41A07C3F3C0008B
:1008A000F7D583F08000C009F3E700BF403900208E
:1008B00070B500F50055D5ED747AF5EEC07AF1EE1D
:1008C00010FA8AB004464FF0000345D90793089305
:1008D000099307AE06AB019303AA05AB04A90096E2
:1008E00000F5965007F04CF9304620F0B9FFD5EDF1
:1008F000747A9DED047ADDED036AB4EEE70AF1EE59
:1009000010FAF4EEC77AACBF01230023F1EE10FA1F
:10091000F4EEE67A77EEA76A98BF0133F1EE10FAAB
:1009200098BF0133B4EEE67A98BFDBB2F1EE10FA6D
:1009300010DAF4EEC77AF1EE10FA9CBF0133DBB2A5
:10094000012B07D82046FFF781FF80F00100C0B2DD
:100950000AB070BD0120FBE70020F9E770B500F593
:10096000A045044695F868362BBB012685F86866D5
:1009700047F0FCFD3246112147F0B0FBD5F8500698
:1009800003685B6A9847B0B104F5005393F9CE3120
:100990008BB1022B06D004F5B8410622283120463F
:1009A00004F0BCFC04F5A740034ABDE870400221F6
:1009B00020304AF02BBD70BDC12D0B0838B500F5B5
:1009C000A043044693F868268AB1002583F8685648
:1009D00047F0CCFD2A46112147F080FB04F5A740E3
:1009E000034ABDE83840022120304AF00FBD38BD2F
:1009F000307B0B08F0B585B0054668460CF07EFEEE
:100A0000694605F5965007F08BF9D8B105F57A508F
:100A10000C306EF047FF344C344E40B105F50053B6
:100A2000D3ED747AF5EEC07AF1EE10FA0CD8238883
:100A300023F4FF7323F00103238028460023F3737C
:100A4000FFF7BCFF05B0F0BD2846FFF731FF0746B2
:100A500088B36378DB0705D423780133DBB2092B35
:100A600005D82370637803F00103F373EAE7238862
:100A700023F4FF7323F0010343F48573238047F0CD
:100A800075FD0222102147F029FB76F0D1FE636844
:100A9000C01A47F23053984209D905F5A740144AC5
:100AA000022120304AF0B2FC76F0C2FE6060284697
:100AB000FFF754FFD6E72378002BD3D0013B2370F8
:100AC0002388C3F30803B3F5807FCBD1637860F349
:100AD0000003637047F04AFD3A46102147F0FEFAE2
:100AE0002846FFF76BFFBDE7FC860020B587002096
:100AF000487B0B0810B5044676F08EFE0E4AB4F81B
:100B0000BE1013888B420D4B02D01180186010BDAF
:100B10001B68C01A0A4B9842F9D904F57A540C3470
:100B200020466EF0BFFE0028F1D020460122BDE82D
:100B300010400621FCF76EBE0487002008870020C5
:100B4000400D03002DE9F84F00F5A04591460446FD
:100B500095F858260E46002B71D042EA010385F81D
:100B6000583622B91BB176F063FEC5F85C0695F8DD
:100B7000603653B195F858363BB904F5A7404B4A57
:100B80004B46062120304AF041FC95F8603695F836
:100B90005826134085F86036002B40F08580002AE7
:100BA00000F0828076F044FED5F85C36DFED406AD6
:100BB000C01A04F5005A07EE900A9AED717AF8EE21
:100BC000677A27EE267AF4EEC77AF1EE10FA6BDD3B
:100BD000D5F8503604F5BF4808F11808434563D0EE
:100BE00004F5B8472837BB4205D104F54053D3F884
:100BF000943BDB0758D504F5A74B95F858362D4A9A
:100C000085F860360BF1200B4B46042158464AF01C
:100C1000FDFB52F05FFCD5F8502604F5BA4348338B
:100C20009A4214D1012E0DD19AF9C831022B0ED15E
:100C30005846214ABDE8F84F04214AF0E7BB22EAB2
:100C400001038CE7022E02D19AF9CC31EEE79AF932
:100C5000C031013B042B27D8DFE803F00B11031848
:100C60001D0004F5BF4119225431204604F056FB03
:100C7000D0B919224146204604F050FBA0B93946AC
:100C800020461922BDE8F84F04F048BB04F5BF41E7
:100C900019225431EFE704F57A500122BDE8F84FEC
:100CA00014210C30FCF7B6BDBDE8F88F587B0B085B
:100CB00000007A446C7B0B08787B0B08013A10B576
:100CC0000446042A2AD8DFE802F00A12031B200097
:100CD00000F5BF410422543104F020FBF0B904F5C3
:100CE000BF4104221831204604F018FBB0B904F5C6
:100CF000B84120460422BDE81040283104F00EBB64
:100D000000F5BF4104225431EDE700F57A50BDE80B
:100D10001040012207210C30FCF77CBD10BD000003
:100D20002DE9F84300F5025700F500582037044636
:100D30000021384698F8DC905CF00EF904F57A56FC
:100D40000C36054630466EF0ADFD002846D0002D2D
:100D500041D098F9A6305BB3294638465CF062F979
:100D6000DFED1F7AB4EEE70AF1EE10FA19D898F920
:100D7000A630013B042B1BD8DFE803F00B13032242
:100D8000270004F5BF410A225431204604F0C6FA78
:100D900070B904F5BF410A221831204604F0BEFAAA
:100DA00030B904F5B8410A222831204604F0B6FAD9
:100DB00047F0DCFB2A460921BDE8F84347F08EB92D
:100DC00004F5BF410A225431E7E701220F213046E2
:100DD000FCF720FDECE7B9F1000FE9D1BDE8F8839D
:100DE0000000C84201207047002070470120704772
:100DF0000120704710B50368DB680446984748B186
:100E0000E368DFED067A03F5C75393ED040A20EE9D
:100E1000270A10BD9FED020AFBE700BF0AD7233C5B
:100E20000000000010B50368DB680446984748B12D
:100E3000E368DFED067A03F5C75393ED030A20EE6E
:100E4000270A10BD9FED020AFBE700BF0AD7233C2B
:100E50000000000010B50368DB680446984728B11D
:100E6000E36803F5C75393ED050A10BD9FED010A32
:100E7000FBE700BF0000000010B50368DB68044614
:100E8000984728B1E36803F5C75393ED020A10BDF4
:100E90009FED010AFBE700BF0000000010B50368EA
:100EA000DB680446984738B1E06800F5CB50BDE8F0
:100EB0001040083003F0D2BE10BD000070B52DED1B
:100EC000028B5A4D84B0D5ED460A8DED010A0446D9
:100ED000806A0E4670F082FB8DED010A7EB3E068F9
:100EE00000F57766A06A70F04DFB6368D5ED461A91
:100EF00093ED831AF6EE000A60EE200A30469FED6D
:100F00004C0A01A95EF0ACFFE06800F5CB50083058
:100F100003F038FE98B1E66876F08AFCD6F8983F80
:100F2000C01AB0F5FA7F0AD205F5A043D3F85006EF
:100F300003F69843984202D003685B6D9847E068D7
:100F40009DED010A0023039300F5805393F968395E
:100F5000002B10DD00F5CB5003A9083003F0ECFFA7
:100F6000E0689DED030A00F51F6074F00FF904B00E
:100F7000BDEC028B70BDDFED2F7ADFED2F8A9FED88
:100F80002F8AB0EEC00AB4EEE70AF1EE10FA1FD4D1
:100F9000E368A06A93F8F0395A0745D490F84413EF
:100FA000D5ED461A9DED010A1B07A36858BF90F8BE
:100FB000442393F91E60D3ED040A01EE106AB8EEE3
:100FC000C11A48BF012221EE281A70F063FB1DE010
:100FD0001648FFF7ADF90028DAD1A268E36892ED70
:100FE000040A93F8F01992F91E3095ED461AA06A9A
:100FF00007EE903AF8EEE77AC1F3C00267EEA80A6E
:101000000DF10B03C1F3800170F0F2FB20EE080A32
:1010100006488DED030AFFF78BF90028A0D003489E
:1010200003A9FFF74FF99BE70121B9E780260020CC
:1010300000000000000000340AD7233C0000C84232
:101040000C4A02600C4A426002F56E6102F572625F
:10105000C2600A4A0261043242610432826104328F
:10106000C2610432026204324262A2F58E52816091
:1010700082627047A07B0B08403900208864002002
:101080000368DB6D1847000037B51D4B1B68DB6A32
:1010900093F89C3004460BB301A91A4806F006FAEF
:1010A0001948FFF7D3FB054620B1184B93F8685653
:1010B00085F00105236820465B6A984700B14DB171
:1010C000236820469B6A984740B13DB99DF804309B
:1010D0009B0703D40025284603B030BD2368204673
:1010E0009B6D984705460028F5D0236820461B6D68
:1010F0009847E06800F5CB50083003F0C1FCEAE700
:1011000078260020403900208026002080760020AC
:1011100070B52DED028B2F4C94F85836DB070D4639
:10112000164605D500230B601360BDEC028B70BD25
:10113000836893F91F30012BA4F5005420D0032BB2
:10114000D4F80C3EB3F9083007EE903AF8EEE77A9F
:10115000C2ED007A35D0002BD4F8083EB3F9083040
:10116000FFEE007AB7EE007AB8BFB0EE677A07EE0E
:10117000903AF8EEE77A67EE877AC5ED007AD4E721
:10118000D4F8080E52F0A8FBD4F80C0EB0EE408A4A
:1011900052F0A2FB78EE007AB6EE007A67EE877A1C
:1011A000DFED0D6A38EE408A67EEA67A28EE078AF0
:1011B000C6ED007ADFED097A28EE278A85ED008AF0
:1011C000B3E7D4F8083EB3F9083007EE903AF8EEEA
:1011D000E77AD2E7807600200000C84200A08C4564
:1011E00070B506462DED028B0D461446FFF790FFB5
:1011F000F06800F51F6074F06BF8A0B3DFED317A92
:1012000095ED000A722080EE270AB7EE001AFFEE75
:10121000000A1CF0FDFFDFED2C7AB0EE408A94ED61
:10122000000A732020EE270AB7EE001AFFEE000A2C
:101230001CF0EEFFB0EEC88AB0EEC00A38EE000A2D
:10124000F7EE007AB4EEE70AF1EE10FA0BDD95ED59
:10125000007AC7EE007AC5ED007A94ED007AC7EE09
:10126000007AC4ED007A194BF068D3ED460A94ED8C
:10127000000A00F51F6074F013F8DFED157A94EDA5
:10128000007AB4EEE77AF1EE10FAB4EEE70A94BF12
:1012900001220022F1EE10FA94BF012300239A42AA
:1012A0000BD0B36893F91F3033F0020302BFD5EDC2
:1012B000007AF1EE677AC5ED007ABDEC028B84ED21
:1012C000000A70BD00A08C450AD7233C8026002070
:1012D000000000B40A4B93F85826D2070DD4A3F5AA
:1012E0000053D3F8103E43B1B3F9083007EE903AFB
:1012F000F8EEE77AC1ED007A7047DFED027AF9E7A0
:10130000807600200000000070B5C36905461868AB
:101310000E46144658B152F09FFA86ED000A2B6A29
:10132000186838B152F098FA84ED000A70BD0023B5
:101330000B60F4E700232360F8E7000010B5436A70
:1013400018680C4620B152F087FA84ED000A10BDEF
:1013500000230B60FBE70000C36851B103F668721D
:1013600092ED000ADFED057AB4EEE70AF1EE10FA2D
:1013700003DA03F5805393ED500A70470000003400
:10138000C36803F5805383F8CD18704730B52DED51
:10139000028B3C4D9FED3C8A83B0002304462846D7
:1013A0008DF80330FEF7C4FFD4E90223DFED370ADE
:1013B00093F8F01992F91E30002848D001EE103A47
:1013C000B8EEC11AA06AD5ED461A9FED310A21EE9A
:1013D000201AD2ED040AC1F3C002C1F3800170F0FB
:1013E00059F920EE080A01A928468DED010AFEF7F9
:1013F00069FFE06800F5CB50083003F0A1FAE0681F
:101400009DED010A00F51F6073F0C0FE9DF80330EA
:10141000ABBBE368D5ED460A93F8F0199FED1C0AC3
:10142000A06AC1F3400201F001016FF067FFE068BC
:10143000DFED187A012120EE270A00F51F6073F016
:101440009FFE9DF8030003B0BDEC028B30BD07EE9C
:10145000903AF8EEE77A92ED040A95ED461AA06A02
:10146000C1F3C00267EEA00A0DF10303C1F38001CE
:1014700070F0BEF920EE080A8DED010AB9E79FED84
:10148000040AD4E7802600200000C8420AD7233C83
:101490000000000000A08C45B7EE007AF4EEC70A09
:1014A000F1EE10FA18DCDFED107AF4EEE70AF1EE57
:1014B00010FA11D4C368DFED0D6A03F5CD53D3EDF7
:1014C000037AF4EEE67AF1EE10FAB6BFC7EE207AB0
:1014D000B0EE670A20EE270ADFED050A40F27D1024
:1014E000B3EE0E1A1CF094BECDCC4C3D000000347F
:1014F0000000000070B52DED028B044682B0154649
:1015000001AA0E46FFF704FEA3689DED010A93F9B8
:101510001E20DFED200A07EE902AF8EEE77A20EE93
:10152000208A204667EEA00A93ED040AFFF7B4FF75
:1015300028EE000A184B85ED000AE068D3ED460A54
:1015400000F67C2070F04AF8DFED147A95ED007A11
:10155000B4EEE77AF1EE10FAB4EEE70A94BF012296
:101560000022F1EE10FA94BF012300239A420BD01F
:10157000A36893F91F3033F0020302BFD6ED007A5F
:10158000F1EE677AC6ED007A85ED000A02B0BDEC97
:10159000028B70BD0AD7233C80260020000000B4D7
:1015A000F8B5324F2DED028B0446D7F8080E0E46E3
:1015B000154652F091F9B7EE001AFFEE000AA62088
:1015C0001CF026FED7F80C0EB0EE408A52F084F9DB
:1015D000A720B7EE001AFFEE000A1CF019FEA36860
:1015E00093F91F30012BF0EE408A09D178EE008A82
:1015F00038EE407AF6EE007A68EEA78A27EE278A60
:10160000F0EE680AB0EE480A9AF036FFDFED187A7D
:1016100020EE270A1CF090FD86ED000A28EE080A4D
:10162000A8EEA80A1CF024FDA368DFED120A93F9C6
:101630001E20F7EE007AB4EEE70AB0EE408AF1EE33
:1016400010FA58BFB0EE678A07EE902AF8EEE77AF4
:1016500093ED040A67EEA00A2046FFF71DFF20EE77
:10166000080ABDEC028B85ED000AF8BD805600200B
:10167000A00CB3450AD7233C30B52DED028B83680F
:101680009B7F053B5F2B83B00546F0EE408A0C46FE
:1016900021D801AA6946FFF73BFDAB68DFED200AC0
:1016A00093F91E209DED018A93ED040A07EE902A1E
:1016B000F8EEE77A28EE208A284667EEA00AFFF7C0
:1016C000EBFEDFED187A28EE000AB4EEE70AF1EE41
:1016D00010FA03DBE4B1B0EE680A0DE0DFED127A38
:1016E000B4EEE70AF1EE10FA0AD8002CF3D0B4EE0B
:1016F000E80AF1EE10FAEEDC03B0BDEC028B30BD6F
:10170000002CF4D1B4EEE80AF1EE10FAE3D4F3E7DA
:10171000DFED057AB4EEE70AF1EE10FAF2D8DAE777
:101720000AD7233C00000034000000B410B52DEDB2
:10173000028B0368DB680446B0EE408A9847A8B184
:10174000E36803F5805393F93831002B0EDDBDEECD
:10175000C80A10EE103A1BB200EE103A2369B8EE38
:10176000C00A186852F0ECF9B0EE408AB0EE480AB0
:10177000BDEC028BE0680121BDE8104000F51F6060
:1017800073F0FEBC10B5C36893F8F019094B04461A
:10179000C1F34002806AD3ED460A01F001016FF007
:1017A000ADFDDFED057A204620EE270ABDE81040AA
:1017B000FFF7BCBF8026002000A08C4510B59FED30
:1017C000107AC368DFED0F7A93F8F0190E4B20EE14
:1017D000070A044660EEA70A20EE270A806A93ED06
:1017E000461AC1F3400201F001016FF087FEDFED00
:1017F000077A204620EE270ABDE81040FFF796BF83
:101800000AD7233C35FA8E3C8026002000A08C4568
:1018100010B5836ADFED157A93EDB91AB4EEE71AC5
:10182000F1EE10FAD8BFB0EE671ADFED117A21EEB3
:10183000271A0446F1EE410A4FF4F2701CF0E8FC5E
:10184000E368A06A93F8F0190A4BC1F34002D3EDA4
:10185000460A01F001016FF069FEDFED077A2046CC
:1018600020EE270ABDE81040FFF760BFCDCCCC3D8D
:101870000AE81C418026002000A08C45102937D89A
:10188000DFE801F0090D36111519361D3620232722
:101890002A36362E320000F5B8406030704700F529
:1018A000B9401830704700F5BE405C30704700F515
:1018B000B8402830704700F5BE401030704700F542
:1018C000C040FAE700F57550F3E700F5BA4048303C
:1018D000704700F5BF40E4E700F5BF405430704763
:1018E00000F5B9405030704700F5B7407030704790
:1018F0000020704782B073B50E4606A981E80C003F
:10190000C5680446DDE908018DE8030006AB05F56E
:1019100089500CCB31461C3071F0F2FA40B1E368CB
:1019200003F5C75318331B68E362002384F8303093
:1019300002B0BDE8704002B07047000070B52DEDF8
:10194000028BC368554D03F5805303F6D40293F818
:10195000CD1892ED000A0029B7EE007AFFEE007A6A
:1019600008BFF0EE477A044682B027EE800AFFF700
:1019700083FEE06841F23C16B0EEC00A304470F0DD
:1019800033FCE06895ED460A304471F0B7FAE06840
:1019900000F5C753183300F5CB501B68E3620830DD
:1019A00003F0F0F878B1E66875F042FFD6F8983F9A
:1019B000C01AB0F5FA7F06D205F5A045D5F8500655
:1019C00003685B6D9847E368226803F5C753126E9E
:1019D00093ED000A002120469047E06800F5895009
:1019E0001C3071F07FFAE06841F668163044B0EEC2
:1019F000408A03F047F9E56808B3A819B0EE480A31
:101A000003F074F9E0688DED010A304403F032F917
:101A10009DED010A80B1E36803F58053B3F94A31C3
:101A200000EE903AF8EEE00A204602B0BDEC028BE0
:101A3000BDE87040FFF7C2BEDFED190AF4E705F517
:101A4000C75393ED018A75F0F3FED5F8983FC01A9D
:101A5000B0F5FA7F17D2A06A6FF0B2FDA36AD3ED9A
:101A6000B67AF5EEC07AF1EE10FAD8BFDFED0C7A57
:101A7000B0EEC00AB4EE670ADFED097AF1EE10FAB3
:101A800098BFB0EE678AB0EE480A204602B0BDECBF
:101A9000028BBDE87040FFF775BE00BF80260020B6
:101AA000000000000120704700487047047C0B08CC
:101AB0000120704700207047F0B52DED028B85B0F6
:101AC00001A90446806A3D4D6FF092FB03AA02A96A
:101AD00000284DD12046FFF783FB2846FEF728FC5F
:101AE00018B103A92846FEF7EDFBE0689DED030A57
:101AF00000F51F6073F04AFBDDED027A9FED307A4E
:101B0000F0EEE77AF4EEC77AF1EE10FA05D4E06869
:101B100000F5CB50083002F0B3FFE0689FED298A52
:101B200041F66816304403F0A5F8E36858B39819F5
:101B3000A76A02F0B1FFE36895ED461A93F8F01931
:101B400003F58053C1F34002B3F94A3100EE903AF5
:101B500001F00101F8EEE00A38466FF0CFFC20EE0C
:101B6000080A2046FFF7E2FD05B0BDEC028BF0BD90
:101B70002046FFF7BFFC23689DED030A1B6E012181
:101B800020469847B8E7DDED027A93F8F0199FED0B
:101B90000E7AD5ED460AA06A87EE880A03F6B4638A
:101BA000C1F3400201F00101D3ED007A67EE877ABC
:101BB00020EE270A6FF0A2FBD1E700BF80260020AD
:101BC0000000003400A08C4535FA8E3C08B5C06892
:101BD00000F51F6073F07CFB80F00100C0B208BD0F
:101BE000C06800F5CB50083003F00CB80A207047ED
:101BF00000487047787C0B080120704790F830014E
:101C000000F0FD00031F58425841704790F83C30E7
:101C1000012B02D138301FF06BBF704790F9702054
:101C200022B190F8711009B9FFF7AABB7047000004
:101C300010B504460348FFF727FA10B1022384F8D1
:101C4000303110BD1886002030B52DED028B90F894
:101C5000324183B00546002C39D1AB6893F9151099
:101C60004A1C52D1D3ED067A9FED307AF0EEE77A36
:101C7000F4EEC77AF1EE10FA53D4AB689FED2B7AED
:101C8000D3ED067AF0EEE76AF4EEC76AF1EE10FAE9
:101C900049D4274B93F8AB2B0C2103F6980301FB97
:101CA000023393ED628AF4EEC87AF1EE10FA3AD874
:101CB00050F05CFA044618EE100AFAF725FC1D4AAB
:101CC000CDE900010421204649F0A0FB29E083680A
:101CD00093F915104B1C13D01548C9B203F09AFCA8
:101CE000012809D150F042FA134A042149F08EFB31
:101CF000002485F8324103E095F83231002BACD056
:101D0000204603B0BDEC028B30BD0948C9B203F0D8
:101D100081FC0028B1D150F029FA084A042149F089
:101D200075FB0124E5E70024EAE700BF000000346A
:101D300080260020AB7C0B08807C0B08937C0B0872
:101D400010B504460348FFF79FF910B1032384F848
:101D5000303110BD9085002010B5B0F86C30012BEB
:101D6000044607D850F002FA114A052149F04EFB0B
:101D7000002010BDC0689FED0F0A00F589501C308F
:101D800070F040FF00230C4884F8323101F052FB20
:101D90000A4803F05BFC18B12046FFF7D1FF10B9E9
:101DA000052384F83031012084F83101E1E700BFD8
:101DB000C87C0B0800000000508300208026002013
:101DC00070B505460E480C46FFF75EF9B0B1042326
:101DD00085F830310A4801F033FBA3680BB9E3689A
:101DE00053B194E80F0005F5A27686E80F00054987
:101DF00030460BF097FD012385F8543170BD00BFCC
:101E0000508300203C7C00201FB590F854310446DC
:101E10002BB375F00DFDD4F858311BB1C31AB3F5CF
:101E20007A7F1CD90DF10F03C4F8580100930D48B7
:101E30000DF10E030DF10D0212214BF021FA70B1DC
:101E400050F094F903689DF80F101B6998479DF8AE
:101E50000E209DF80D1004F5A2734FF009F804B0A0
:101E600010BD00BF6D8A002010B5144A13780446D7
:101E700043F08003137050F079F9114A052149F0BD
:101E8000C5FAE36803F5805393F93031022B0BD088
:101E9000032B0FD0012B03D12046FFF751FF10B9C0
:101EA000052384F8303110BD06490822064803F0A6
:101EB00035FAF4E705490822F8E700BFD487002087
:101EC000E47C0B081883002080260020E08200209C
:101ED0002DE9F04701F108030446884691460FCBEF
:101EE00092B003AE86E80F00274930460BF01AFD8A
:101EF000B8F9043023EAE372A4F83A2100229342AD
:101F00000DAFC4F83C21C8BF4FF0010938460BF0B3
:101F1000F5FB07AD0DF1240AB9F1000F15D02368C8
:101F200028465F6C0BF0EAFB9AE803008DE803009B
:101F3000314695E80C002046B84718B1002384F8D4
:101F40004031012012B0BDE8F087B8F8001001312F
:101F50000BAA89B204F1380021F006FE0028DED079
:101F600097E80F0085E80F00314628460BF0DAFCB1
:101F70009AE803008DE80300276895E80C003146D5
:101F80007D6C2046A847D8E73C7C002037B5044646
:101F90000D4675F04DFCC4F868011C4803F056FB73
:101FA00018B12046FFF7CCFE10B9052384F8303174
:101FB000D5ED027AF5EEC07AF1EE10FA16DD9FED5E
:101FC000147A67EE877AFCEEE77AC4ED597A50F01E
:101FD000CDF8D4F864214FF47A73B2FBF3F30D4AD1
:101FE000062103B0BDE8304049F010BA5AF0D8FAE3
:101FF0000023009395F90D2095F90E3095F90C10FA
:102000005AF06AFAC4F86401E1E700BF80260020B4
:1020100000007A44F87C0B088B8813B10831FFF775
:10202000CFBE704738B59FED180A0B7C2DED028BA3
:1020300091ED028A044628EE008A0D4653B14368AA
:1020400093ED800AB8EEC00A30EE080A1CF08AF858
:10205000B0EE408AE36895ED030A03F5805393EDF3
:10206000501A40F22F30F1EE410A1CF0D1F884ED05
:102070000D8ABDEC028B002384F83831012384EDF6
:102080004D0A84F8303138BD0000C84273B503688A
:102090009B6C05460E469847044640B395F8403180
:1020A0009BB9B5F83A31012285F8402113B350F0BD
:1020B0005DF8B5F83A31134A00930621338849F0A8
:1020C000A5F975F0B5FBC5F83C01B5F83A3173B127
:1020D00075F0AEFBD5F83C41041B4FF47A70B4FBAD
:1020E000F0F4B5F83A01844234BF002401242046BC
:1020F00002B070BD50F03AF83388034A062149F027
:1021000085F9E2E7087D0B08347D0B0810B504461D
:1021100075F08EFBD4F86831C01AD4F86431984257
:102120004FF0000084BFC4F86401012010BD00001E
:1021300003689B6C1847000010B5FFF7A7FF044623
:1021400028B150F013F8034A042149F05FF9204602
:1021500010BD00BF4C7D0B0810B590F83031042B3A
:10216000044618D18B88B3B190F8543123B9BDE837
:1021700010400A4801F072B900F5A27108480BF04E
:102180007FFDE36803F58053D3ED517AB4EEE70A9F
:10219000F1EE10FAEBD8012010BD00BF50830020F3
:1021A0003C7C00207FB501F108030C4606460FCBAE
:1021B0006D4685E80F00124928460BF0B3FB628894
:1021C000A388122A4FEA132305D1227ED20744BFE7
:1021D00003EB83035B00F068227A07EE903A00F588
:1021E000DC50B8EE670AC2F340022946083000F01E
:1021F0002DFF10B1072386F8303104B070BD00BF49
:102200003C7C00200B799FED0F6A07EE903A0B7E25
:102210009B07C36848BF9FED0C7AF8EE677A03F519
:10222000DC5348BF67EE877A93ED247AB0EEC77A25
:10223000C7EE066AF4EEE76AF1EE10FAACBF0120D1
:1022400000207047DB0FC9400000803B38B50446D2
:102250000D4675F0EDFAC4F86001D5ED027A9FEDF8
:10226000047A67EE877AFDEEE77AC4ED577A38BDD7
:1022700000007A4410B5044675F0DAFAD4F86031FB
:10228000C01AD4F85C3198424FF0000084BFC4F803
:102290005C01012010BD000010B503680446DB6B33
:1022A0009847D4ED577AF8EEE77A0020B4EEE70AC3
:1022B000F1EE10FA44BFC4F85C01012010BD00002B
:1022C00010B54B885C2B02460C4671D041D8103BB0
:1022D00099B2042936D94FF049FF63883E4A042158
:1022E00049F094F847E0C23B132BF4D801A151F810
:1022F00023F000BF7723010877230108D7220108C4
:1023000077230108D7220108D7220108D722010824
:1023100077230108D7220108D7220108D722010814
:10232000D72201087723010877230108D722010863
:10233000D7220108D7220108D7220108D722010895
:10234000C9230108042BC6D8DFE803F01A23282D7F
:102350001F00722B34D007D85D2B2DD0702BBAD133
:10236000BDE81040FFF786BFD52B06D8C12BBAD8E1
:10237000B23B012BAFD801200FE0DE2BFBD0AAE748
:102380002146BDE81040FFF781BEBDE81040FFF7D1
:10239000CFBE2146FFF77AFE002010BD2146BDE8E2
:1023A0001040FFF72FBF2146BDE81040FFF7C4BE25
:1023B000BDE81040FFF7D0BEBDE81040FFF7A6BE55
:1023C000BDE81040FFF768BF92F83031012BD2D141
:1023D00092F83801E1E700BF647D0B0838B50D467F
:1023E000FFF76EFF044620B14FF0C0FE29884DF084
:1023F00063F9204638BD000037B50368D1F80920DD
:10240000DB6C00EE102A0C46984768B14FF0AEFE28
:102410000546D4F80900FAF777F8044ACDE9000137
:102420000621284648F0F2FF03B030BD807D0B083E
:1024300089884B1E59425941FEF7A2BF8B8891ED06
:10244000040A03484FF47A71594300F0EFBF00BF0C
:102450005083002030B5684B1B68DB6A93F89C30D2
:1024600085B0044633B9B0F86C30012B9CBF05230E
:1024700080F8303194F83131E3B168460BF03EF921
:102480006068694605F04CFC50B104F1380021F059
:102490005FFF002384F8313104F5B6701FF0C0FAF5
:1024A00094F83031072B43D8DFE803F02444878DBC
:1024B0009381969C04F5B6701FF0B2FA04F13805CA
:1024C00080B194F83C30012B0CD194F830314BB9E9
:1024D000284621F0ABFD48B14FF048FE474A0221A3
:1024E00048F094FF284621F0CFFDD9E74FF03EFE9B
:1024F000434AF4E7434803F0A9F828B9204605B059
:10250000BDE83040FFF71ABAE06800F589501C308A
:1025100070F0CCFC0028F1D0E36803F5805393F809
:102520008C38002BEAD12046FFF70AFC0028E5D0C2
:1025300005B030BD94F8383183BBDFED330A94ED3C
:102540000D0A2046FFF73AF9DFED307A94ED4D0A97
:102550002368B4EEE70AF1EE10FA94BF01210021DE
:1025600020461D6EFFF788F801212046A8476368C2
:10257000D4ED0D7A93ED807AB8EEC77A77EEC77A0C
:102580009FED237AF0EEE77AF4EEC77AF1EE10FAD7
:102590004CBF0123002384F83831C9E7194803F000
:1025A00055F820B12046FFF7CBFB0028C0D12046CC
:1025B00005B0BDE83040FEF7E9BE164805B0BDE8FD
:1025C000304001F083BB144805B0BDE8304001F055
:1025D00069B92046FFF718FC104805B0BDE8304047
:1025E00000F07CBFE06800F5DC50083005B0BDE8C5
:1025F000304000F0E7BB00BF78260020907D0B083C
:10260000B87D0B088026002000000000000000B408
:102610000000FA4318860020908500205083002097
:1026200013B504468DED010A0091FFF70DFB0099EB
:102630009DED010A28B9204602B0BDE81040FEF722
:10264000A5BE204602B0BDE81040FEF737BC000032
:1026500090F83031072B1FD8DFE803F0041E0E116D
:10266000151E1518C36803F5C75393ED040ADFED73
:102670000C7A20EE270A70470A48FEF7BBBB0A4BCC
:1026800093ED000AF3E7094800F0E8BDC06800F5E3
:10269000DC50083000F018BA9FED050A704700BF03
:1026A0000AD7233C18860020C485002050830020D0
:1026B0000000000090F83031072B1FD8DFE803F04E
:1026C000041E0E11151E1518C36803F5C75393EDAC
:1026D000030ADFED0C7A20EE270A70470A48FEF75E
:1026E000A1BB0A4B93ED000AF3E7094800F0D2BD05
:1026F000C06800F5DC50083000F0B8B99FED050A5D
:10270000704700BF0AD7233C18860020C4850020EC
:10271000508300200000000090F83031072B17D8BC
:10272000DFE803F004160A160D160D10C36803F552
:10273000C75393ED050A70470748FEF78BBB074860
:1027400000F0C4BDC36803F5DC5393ED260A70475F
:102750009FED030A704700BF1886002050830020B9
:102760000000000090F83031072B19D8DFE803F0A3
:1027700004180A0D0F180F12C36803F5C75393ED21
:10278000020A70470848FEF777BB0848FBE708488D
:1027900000F0A4BFC06800F5DC50083000F048B974
:1027A0009FED040A704700BF188600209085002026
:1027B000508300200000000090F83031072B17D81C
:1027C000DFE803F00416070B0D160D1090ED0B0A51
:1027D0007047094B93ED000A7047084BFAE7084829
:1027E00000F082BDC36803F5DC5393ED0D0A70471A
:1027F0009FED040A704700BF44860020BC8500207E
:10280000508300200000000038B590F830310C46AD
:10281000072B2CD8DFE803F0042B14191E2B1E23E2
:10282000C06800F5805393F8CC583DB100F589504D
:102830001C3070F04DFB0FC884E80F00284638BDEF
:10284000BDE838400B4801F083BABDE838400A487B
:1028500001F020B8BDE83840084800F055BFC06816
:1028600000F5DC50BDE83840083000F0E7B800253E
:10287000E4E700BF188600209085002050830020E8
:1028800082B037B50D4606A981E80C000446DDE9A3
:1028900008018DE8030006AB0CCB29462046FFF764
:1028A00029F810B1002384F8303103B0BDE830407E
:1028B00002B0704790F83031062B11D8DFE803F0F2
:1028C00004100A100D100D00C06800F589501C306E
:1028D00070F0ECBA034801F0F3B9034800F0F2BD20
:1028E00001207047188600205083002090F8303176
:1028F000072B1BD8DFE803F0040A0E1A1104111489
:10290000C06800F589501C306FF05EBC80ED4D0A48
:1029100001207047064801F089B9064800F0F8BC6C
:10292000C06800F5DC50083000F042BB0020704762
:1029300018860020508300208B88012B08D107487F
:1029400090F86C3623B10021A0F5A040FDF7F8BC4B
:10295000034800220831FDF719BD00BF8076002032
:102960008026002038B54B88702B04460D4642D097
:1029700010D8142B08D80F2B0AD9113B032B20D8C1
:10298000DFE803F02A2C2A265C2B2BD05D2B2FD0DE
:10299000002020E0C22B37D00CD8B22B2ED0B32B86
:1029A0002FD0722BF4D1D1ED027AFDEEE77AC0ED93
:1029B000577A0FE0D52B18D0DE2BE9D1FFF73EFD7B
:1029C00008E0002229462046BDE83840FFF780BADB
:1029D000FFF72EF9012038BD0122F3E7BDE83840AA
:1029E000FFF7E0BBFFF718FBF4E7FFF71BFBF1E78E
:1029F000FFF7CCFAEEE7FFF729FCEBE7FFF7FCFC6B
:102A0000E8E7FFF799FFE5E7FFF712FDE2E70000CF
:102A1000092070470048704789670B0801207047FC
:102A200090ED240A7047000090ED0B0A70470000FB
:102A3000C36803F5CD5393ED740A704738B500F1C0
:102A4000440305460C460FCB84E80F00DFED067A01
:102A500095ED1B0AD5ED170A204620EE270A0BF04C
:102A600085F9012038BD00BFE02E654207B5C0687A
:102A700000F5CD5018306FF079F8DFED107A8DED5C
:102A8000000AB0EEC00AB4EEE70AF1EE10FACDED9E
:102A9000010A06D5F0EEE00AF4EEE70AF1EE10FACC
:102AA00009D468461DF0A4FFDFED057A20EE270A61
:102AB00003B05DF804FB9FED030AF9E70000003462
:102AC000E02E65420000000010B586B000230446E9
:102AD0000093019305F01EFB694604F07DFA18B9D6
:102AE0009FED130A06B010BD636F226F0492694612
:102AF00004A805931DF00AFFDFED0E7A8DED020AA2
:102B0000B0EEC00AB4EEE70AF1EE10FACDED030A1A
:102B100006D5F0EEE00AF4EEE70AF1EE10FADFD4A3
:102B200002A81DF065FFDFED047A20EE270AD9E741
:102B30000000000000000034E02E654210B504469D
:102B4000FEF77EFA20460B4B40F8443B0AF0D6FDD8
:102B50000023204608496365A36523676367A3676D
:102B6000E367C4F88030C4F884303BF06BFD204646
:102B700010BD00BF207F0B08D87E0B081FB50023B7
:102B800004460093019305F0C5FA694604F024FA5F
:102B900030B905F0BFFAD0F80C32E36604B010BDCE
:102BA00004F1540168461DF0B1FE02A88DED020A41
:102BB000CDED030A1DF066FFDFED077AB0EEC00A27
:102BC000B4EEE70AF1EE10FAE3D402A81DF010FF0C
:102BD00084ED1B0AE2E700BF0000003413B5D0ED1E
:102BE000170AC3689FED217A90ED1B0A426DF6EE3D
:102BF000007AF4EEE70ADFED1E7AF1EE10FA03F543
:102C00006B63B8BFF0EE477A93ED007A90F88C30A2
:102C10000267B4EE677AF1EE10FAC8BFF0EE477AB9
:102C200090ED247AB4EEE77AF1EE10FA98BF43F013
:102C30000103DFED107A80F88C3000F17001836DB4
:102C40004367044620EE270A084601911DF0C0FFA5
:102C5000E068094B019993ED460A00F5CD50183014
:102C600002B0BDE810406EF043BF00BFCDCCCC3DFC
:102C7000CDCC4C3EE02E65428026002030B52DEDB7
:102C8000048BC3684B4D90ED180A03F5CD5393EDBB
:102C9000611AF6EE007A21EE271AD5ED467A21EE7A
:102CA000271AD0ED1A7A044630EE670A85B0D32091
:102CB000F1EE410A1BF0ACFAD4ED1A7A94F8943094
:102CC00070EE277AF0EE408AC4ED1A7A002B6CD1B0
:102CD000DFED396A94ED177A636E95ED469A94EDBF
:102CE0001B0A27EE267A002B87EE878ABFEE007A32
:102CF00028EE268AF7EE007A18BFF0EE477A28EE23
:102D0000278AA9EE080A1BF06FFAD4ED227A84ED27
:102D10001B0AE9EE087AC4ED227A94ED1B0ADFED76
:102D2000277AA36D626DD4ED170A226704F1700152
:102D3000084620EE270A636703911DF049FFA36E42
:102D400094ED1B0ADFED1E7AA36704F178020023DD
:102D5000104630EE270AE36702921DF05FFFD4EDC4
:102D60001A7AD5ED466A94ED176A94ED1B0A67EE60
:102D7000E77A88EEA67A04F1800318460193C7EE3D
:102D8000866A84ED217AC4ED206A1DF047FFE06871
:102D90000399DDE9013200F5CD50183005B0BDECE6
:102DA000048BBDE830406EF0B1BE2046FFF7E6FE72
:102DB000B3E700BF80260020DB0FC940E02E65424C
:102DC000DB0FC93F30B52DED028B8BB000230446DD
:102DD0000293039305F09EF902A904F0FDF830B9BF
:102DE0002046FEF7D3FA0BB0BDEC028B30BD04F1E8
:102DF000540102A81DF08AFD636F226F079302A998
:102E000006A8CDED050A06928DED040A1DF07EFDA3
:102E100008A8CDED090A8DED080A1DF033FE04A8BF
:102E200084ED0B0A1DF02EFED4ED177A94F88C3049
:102E300030EE670AB0EEC00A84ED240AEBB92046F2
:102E4000FFF7CCFEE068344B00F5CD5093ED460A19
:102E500018306EF0BFFFE36803F5CD5393ED730AAE
:102E600093ED728A2046FEF78DFC236801211B6ECC
:102E7000B0EE480A20469847B5E7B6EE007AE36818
:102E8000F4EEC77A9FED257ADFED257AF1EE10FAA0
:102E900003F56B63B8BFF0EE477A93ED007AB4EEBA
:102EA000677AF1EE10FAC8BFF0EE477A37EEA77AEC
:102EB000B4EEC70AF1EE10FA1BDD94F8943023BB90
:102EC0009FED187AD4ED187A67EE877AC4ED187AF8
:102ED0004FF04CF90546206EF9F716FB124ACDE982
:102EE00000010421284648F091FA012384F8943027
:102EF000A8E7B4EEE70AF1EE10FA02D594F89430A0
:102F000043B92046FFF7BAFE9CE7B4EEE70AF1EEBC
:102F100010FAF6D50023E9E780260020CDCCCC3D81
:102F2000CDCC4C3ECDCC4C3F587E0B0837B5C3685A
:102F3000DFED1B7A03F5566393ED000AB4EEE70A62
:102F4000F1EE10FAD8BFB0EE670ADFED167A20EE88
:102F5000270AD0ED177A20EE270A04461BF088F8DE
:102F6000B5EEC00AF1EE10FAD8BF9FED0F0AD4ED0E
:102F7000187AF4EEC07AF1EE10FA0EDD84ED180A3C
:102F80004FF0F4F80546206EF9F7BEFA074ACDE98E
:102F900000010421284648F039FA03B030BD00BFD3
:102FA000CDCCCC3D0AE81C4100000000847E0B081B
:102FB000DFED137AB4EEE70AF1EE10FA10B504462D
:102FC0001CDB80ED180AFFF7B1FFE06894ED180AEA
:102FD00000F5CD53D3ED607AB4EEE70AF1EE10FAC6
:102FE00003F1180308DDD3ED5D1A93ED5C1AD3ED00
:102FF0005B0A18466EF0F4FC012000E0002010BDD2
:103000000000003437B5C36890ED177A03F56B63A1
:10301000D3ED007AB4EEE77AF1EE10FA044611D55A
:10302000C0ED177A4FF0A2F8E36803F56B6305462D
:103030001868F9F769FA044ACDE900010421284625
:1030400048F0E4F903B030BDA07E0B08F0B52DEDDB
:10305000028B0D4683B00023044669462846B0EE35
:10306000408A1746009301930AF0D0FC28B9002645
:10307000304603B0BDEC028BF0BD236820469B6D4B
:10308000984706460028F2D09FED110A68461DF0C9
:103090004DFCDFED107A84ED150AB0EEC80AB4EEEF
:1030A000E70AF1EE10FAD8BFB0EE670AC4ED160ACF
:1030B00084ED170A2046FFF7A5FF67662046FFF755
:1030C0005DFD95E80F00443484E80F00D0E700BFB1
:1030D0000AD7233CCDCCCC3D70B504462DED048BF6
:1030E00005F018F804F1540103F076FF06460028B5
:1030F00000F09C80D4ED0E7ADFED4E9A9FED4E9A53
:10310000DFED4E8AF0EEE77AF4EEE97AF1EE10FAAE
:10311000D8BFF0EE697AC4ED177A2046FFF772FF48
:1031200094F94030D4ED0F7A5A1EF4EEC97A534226
:103130005341F1EE10FA6366BEBFE36803F58053B6
:10314000D3ED507AC4ED187A04F0E4FFD0F80C32D5
:10315000E3663B4BC4ED1A8A0FCB04F1440585E8C6
:103160000F002046FFF7E2FE002384F89430E36866
:1031700003F67C2003F6485393ED008AB4EEE88A08
:10318000F1EE10FAD8BFB0EE688A6EF0FBF9B4EE3B
:10319000480AF1EE10FAF0EE400AC8BFF0EE480A15
:1031A000E068F4EEC90AF1EE10FAF7EE007A00F5E5
:1031B0008053B8BFF0EE670AD3ED577AF4EEC97AC0
:1031C000F1EE10FA06DBF4EE670AF1EE10FAC8BF72
:1031D000F0EE670AD3ED581A9FED167A9FED191A93
:1031E00094ED180A00F55663D3ED007AF4EEC91A8F
:1031F000F1EE10FAF4EEE97AB8BFF0EE601AF1EEF3
:1032000010FAD8BFF0EE477A41F6B81527EE811ACA
:1032100028446EF0E5FBE06828446EF063FD00236F
:10322000C4ED228A84F88C30C4ED248ABDEC048B72
:10323000304670BDCDCCCC3D000000340000000015
:103240003C7C00200AE81C410F2070470048704772
:10325000847F0B08012070470120704790F83830B8
:1032600023B1032B0CD09FED080A7047C36803F508
:10327000C75393ED040ADFED057A20EE270A704765
:10328000034B93ED000AF6E7000000000AD7233C49
:10329000C485002090F8383023B1032B0CD09FED6B
:1032A000080A7047C36803F5C75393ED030ADFEDBF
:1032B000057A20EE270A7047034B93ED000AF6E7E4
:1032C000000000000AD7233CC485002090F8383065
:1032D0002BB9C36803F5C75393ED050A70479FEDFB
:1032E000010A70470000000090F8383023B1032B2A
:1032F00005D09FED050A704790ED0B0A7047034B10
:1033000093ED000A704700BF00000000BC8500205C
:1033100090F838302BB9C06800F589501C306EF039
:1033200053BF00207047000030B52DED028B012502
:1033300087B080F838500446F0EE408AB0EE608ADC
:1033400074F076FA0023E0630193029304930593EB
:1033500094F838100948C4ED0D8A84ED128A84F877
:10336000395003AB6A46CDED008A8DED038AFBF739
:1033700015FD07B0BDEC028B30BD00BF80260020DC
:1033800010B52DED028B022386B080F8383004464C
:10339000F0EE408AB0EE608A74F04AFA012384F8B5
:1033A00039300023E063019302930493059394F86A
:1033B00038100848C4ED108A84ED128A03AB6A46BF
:1033C000CDED008A8DED038AFBF7E8FC06B0BDEC7D
:1033D000028B10BD8026002010B504460348FDF77F
:1033E00053FE10B1032384F8383010BD90850020BF
:1033F00010B504460B4802F029F918B12046FFF732
:10340000EBFF10B9052384F83830E0689FED060A19
:1034100000F589501C306FF0F5FB002384F8443030
:10342000012010BD8026002000000000C16580ED55
:10343000180A70470023C365002303667047000025
:1034400010B5044674F0F4F9034B60660FCB683492
:1034500084E80F0010BD00BF3C7C002010B5C36D98
:10346000044653B994ED187ADFED107AB4EEE77A9A
:10347000F1EE10FA0ADA002010BD74F0D9F9636E8B
:10348000C01AE36D9842EDD30120F5E7084804F136
:1034900068010AF0F5FBD4ED187AB4EEE70AF1EE14
:1034A00010FACCBF01200020E6E700BF0000003486
:1034B0003C7C0020C36803F58053D3F8780BC0F33D
:1034C0008010704790F838302BB9C06800F58950EB
:1034D0001C306FF0EBBC01207047000070B590F815
:1034E00038300446052B00F2D880DFE803F0032DC6
:1034F000709FA44AC06800F589501C306FF0D6FC5C
:1035000020B92046BDE87040FEF718BA94F8443060
:103510002BB10021654884F844104CF0CDF8644884
:1035200002F094F818B12046FFF756FF10B9204674
:10353000FDF72CFFE1685F4801F5C5510C310AF039
:103540009FFB84ED0B0A70BD90F8393083B174F0A5
:103550006FF9E36BC01A40F6B833984216D94EF0B3
:1035600005FE554A042147F051FF002384F8393005
:103570004F4802F06BF820B12046FFF72DFF0028DE
:10358000E1D12046BDE87040FDF700BF94F8393026
:10359000002BEDD0DFED490A94ED0D0A2046FEF731
:1035A0000DF994ED120ADFED467A2368B4EEE70ACE
:1035B0001D6EF1EE10FA204694BF01210021FEF7A6
:1035C0005BF820462B460121BDE87040184790F873
:1035D0003930002BCCD074F02BF9E36BC01A40F6D5
:1035E000B8339842BBD894F83930002BC0D0E36888
:1035F000D4ED107A9FED330A93F8F0192C4BA06AA2
:10360000D3ED460A67EE807A9FED2F0AC1F34002A0
:1036100027EE800A01F001016DF070FEDFED2B7ADC
:10362000204620EE270AFEF781F8BAE7BDE8704091
:10363000274800F037B990F84C30002B98D074F040
:10364000F7F8236DC01A40F6B833984208D9002322
:1036500084F84C304EF08AFD174A042147F0D6FE1C
:1036600094F84C30002B83D094ED150AE068DFED20
:10367000177A00F51F6020EE270A002171F080FD07
:1036800094ED160AE068DFED137ABDE8704020EE95
:10369000270A00F51F6071F079BD4EF067FDBDE8A7
:1036A00070400D4A042147F0B1BE00BF207A0020CF
:1036B000802600203C7C00208C7F0B08000000004E
:1036C000000000B40AD7233C35FA8E3C00A08C459C
:1036D000908500200000C842B57F0B0890F8383074
:1036E00023B1032B08D09FED060A7047C36803F58A
:1036F000C75393ED020A70470248FDF7BDBB00BFF8
:10370000000000009085002038B590F838300C4655
:1037100023B1032B12D00025284638BDC06800F520
:10372000805393F8CC58002DF6D000F589501C300A
:103730006FF0CEFB0FC884E80F00EDE7BDE838401E
:10374000014800F0A7B800BF9085002082B070B596
:10375000054688B00CAC84E80C00FFF7ABFEEC68C3
:1037600004F589540E461C34002833D0DDE90E01DF
:103770008DE803000CAB0CCB314620466FF0C0FB4C
:1037800030B30021012485F8381085F84440EB68F7
:10379000D6ED027A114803F5C653B8EEE77A143332
:1037A000D6ED037A1B6805930022F8EEE77A0492BF
:1037B0000692079205AB02AA8DED027ACDED037A4F
:1037C000FBF7ECFA204608B0BDE8704002B0704745
:1037D0000020F8E720466FF0CDF9D1E780260020E1
:1037E0000420704700487047917A0B08002070470A
:1037F000002070470020704713B50023044610488E
:103800000193FCF795FD18B10D4801A9FCF75AFD8D
:10381000E06800F5CB50083001F092F8E0689DEDCB
:10382000010A00F51F6071F0B1FCE0689FED050A28
:10383000012100F51F6071F0A3FC02B010BD00BFB4
:1038400080260020000000000520704700487047D7
:10385000A4800B080120704790ED0D0ADFED027A7D
:1038600020EE270A704700BF0AD7233C90ED0D0ACF
:10387000DFED027A20EE270A704700BF0AD7233C0B
:103880009FED010A704700BF0000000090ED0B0A99
:103890007047000010B538300C460FC884E80F00A0
:1038A000012010BD30B52DED028B044683B000F130
:1038B00038017C4801910AF0E3F9E06884ED0B0AD5
:1038C00000F5CB50083001F05DF9E368019900285C
:1038D00055D003F5CC5292ED027AD4ED0B7AF4EE8A
:1038E000C77AF1EE10FA4FD841F66815581901F071
:1038F00049F96D4BDFED6D7A9FED6D0AD3ED460A08
:10390000002808BFB0EE670AA06A6DF067FEE068A5
:1039100084ED120A284401F035F990B9E36803F503
:10392000805393F96829002A0BDDD3ED2C7A9FEDA3
:10393000617A67EE877A9FED607A67EE877AC4EDE9
:103940000D7AE06894ED0D0A41F66815284401F0FF
:1039500099F9002840F08D80DFED540A94ED0D0AAE
:103960002046FDF72BFF236894ED120A1B6E012100
:10397000204603B0BDEC028BBDE83040184703F58C
:10398000805292ED137AA8E703F5805303F51B628A
:1039900077EEC77A92ED007A4248DFED488A67EE0B
:1039A000877A93ED507AF4EE477AF1EE10FA48BF39
:1039B000B0EE677A84ED127A0AF07CF8B6EE008AEF
:1039C0009FED3F7A6368F0EE487AE0EE077AFDEE0D
:1039D000E77AF8EEE77AC4ED0D7A93ED800AB8EE57
:1039E000C00A37EEC00A1AF0BDFBF0EEC07AF4EE62
:1039F000E87AF1EE10FAE36804DD03F5805292F9FB
:103A000049202AB103F5805393F94930022B18D18C
:103A1000DFED2C7A94ED0D0A30EE270A1AF0A2FBA6
:103A2000636884ED0D0AD3ED807AF8EEE77A30EE24
:103A3000670A1AF097FBD4ED127AF1EE677AC4EDBB
:103A4000127AC0EE287A3620DFED180AB0EEE70AC7
:103A5000B7EE001A1AF0DCFBF7EE007AE0EE487AD7
:103A6000B0EE677AD4ED127A67EE877AC4ED127AF7
:103A700067E7E06894ED0D0A284401F037F9E06843
:103A800084ED0D0A284401F0F5F800283FF464AFF6
:103A9000E36803F58053B3F94A3100EE903AF8EE4B
:103AA000E00A5BE73C7C002080260020000000004C
:103AB000CDCCCC3DE02E65420000C84200A00C46B3
:103AC000A00CB34500A08C4638B50446C06800F58C
:103AD000895004F138011C306EF0E8FB054670B1E6
:103AE000A06A04F148016DF083FB08B90023A364C8
:103AF0006368D3ED807AF8EEE77AC4ED0D7A284654
:103B000038BD0000002070470048704718810B083E
:103B10000120704700207047002070470020704748
:103B2000C0689FED030A00F51F6071F04BBB00BF3A
:103B30000000000010B52DED028B86B0044601AAEE
:103B40006946FDF74DFB204602A9FDF7C3FBE3687C
:103B50009FED2D8A9DED000A03F5DC5380EE080AE7
:103B6000D3ED000A1BF002F820EE080A27488DED7D
:103B7000000AFCF7DDFB18B1244801A9FCF7A2FB01
:103B800004AA03A92046FDF7BFFB05A92046FDF7BF
:103B9000D5FBE0689DED030A00F51F6071F022FB84
:103BA000E0689DED040A00F51F6071F027FBE068F6
:103BB0009DED050A00F51F6071F02EFBE06800F531
:103BC000CB50083000F0D8FEE0689DED010A00F50A
:103BD0001F6071F0DBFAE0689DED000A00F580538C
:103BE00000F51F60D3F87C1B01F0010171F0C8FAE9
:103BF000E0689DED020A00F51F6071F0E3FA06B07F
:103C0000BDEC028B10BD00BF00A08C4580260020BB
:103C10000B207047004870471C3D0B08012070477F
:103C20000020704790ED0B0A70470000C06800F557
:103C300089501C306EF0C8BA70B58AB0044604F0E2
:103C400069FA90F87C32DB0702D400200AB070BD1C
:103C5000E36803F5895003F6687393ED000AB5EE47
:103C6000C00AF1EE10FA48BF9FED130A1C306EF047
:103C7000C9FF6368E66893ED9C0A104A06F5825115
:103C80001031B8EEC00A02A806AD3BF037FD284659
:103C900009F034FD0AAB13E903008DE8030006F5D3
:103CA000895095E80C0002A91C306FF029F9002812
:103CB000CBD001232387C9E7000000003C7C002013
:103CC000C06800F589501C306FF0F0B810B504469C
:103CD000C06800F589501C306FF0E8F820B9204624
:103CE000BDE81040FDF72ABE94F8383043B10023F8
:103CF00084F838304EF03AFA114A062147F086FB34
:103D0000104801F0A3FC60B92046FDF73FFBE168D5
:103D10000D4801F5C5510C3109F0B2FF84ED0B0AD5
:103D200010BD94F839301BB10848FFF7BBFDEEE732
:103D30000648FDF7A9F984F839000028E4D0F3E734
:103D40008C810B08802600203C7C00209085002080
:103D500038B5C06800F580530C4693F8CC583DB197
:103D600000F589501C306FF0B3F80FC884E80F00DD
:103D7000284638BD07207047004870470C820B0862
:103D800013B5044601AA6946FDF70AFCE36803F58A
:103D9000805393F964304BB994ED0E0ADDED007A4F
:103DA00030EE270A1AF0C8F98DED000ADFED0E7A21
:103DB0009DED017ADFED0D0AB4EEE77AF1EE10FA2F
:103DC000B5BFE36B009B0093E3639DED000A2046C3
:103DD000FDF7F4FC23689DED010A1B6E01212046CE
:103DE000984702B010BD00BF000000340000000082
:103DF0004368D3ED807AF8EEE77AC0ED0E7AD3ED22
:103E0000807AF8EEE77AC0ED0F7A70470C207047A1
:103E1000004870471B3D0B08012070470020704789
:103E200090ED0B0A7047000090F83800831E58424E
:103E300058417047C06800F589501C306EF0C4B915
:103E400030B590F83830012B0C460CD1C36803F51F
:103E5000805393F8CC5825B103F6AC030FCB84E81C
:103E60000F00284630BD0025FBE700001FB50446C3
:103E7000684609F043FC6068694603F051FF10B9D9
:103E8000002004B010BDE36893F8C42E002AF7D0D8
:103E900003F5895003F6687393ED000AB5EEC00A86
:103EA000F1EE10FA54BFBDEEC00A9FED0A0A1C30B5
:103EB000B8EEC00A6EF0A6FEE06800F589501C302E
:103EC0006EF040FA0028DBD0002384F8383084F804
:103ED0003A30D6E700000000064BC068D3F8502601
:103EE00003F6D473D21A18BF0122012100F6B8607C
:103EF0006FF06CBD8076002030B590F83830012B23
:103F000087B0044615D004D9023B012B72D907B003
:103F100030BDC068002100F6B8606FF00BF810B13A
:103F200040F201132387204607B0BDE83040FDF77B
:103F30002DBA90F83930002B3AD0C0680025694678
:103F400000F6B8600095019502956FF031FC48B914
:103F50004EF00CF9344A062147F058FA022384F84F
:103F60003830D4E7E068039503A900F6B8600495FB
:103F700005956FF04FFCE56841F23C1338B303AA96
:103F80006946E8186EF05CF978B94EF0EFF8274A08
:103F9000062147F03BFA032384F8383042F0B0FCA6
:103FA0003D224FF4801142F063FC002384F8393045
:103FB0002046FDF7C3FCE06800F589501C306EF028
:103FC00075FF0028A3D0012384F839309FE76946A4
:103FD000E8186EF00FF90028E7D14EF0C7F8134A41
:103FE000062147F013FA032384F8383042F088FCA6
:103FF0004522D6E7012380F830300D4801F026FB3A
:10400000002890D094F83A302BB10A4807B0BDE8A8
:104010003040FFF747BC0748FDF736F884F83A0010
:10402000002880D0F1E700BF8C810B0880820B084C
:1040300080260020908500200320704700487047AC
:1040400021550B0801207047002070470120704760
:1040500090ED0E0A7047000070B52DED048B84B012
:10406000044601A9806A6DF0C3F8B0B99FED4E8A8D
:10407000E068B0EE480A00F51F6071F087F8E0686C
:104080000121B0EE480A00F51F6071F079F884ED67
:104090000E8A04B0BDEC048B70BD03AA02A92046B1
:1040A000FDF728FADFED418A9DED039AE0689FED68
:1040B000408AB4EEE89AF1EE10FA00F51F6094BF62
:1040C0000126002671F004F9E368A56A98B3DDEDD6
:1040D000037A9FED387AF0EEE77AF4EEC77AF1EEE4
:1040E00010FA28D5DDED027A9FED337A87EE880A43
:1040F00003F6B4622846D2ED007A0022A26393F858
:10410000F0192E4B67EE877AC1F34002D3ED460AD1
:1041100020EE270A01F001016DF0F0F8204620EEB4
:10412000080AFDF703FB23689DED030A1B6E0121BE
:1041300020469847ADE703F56B63DFED210AD3ED29
:10414000007A95EDB97A9DED010A9FED1E1AF4EE05
:10415000E07AF1EE10FAB4EEE07AD8BFF0EE607AD1
:1041600020EE000AF1EE10FAD8BFB0EE607A27EE2A
:10417000011A80EE270A26201AF04AF83146204616
:104180009DED027AC7EE087AB4EEE89A27EE800A2F
:10419000F1EE10FA98BFB1EE400A84ED0E0A94EDEC
:1041A0000E0AFDF735FBBEE700000000000000B47A
:1041B00000A08C450000003435FA8E3C802600209B
:1041C000CDCCCC3D0AE81C4170B500F5A0460446B4
:1041D00096F8ED3BF3B16CF06FFD0368012203210B
:1041E0009B6898470C4B00251D6004F507500B4B4E
:1041F0000C301D603AF0FCFA04F5075008303AF034
:10420000F7FA04F507500D303AF0F2FA044B86F84D
:10421000ED5B5D7270BD00BF108700201487002029
:10422000B587002037B500F5A043044693F8ED3B71
:10423000002B34D073F0FCFA294B1B68C01A294BB1
:104240001B68984205D3204603B0BDE83040FFF715
:10425000BBBF254B1B78012B11D0022B21D0F3B90A
:10426000224BB3F9003000EE103A214B04F52F50E9
:10427000B8EEC00A1978103071F01AFD0DE01B4B32
:10428000B3F9003000EE103A194B04F52F50B8EE98
:10429000C00A1978103071F05BF80028D3D003B051
:1042A00030BD134B197804F52F55022905F110057F
:1042B00004F540530BD1D3F8080E01914FF00CFBDD
:1042C000DFED0C7A019920EE270A2846D4E7D3F8CF
:1042D0000C3EB3F9083000EE103AB8EEC00AF4E72D
:1042E0001087002014870020188700201A870020DC
:1042F0000C8700200000C8422DE9F843984600F5DD
:10430000A0439DF8206093F84C56BDF924700C46EC
:104310003DB9224A022120464AF0D6FA2846BDE895
:10432000F8836AB100F57A5001210C30F9F754F99D
:1043300030B91B4A022120464AF0C6FA0025EDE7B3
:10434000184B1B68D86A0368DB699847012801D1BC
:10435000154AEFE7B8F1040F06D9144A4346022183
:1043600020464AF0B1FAE9E7022E02D9104A334654
:10437000F5E7012E06D140F698039F42CEDD0D4AA7
:104380003B46ECE7002EC9D1642FC7DD0A4A3B4605
:10439000022120464AF098FA3546BFE77C830B0895
:1043A0009B830B0878260020B9830B08D3830B0866
:1043B000F2830B0818840B0836840B082DE9F043B0
:1043C0002DED028B00F5A04583B01E4695F8ED3B20
:1043D000BDF9308004461746B0EE408A2BBB134629
:1043E000721E18BF0122CDE90068FFF785FF28B9CA
:1043F000042003B0BDEC028BBDE8F0834FF001094F
:1044000085F8ED9B04F57A550C3528466BF04AFA91
:1044100050B304F50054002384F8CC3184F8C8313B
:1044200084F8CD31144B01225A7273F001FA9FEDDA
:10443000130ADFED137A134B28EE000A1860B4EE6E
:10444000E70AF1EE10FA58BFB0EE670A0E4BBCEE69
:10445000C00A002083ED000A0C4B1F700C4B1E702D
:104460000C4BA3F80080C4E74A4603212846F9F71D
:10447000A7F90028CDD1BBE7B587002000007A441A
:104480000060EA4610870020148700200C87002077
:10449000188700201A87002070B500F507562436CB
:1044A000054630464FF0EEF805F54054C4F8080EC6
:1044B00030464FF0FBF8C4F80C0E30464FF000F9D0
:1044C00041F29411C4F8100ED4F8080E4FF048F9D8
:1044D000D4F80C0E64214FF043F9D4F8100E10B14B
:1044E00064214FF03DF9C921304650F091F8CA21BE
:1044F000C4F8140E304650F08BF8D321C4F8180ECF
:10450000304650F085F8C4F81C0ED4F8140E40B1B3
:1045100041F294114FF024F9D4F8140E1E214FF0FB
:1045200023F9D4F8180E40B141F294114FF018F964
:10453000D4F8180E1E214FF017F9D4F81C0E40B114
:1045400041F294114FF00CF9D4F81C0E1E214FF0DB
:104550000BF905F56D50083000F0F4F805F57A50C8
:104560000C306BF09FF940B905F52F5410342046FC
:1045700070F0DAFD204670F0B7FD084B1B685B6AEF
:104580004FF47A72DA804FF4FA6205F514501A810A
:10459000BDE870404621343050F092BB78260020B0
:1045A00010B500F540541E21D4F8080E4FF0DCF889
:1045B000D4F80C0E1E214FF0D7F8D4F8100E20B10D
:1045C000BDE810401E214FF0CFB810BD70B500F50A
:1045D0000053054693F9C8210C46DAB1B3F9CA6114
:1045E00073F026F905F5A043D3F86436C01AB0F588
:1045F000FA7F0DD8B3B29C422CBF00230123064A98
:1046000093722846054ABDE870400121FCF79ABA2A
:104610000123F4E770BD00BFB58700205C840B0860
:104620002DE9F84300F54058054698F99C9EB9F1EC
:10463000000F09D0D8F80C0E4FF000FA05F5A04491
:1046400020B90023C4F8CC3BBDE8F883D4F8500669
:1046500003685B6998470028F3D005F57A560C3655
:1046600030466BF01FF90746B8B9D8F8083EB3F9E1
:104670000830B3F57A6FE4DD73F0DAF8D4F8CC3BA8
:1046800073B3C31AB3F5FA6FDED30122394630464D
:10469000F9F796F8C4F8CC7BD6E7B9F1020FD3D17D
:1046A00005F52F50103071F037FF05460028CBD1AB
:1046B000D8F8083EB3F9083013F57A6FC1DA73F011
:1046C000B7F8D4F8CC3B5BB1C31AB3F5FA6FBBD3E0
:1046D000012229463046F9F79DF8C4F8CC5BB3E7D0
:1046E000C4F8CC0BB0E7000038B5044600F507501D
:1046F00024304EF0A9FE04F5405538B9D5F80C3EEB
:104700002046D988BDE83840FFF760BF73F090F8C5
:1047100004F5A043C3F86406D5F80C3E2046D988BA
:10472000FFF754FF2046BDE83840FFF779BF00008F
:1047300010B50349044639F085FF204610BD00BF7F
:10474000D0840B0810B504464EF0C4FFCF214FF0C3
:104750005FFF48B1606264214FF002F8606A1E2179
:10476000BDE810404FF000B8024BD3F80C3E636236
:1047700010BD00BF8056002038B52DED088BDFED51
:10478000627A624D9FED62BAD5ED460ADFED61BAFD
:10479000DFED618AF0EE40AA90ED040A044620EEB7
:1047A000270A5E4805F540556CF0B4FCD5EDA27AB9
:1047B0009FED5B7A67EE877ABFEE008AF4EECB7AE4
:1047C000F1EE10FAB7EE001AF4EEEBAA88BFB0EEE5
:1047D000418AF1EE10FA20EE28AAB0EEE79A76DBD5
:1047E00094ED030A94ED021AD4ED010AD32039EEB8
:1047F000400A19F00DFDF0EE680AB0EE401A94ED93
:10480000022AD4ED011A9FED470A19F041FCDFEDB1
:10481000450A3AEE000AD820B0EE681A19F0F8FC02
:10482000414870F007FDF4EECBAAF1EE10FADFED8F
:104830003A7A3D48B4EEE8AAF7EE009ABFEE000AD5
:1048400088BFB0EE690AF1EE10FA48BFF0EE4A7A7E
:1048500078EEE78A68EE888A28EE800A70F0FCFC21
:10486000F4EEEBAAF1EE10FA4BDB94ED037AB4EE22
:10487000C97AF1EE10FA44DCDFED2C8A77EE287A63
:10488000F4EEC97AF1EE10FA24DDDFED296AF0EEDC
:10489000697AEAEE667AF5EEC07AF1EE10FAD8BFE0
:1048A000DFED207AA7EE679A28EE091A94ED022A26
:1048B000DFED190A9FED1F0AF1EE421A19F0E8FB2D
:1048C000BDEC088B1848BDE8384070F0D7BCB0EE9E
:1048D000680AA5E7DFED187AB4EEE79AF1EE10FA70
:1048E0000CDD892050F090F89FED141AB4EECB0A3D
:1048F000F1EE10FA88BFB0EE681AD7E728EE281A52
:10490000D4E79FED080ADBE735FA8E3C80260020CD
:10491000000000B4000000340000C842DC52002057
:10492000E02E654200000000505200200000B4421A
:104930000AD7233C0000C8C2000007430000B4C2ED
:1049400007B59FED0A0A0A4870F074FC9FED090A4A
:1049500007488DED010A70F07FFC9DED010A0448C7
:1049600003B05DF804EB70F089BC00BF0000C842E2
:10497000505200200000000010B5204B93F858362C
:10498000DB07044601D4436A23B92046BDE8104042
:10499000FFF7D6BFB3F908309FED191ADFED190AFA
:1049A00000EE103AB720B8EEC00A19F031FC1648F4
:1049B00070F040FC636A9FED121AB3F90830DFED26
:1049C000130A00EE103AB820B8EEC00A19F020FC25
:1049D0000D4870F041FC636A9FED091AB3F9083085
:1049E000DFED0A0A00EE103AB920B8EEC00A19F05D
:1049F0000FFCBDE81040044870F040BC80760020F9
:104A00000000C84200000000505200200000C8C250
:104A100013B5154801A96CF0EBFB10B3134CD4F897
:104A200050060368DB68984718B99DED010A02B08B
:104A300010BD0F4B9FED0F7AD3ED007AA4F56C53A8
:104A400067EE877A13ED0D0A9FED0B7A97EE870AD2
:104A500019F0CAFB97F0EEFADDED017A20EE270A95
:104A6000E5E79FED060AE2E7DC52002080760020B1
:104A7000506100200AD7233C35FA8E3C000000002C
:104A800010B5002380F8283080F83C3003630446DA
:104A900072F0CEFEA06310BD10B5114B90ED0B0A65
:104AA000D3ED007A30EE670A044619F09DFBDFED86
:104AB0000D7AB0EEC00AB4EEE70AF1EE10FA05D5B1
:104AC0002046FFF7DDFF94ED0B0A10BD72F0B0FE3B
:104AD000236BC01A41F288339842F1D8F3E700BF44
:104AE0004C3B0020C2B8323E70B5054616460C4617
:104AF00009B92C6470BD0C4870F0EAFB0028F8D1AD
:104B0000462050F011F90028F3D1084B93F92832D0
:104B1000002BEED1002EEDD04DF028FBBDE870400B
:104B2000034A042146F072BC5052002080560020F7
:104B300064840B0810B5036C012B044601D00020DF
:104B400010BD90ED067ADFED0C7AB4EEE77AF1EE67
:104B500010FAF4DB09486FF0F7FB0028EFD0084BA0
:104B6000D4ED067A93EDBB7AB4EEE77AF1EE10FA63
:104B70004CBF01200020E3E700000034C8580020AB
:104B80008056002008B590F90020002A08DD036C4B
:104B9000022B05D0FFF7CEFF80F00100C0B208BDA8
:104BA0000020FCE713B590F90030002B04460EDD21
:104BB000002311488DF807300DF107013AF060FB32
:104BC000236C0E4A023B18BF012382F86E3A20463E
:104BD000FFF7D8FF38B1012309488DF807300DF1F0
:104BE00007013AF04DFB00220121204602B0BDE84A
:104BF0001040FFF779BF00BF1058002080560020FA
:104C0000A958002010B52DED028B0446FFF7BAFF1E
:104C1000E0B194F82830CBB9012384F828300D4B4B
:104C200093ED008A0C4B93EDA40A30EE480A19F07C
:104C3000DBFAF0EE007AA0EE278AB0EE480A19F00F
:104C4000BDFA84ED0B0A72F0F3FD2063BDEC028B1C
:104C500010BD00BF4C3B00208056002010B504461C
:104C6000FFF790FF28B194F8283013B972F0E0FDF7
:104C7000206310BD10B50446FFF784FF08B194F817
:104C8000280010BD10B52DED028B0446B0EE408A11
:104C9000FFF778FF00B394F82800E8B9DFED107A49
:104CA000104B27EEC87A93EDA40A9FED0F8AA7EE6A
:104CB000080A19F099FAD4ED057AB2EE047A77EE83
:104CC000877AB0EEC00A67EE887AB4EEE70AF1EEB2
:104CD00010FA94BF01200020BDEC028B10BD00BF74
:104CE0000AD7233C8056002035FA8E3C2DE9F84344
:104CF0002DED048B0446B0EE408AFFF743FF81465A
:104D0000002800F0D580DFF82C82DFED7E7AD8ED28
:104D1000A49ADFED7D8A98F8087367EEC87AB0EE42
:104D2000699AA7EEA89AB0EE490A19F05DFAD4ED97
:104D3000057A67EEA87AB0EEC00AB4EEE70AF1EEA3
:104D400010FA40F3A48094F82830002B40F09F80A4
:104D5000B0EE490A19F048FADFED6C7AB4EEE70AD2
:104D6000F1EE10FA8CBF012300239F4200F0A080D7
:104D7000D8EDA27AB0EEC00AF0EEE77A37EE800AFC
:104D8000DFED637AB4EEE70AF1EE10FA40F19080BD
:104D90004E4672F04DFD236B054653B14EB994F863
:104DA000282032B9C31AB3F5FA7F2CBF002601269A
:104DB000226308F6D42898ED007AD4ED077AF0EE55
:104DC000C76AF4EEE76AF1EE10FA1EDBDFED516A16
:104DD000F0EEE77AF4EEE67AF1EE10FA15D4A6B921
:104DE00094F828308BB9B4EEE67AF1EE10FA02DBD3
:104DF0007B1E5E425E41DFED457AB4EEE77AF1EE6E
:104E000010FA02D8002F08BF4E46D4ED057A9FED68
:104E1000428AB0EE690AA7EEA80A19F0CFF9D4EDDC
:104E2000057AB0EE409AB0EE690AA7EEE80A19F0EA
:104E3000C5F9DFED3A9AF0EE408A86B3A36B41F2F2
:104E40008832EB1A93422AD94DF090F9344A062160
:104E500046F0DCFAEFB1012F1ED0012384F8283090
:104E60006563304B94ED0B0AD3ED007A30EE670AA0
:104E700019F0BAF9DFED2C7AB0EEC00AB4EEE70A09
:104E8000F1EE10FA1AD82046FFF7FAFD2CE00026C2
:104E90007FE7C4ED0B8AE0E784ED0B9ADDE794F839
:104EA0002830002BDDD10FBB29EE299A29EE088A84
:104EB000B0EE480ABDEC048BBDE8F883606B41F2AC
:104EC00088332D1A9D420FD9236C012B13D107EE85
:104ED000905A9FED167AF8EE677AF4EEC77AF1EE03
:104EE00010FA08D584F83C30D4ED0B8A68EEA98A14
:104EF00028EE888ADCE74DF039F90D4A062146F0A4
:104F000085FAC0E70AD7233C35FA8E3C000000B48E
:104F1000DB0F4940000000340000C842E02E65422B
:104F200088840B084C3B0020C2B8323E00606A46C1
:104F30009A840B088056002038B52DED028B002393
:104F40000B6090F90030002B0446B0EE408A0D460D
:104F500006DCBDEC028B2046BDE83840FFF7F0BC14
:104F6000036C022B2ED11D4A9FED1D1AD2ED461A5D
:104F700002F50053D3ED6C0A93F9BE0193F8D01BF0
:104F800007EE900AF8EEE77AC1F3C00227EE811A25
:104F9000C1F38001B0EE480A03F65C406CF07AFB86
:104FA000DFED107A20EE270A85ED000A236C022B34
:104FB000CFD0B0EE480ABDEC028B2046BDE83840A9
:104FC000FFF7DABB012B03D190F83C30002BCAD19C
:104FD0002046FFF7AFFD0028C5D1E7E78026002077
:104FE0000AD7233C0000C84200F2545009F080BBAD
:104FF00010B5044609F06CFC90F921308BB190F8A3
:10500000403373B194F978355BB104F57A500C30C4
:105010006AF048FC28B904F25450BDE8104009F089
:105020007FB910BD2DE9F0432DED028B00F500573F
:1050300083B097F8B0390646002B00F0938000F556
:1050400024543C34204668F071FD4FF0000841F2D2
:10505000F46997F8B0295FFA88F5AA420BD9294676
:10506000204668F0B7FD4D4406EB850585ED000A46
:1050700008F10108EDE706F5A04595F8D83BEBB936
:10508000012285F8D82B1D4697F8B0395FFA85F9CB
:105090004B4567D94946204668F07CFD06EB8908F8
:1050A00008F5A04808F6DC3383ED000A494620469F
:1050B00068F036FE0135C8F8E40BE5E795F8EC3BFF
:1050C0000133DBB2934228BF002385F8EC3B95F80F
:1050D000EC1B204668F05EFD95F8EC1B2046B0EE18
:1050E000408A68F01DFE074672F0A2FB95F8EC1BA3
:1050F00006EB810303F5A04303F6DC32D2ED008A10
:1051000082ED008AD3F8E42BA7EB020808F1FF3CFC
:10511000BCF1630F84BF0746A0EB0208C3F8E47B31
:10512000204668F02FFD95F8EC1B0190204668F0B2
:105130001DFD07EE908ADFED0E0A019AF8EE677A00
:1051400078EE688A67EEA00AB0EE401A3946B0EEF3
:10515000680A06F5965003B0BDEC028BBDE8F0433B
:1051600020F080BD03B0BDEC028BBDE8F08300BF32
:105170006F12833A10B5044600F551603AF0E6FD2F
:105180002046BDE81040F9F78FBD0000F9F7B8BF21
:105190000148FBF7AFBC00BF8026002070B52DEDA5
:1051A000048B00F54053044693F94C31022B56D042
:1051B00000F5005505F53D6393ED0A9A95F9BE316A
:1051C00008EE103AB8EEC88AF6EE008A28EE288A71
:1051D000F2EE0E7A00F53156B4EEE78A1C36F1EEA7
:1051E00010FA304658BFB0EE678A6CF0D9F948B172
:1051F00030466CF0E5F9B4EEE80AF1EE10FACCBFF7
:1052000001200020B4EEC98AF1EE10FA04F5A046A0
:105210000BD405F53D6595ED0A7ADFED127AB4EE13
:10522000E77AF1EE10FA16DBA8B172F001FBD6F8BE
:10523000C83B0BB9C6F8C80BD6F8C83BC31AB3F5C0
:10524000FA6F94BF0023012304F5805484F8C93514
:10525000BDEC048B70BD0023C6F8C83BF4E7002307
:10526000F2E700BF0000003408B5044A0B2341F008
:10527000B9F980F00100C0B208BD00BFFC850B0881
:1052800038B5044600F5A740144A0621203046F000
:10529000BDF8134B1B68986A036864215B6804F5CA
:1052A00096559847284601F025FC04F580530122C5
:1052B00083F8C92583F8D424B4F9A43004F69800FF
:1052C0001BB9B4F8A230A4F8A430B4F8A41018F0B4
:1052D00009FB2846BDE8384001F012BD70850B0877
:1052E0007826002070B50B680B4EDB680546084633
:1052F0000C4698473074236820461B689847F07026
:10530000236820465B689847014605F593501030A6
:10531000BDE8704036F0BEB9B58700202DE9F047F2
:1053200000F5A0470646D7F850368B420C4691460A
:1053300064D000F5A748022A08F1200816D10B68AE
:1053400008461B68984701463046FFF78DFF054623
:1053500060B9236820465B689847294A03460521BF
:10536000404646F053F82846BDE8F0872046D7F877
:1053700050A6FBF789FE054688B943F0F7F8236885
:1053800006461B68204698470A210246304642F0EE
:10539000A5FE1C4A0421404646F038F8E3E706F52E
:1053A0000250C7F85046203057F060FED7F850063C
:1053B00003681B689847A0F10A035842584106F554
:1053C000005487F83C065046FBF75AFE84F85C917F
:1053D000D7F8500603681B68984794F85C2101468B
:1053E00006F57C6042F09EFA404600214DF0B8FA86
:1053F000D7F850163046FFF775FFB4E70125B2E73E
:10540000A0850B08E0850B0873B505460A48019294
:105410000E46FCF733FA019A044630B101460648BD
:1054200002B0BDE87040FFF779BF2846314641F031
:1054300021F8204602B070BD802600200148FFF709
:10544000E3BF00BF80260020F0B5044604F5A04667
:1054500000F5935087B0103036F0D0F8D6F85016DB
:105460002046FFF73FFF04F5AD401C3005F0B0FBD0
:1054700004F57850283050F045F804F58650143083
:1054800050F0BEFB04F58F5104F54950083104F586
:10549000866508306EF05EFF284605F04FFA04F589
:1054A000A74020304AF070F904F57B5008305BF0DB
:1054B00063F909F00DFA4FF40063036309F008FA89
:1054C0000AF07EFA04F5005380279F634FF480634F
:1054D000C4F8BC3F002104F551603BF031F80121D4
:1054E0002846C4F8447405F0B9F80423C4F87431AC
:1054F00004F5907010F074FA4FF40023C4F8B03B38
:10550000204604F54057FFF74BF804F52F5097F865
:105510002812103070F0E4F94FF05AFE4FF042FBC1
:1055200004F524503C3068F0CFFA04F591501C305B
:1055300052F090FA04F5AB404C3006F05FFD2F4B73
:105540002F491B68986A03684FF47A72DB6A9847A0
:1055500004F5B74504F54250183070356DF050FE33
:105560001A2229462046FFF7D9FE2046FFF788FE7B
:1055700004F5BB401DF00CFF4FF48073C6F8743E79
:10558000204B0493204B059306AB13E9060004F56A
:105590007C6041F0DFFF04F50053204693F8A91129
:1055A000FCF76CF91A22002814BF01462946204650
:1055B000FFF7B4FE04F50750243099222921019009
:1055C0004FF068F89B22052101984FF063F801988D
:1055D0004EF028F80D48FFF7E5FA97F94C31022B09
:1055E00007D101230A488DF80F300DF10F0139F072
:1055F00047FE012386F84C3607B0F0BD7826002020
:1056000091510108802600208D510108C8610020B9
:105610009059002070B50A4B1D68E86903680022A4
:105620005B680C469847E869036821461B690122BC
:105630009847E86903682146DB68BDE87040184771
:105640007826002000F57C6042F0B6BD00F54050A1
:1056500090F94C01831E58425841704713B50446D7
:10566000143000F0F1FE04F12C0000F0EDFE04F126
:10567000740073F0D1FC04F1F40073F0CDFC4FF032
:10568000FF331549C4F85031204638F0DBFF0023C2
:105690000DF1070104F128008DF8073039F0F0FD15
:1056A00001230DF1070104F129008DF8073039F0CD
:1056B000E7FD0F230DF1070104F125008DF80730F8
:1056C00039F0DEFD054B1A6812B1054872F07EF81C
:1056D00020461C6002B010BDB8870B081C87002054
:1056E00008860B082DE9F0478CB003A938F074F850
:1056F00060B300210D2208A807AF1C4CDFF87080B2
:10570000DFF8709007910B2699F0B0F80697237A8E
:10571000DFF864A08DF81430002554F82530049388
:10572000D8F80000E368B5B90093C06A5346112267
:10573000394615F083FB0021B7EE000A03A838F0C4
:105740004FFA35B1013E04F11004E0D10CB0BDE8D0
:10575000F0870125E1E701930223009311224B46D4
:105760003946C06A15F06AFBE5E700BF58880B08A8
:105770007826002065860B085C860B082DE9F74F1C
:10578000D0F85431044683BBDFF88CA1074600F102
:10579000740800F5AA750126721ED2B297ED070AA9
:1057A0000192404673F058FCFB69C8F83C304FF05A
:1057B0007E53C8F8483097F92830019A013B5FFAC8
:1057C00086FB0E2B20D8DFE803F0133E4A576069B2
:1057D0001F1F1F1F1F1F891F7A00D4F8543103B9E0
:1057E0006361D4F8583103B9E36203B0BDE8F08FC8
:1057F0004820019208F0E4FA814618B1019A214646
:1058000072F0CEFBC5F80090286890B103689B68E1
:105810009847002874D14CF0A9FC3C4A3346032138
:1058200045F0F4FD286810B103685B6898470023D1
:105830002B60022E07F1180708F1800805F1040516
:10584000CBD00226A8E72820019208F0B9FA8146B9
:105850000028D7D0019A214673F0C6FBD2E7682012
:10586000019208F0ADFA81460028CBD0FF23019ABF
:10587000214672F037FEC5E76820019208F0A0FAD1
:1058800081460028BED00023F1E76820019208F08D
:1058900097FA81460028B5D00123E8E74420019219
:1058A00008F08EFA81460028ACD0019A214672F0A9
:1058B00039F9C9F800A00023C9F84030A2E7442014
:1058C000019208F07DFA814600289BD0019A21467A
:1058D00072F028F90E4BC9F80030ECE76020019215
:1058E00008F06EFA814600288CD0019A214672F0A9
:1058F00019F9084BC9F800300023C9F8243081E7B2
:105900002B68002B95D084F84FB192E742860B08A4
:1059100000CE0C0818890B0834D00C0813B50446C7
:10592000FFF7E0FE204638F0ADF868B994F928306A
:1059300013B994F940303BB101230DF10701204622
:105940008DF8073039F0CAFC94F90030002B08DDDF
:1059500094F928302BB1204602B0BDE81040FFF783
:105960000DBF02B010BD00000346406C012807D0F7
:10597000032805D0986C012802D0032818BF022004
:105980007047000090F90030002B0ADD012908D88B
:10599000182303FB010090F92800003818BF0120EC
:1059A000704700207047000037B50446FFF7EAFF54
:1059B0009FED0B0A0D4680B104EB81038DED010ACA
:1059C000D3F8540138B1036801A9DB68984704EBA8
:1059D000C51484F865009DED010A03B030BD00BF19
:1059E0000000000070B50446FFF7CCFF50B104EB97
:1059F0008104D4F8540128B10368BDE870401B69E4
:105A000011461847002070BD2DE9F04F2DED028B97
:105A100090F90030002B83B00646894653DD2C4BAD
:105A20001B68D86A03685B689847044650B14CF01D
:105A30009DFB284A062103B0BDEC028BBDE8F04F68
:105A400045F0E4BC9FED248ADFF890A0DFF890B029
:105A5000354606F14407B04621463046FFF792FF2F
:105A600020B195F8643043B188ED068A803504375B
:105A700008F118083CBB0124EEE7B9F1000F03D090
:105A800098F92630002BF1D1D7F81021631C01932F
:105A90003AB94CF06BFB019B5A46032145F0B6FC2A
:105AA000E4E771F0C5FE0022A5F87020A5F8722089
:105AB0000122A86685ED1B8A3A604CF057FB019BDA
:105AC00052460621EAE703B0BDEC028BBDE8F08F39
:105AD0007826002070860B0800000000AE860B08B8
:105AE00087860B082DE9F0432DED028B85B0044627
:105AF0000D46B0EE408AFFF745FF98B304EBC1199D
:105B0000CF01D9F868306BB371F092FED9F86830E4
:105B1000C01AB0F57A7F03D3B9F872300F2B0CD8C6
:105B2000E31993F86520002A40F08C803C44B4F8D7
:105B300072300133A4F8723014E0B9F8703005F116
:105B4000010805F1100693B94CF010FB04EB860632
:105B50004346454A042145F059FC032373603C4405
:105B60000023A36605B0BDEC028BBDE8F08307EE11
:105B7000903AD9ED1B6AD4F85C21F8EEE77A86EE0C
:105B8000A77A8DED037ACAB394F90230002B35DD84
:105B900007EE903AB2F90C209FED345AF8EEE75A2E
:105BA000F7EE007AE5EE857A182101FB054506EE51
:105BB000902AF8EEE66A95ED066A67EEA67A37EE69
:105BC000467A67EEA77AB0EEC77AE6EEE67AF6EEA8
:105BD000006A67EEA67AF4EEC77AF1EE10FA0DD5F8
:105BE000B0EEC66AB5EEC06AF1EE10FA06DD4CF012
:105BF000BDFA1F4A4346042145F008FC182003A9BA
:105C000000FB084004EB860639F0FEFA02237360BD
:105C10006368DB060ED54CF0A9FA05460398F6F743
:105C200073FC144ACDE9000143460621284645F09D
:105C3000EDFB94E74CF09AFA0F4A4346062145F0F3
:105C4000E5FB8CE7B3F87220052A7FF66FAFD3ED42
:105C50001B7AB3F8702037EE880A013283ED1B0AF5
:105C6000A3F8702062E700BFD0860B080AD7233C58
:105C7000E6860B0813870B083A870B0810B590F9D6
:105C80000030002B02460C461CDD90F84D31CBB99C
:105C9000FFF778FEA8B1182101FB042292F9243005
:105CA00093B1022B0DD146204EF0AEFEDFED077A08
:105CB000B0EEC00AB4EEE70AF1EE10FA4CBF0120D4
:105CC000002010BD0020FCE71846FAE70000003471
:105CD0002DE9F8432DED028B04460E46FFF752FEE8
:105CE000E8B104EB81090DB2D9F85431BBB171F0C0
:105CF0009FFD04EBC6174FEAC6183866D9F8540161
:105D000003685B69984770B1D9F854010368394654
:105D10009B69503198473B6D87F86500FB64BDEC8B
:105D2000028BBDE8F8833146204697F86590FFF76F
:105D30003BFE182303FB064393ED068ABB6E30EE51
:105D4000488A87ED178A1BB131462046FFF7CAFE05
:105D5000B9F1000F43D0DFED447A9FED447A04EBB4
:105D6000080368EE277AD3ED166AE6EE877A1821E3
:105D700004EB080701FB0646C7ED167A96F92730B3
:105D800083B3012B53D1DFED3A8AF1EE487A05EB6C
:105D90004505B4EEE88AC7ED157A04EBC505F1EECA
:105DA00010FA95ED070A58BFF0EE687A27EE800AE0
:105DB00096F0ACFC87ED130A97ED160AB4EEE80AEC
:105DC000F1EE10FA48BFF1EE408A95ED070A28EE91
:105DD000800A96F09BFC444484ED140A9FE7F0EEA1
:105DE000487AC4E7B5EEC08A05EB4505F1EE10FA36
:105DF00087ED158A04EBC505D8BF9FED1D8A95ED8B
:105E0000070A28EE000A96F081FC04EB0803D3EDA4
:105E1000167A83ED130AF5EEC07AF1EE10FAD8BFC8
:105E2000DFED137A95ED070A27EE800AD1E7B0EE91
:105E3000C88A05EB450587ED158A04EBC50494ED8A
:105E4000070A28EE000A96F061FCD7ED167A87ED76
:105E5000130A94ED070AF0EEE77A27EE800A96F02F
:105E600055FC87ED140A5AE79A99993E3333333F2C
:105E70000000000038B50A460446FFF783FD10B362
:105E800004EBC113CD0193F8653033B104EB81030A
:105E9000D3F85431003B18BF0123182101FB024203
:105EA000D2ED067AF0EEE77AF5EEC07AF1EE10FA6E
:105EB00008DC2C4494F8640020B992F926000038DC
:105EC00018BF0120184038BD10B500210446FFF767
:105ED00059FD18B12046FFF7CDFF50B101212046F2
:105EE000FFF750FD30B12046FFF7C4FF003818BF60
:105EF000012010BD0846FCE710B50246FFF742FD41
:105F000020B102EBC11292ED140A10BDBFEE000ADF
:105F1000FBE7000010B50246FFF734FD20B102EBAD
:105F2000C11292ED130A10BDBFEE000AFBE700009C
:105F300010B50246FFF726FD20B102EBC11292ED2B
:105F4000150A10BD9FED010AFBE700BF000000002D
:105F500010B50246FFF716FD20B102EBC11292ED1B
:105F6000170A10BD9FED010AFBE700BF000000000B
:105F70002DE9F04F2DED028B8DB0044671F060FCE1
:105F80009FED3C8ADFED3C8A8046894627462546C0
:105F90004FF0000B04F5AA7A5FFA8BF631462046E3
:105FA000FFF7F0FC002858D05AF82B30002B54D0C3
:105FB0006A462046FFF716FD08B9CDED008A1D227E
:105FC000002104A898F052FCA3238DF804309523F7
:105FD00031468DF80530204672238DF80630CDF815
:105FE0000780CDF80B908DF80F60FFF793FF2046E8
:105FF0008DED040AFFF79CFFDDED007A8DED050ABB
:1060000067EE887A2046FDEEE77A17EE903AADF813
:106010001830FFF79DFF10EE103A2046CDF81A30E9
:10602000BB69CDF81E30FFF729FE31468DF82200FE
:106030002046FFF71FFFD5F8BC300993D5F8C030D4
:106040000A9394F84E318DF823008DF82C3042F0ED
:106050008DFA292201A941F0A5FA18378035BBF144
:10606000000F04D00DB0BDEC028BBDE8F08F4FF0F7
:10607000010B91E70000C84200000000F8B590F95C
:106080000030002B04464DDD0021FFF721FE0121E9
:106090002046FFF71DFE94F90030002B0DDD94F92A
:1060A000403053B14CF062F8012105462046FFF71D
:1060B00023FF1D49284645F01FFC667894F84E7171
:1060C00031462046FFF7D6FE054668B90146204610
:1060D000FFF7D0FE28B901212046FFF7CBFE28B1FB
:1060E000012584F84E5101E084F84E61204671F09C
:1060F000F7FE94F84E31BB4204D042F037FA5A21F1
:1061000041F0CCFFD4F8503101330BD042F02EFADD
:10611000D4F8501142F050F820B12046BDE8F840C4
:10612000FFF726BFF8BD00BF54870B08014B186866
:10613000704700BF1C870020002070477047000098
:1061400001207047436AC3B1B0F850301BB9436DAA
:106150000B600120704707EE903AD0ED136AF8EE1D
:10616000E77A002386EEA77A81ED007AA0F8503016
:10617000002380ED157AC364EBE7184670470000F2
:1061800070B504463FF022FC0022222105463FF074
:1061900079FA606220B300231A461946062014F0EB
:1061A000C7FA0146204671F0F7FC0022222128465A
:1061B000666A3FF087FA0146304614F017FD94F8FE
:1061C0002020E369182101FB0233002283F82420F8
:1061D000E36994F8202003EBC213012083F86400E4
:1061E00070BD000010B5034B0360044671F0AAFCBB
:1061F000204610BD18890B0810B50446FFF7F2FFC2
:10620000204607F0E5FD204610BD000073B590F86C
:10621000455004463DB3012380F846300DF1060198
:10622000002390F828008DF806308DF8073007F02D
:1062300017FA18B90025284602B070BD94F8290055
:106240000DF1070107F00CFA0028F3D09DF8065075
:106250009DF8073043EA051394F84450DBB2EB1A7B
:106260005D425D41E7E790F83830FBB990F828309F
:10627000413B192BDFD890F82930413B192BDAD854
:1062800000F12A0617493046F7F702F910B984F8E9
:106290004850D0E714493046F7F7FAF818B9012307
:1062A00084F84830C7E784F84750C4E790F848209E
:1062B00042B9012BBFD12946283099F035FE84ED33
:1062C000100AB8E7012AB6D1072BB4D129462830E5
:1062D00099F02AFEDFED057A20EE270A84ED0F0AF9
:1062E000A9E700BF08890B080C890B08E4388E3E2B
:1062F000242970B504460D4640D016DC0A291ED06C
:106300000D291CD094F837300D2B9FBF5A1C1B1938
:1063100084F8372083F8285094F8450090B994F811
:1063200044104D4084F844500DE02A2907D02C2910
:10633000E8D190F8443083F02C0380F8443094F88E
:1063400046600EB1002070BD94F84730002BF9D0A4
:1063500094F837302344204683F82860FFF756FF2F
:1063600094F8383084F83760013384F83830A5F178
:106370002A035D425D4184F84550E4E700204FF078
:10638000807384F8380084F837006364DBE700002A
:106390002DE9F0412DED028B436A0446884623B96E
:1063A0000020BDEC028BBDE8F08171F041FA05469A
:1063B000606A9FED248A03685B699847002687B26C
:1063C0003BB2002B26DD606A03689B699847431C3B
:1063D000E6D041B22046FFF78BFF50B194F8483029
:1063E000E565012B08D1D4ED0F7A013638EE278A06
:1063F000B6B2013FBFB2E3E7D4ED137A94ED107A61
:10640000B4F8503077EE877A0133C4ED137AA4F8EC
:106410005030EEE756B9A36DC8F80030E06D281A89
:10642000B0F5FA6F2CBF00200120BAE707EE906AA2
:10643000F8EEE77A88EE277A88ED007A84ED167A0E
:10644000ECE700BF0000000010B50349044638F037
:10645000F9F8204610BD00BF38890B08F0B52DEDC6
:10646000048B91B004466D46284607F047F994F82E
:10647000BC33002B72D004F57A730FCB85E80F0084
:1064800094F8F833D4EDEC8A94EDED8A94EDEE9A1D
:10649000002B63D094F8D033002B5FD02D22002145
:1064A00004A8D4F8C073D4F8C463D4F8C853D4F89B
:1064B000CC4398F0DBF9A3238DF8103095238DF8A9
:1064C000113046238DF8123071F0BAF99FED250A8C
:1064D0009FED257ACDF8171068EE807ACDF813007D
:1064E00067EE877AFDEEE77A17EE903A68EE007A6B
:1064F00029EE000A67EE877AADF81B30FDEEE77AE9
:1065000020EE070A17EE903AADF81D3017F014FE92
:10651000DDED017A9FED157ACDF82D70BCEEC00A45
:10652000F8EEE77A10EE103A67EE877AADF81F3092
:1065300017EE903ACDF82130029BCDF82530039B21
:10654000CDF82930CDF83160CDF83550CDF839404F
:1065500042F00CF82D2204A941F024F811B0BDEC52
:10656000048BF0BDE02E65420000C8420AD7233CF0
:1065700030B52DED028B8BB0044624220D4601A8C8
:10658000002198F073F9A3238DF8043095238DF83A
:10659000053048239FED1F8A8DF8063071F050F9C1
:1065A000D4ED817A2B68CDF80F3067EE887A95EDBF
:1065B000020ACDF80B1017EE903AD4ED827ACDF89E
:1065C000133067EE887A6B68CDF8173017EE903A83
:1065D000CDF80700CDF81B3017F084FD10EE103A0F
:1065E00094ED830ACDF81F3020EE080A17F07AFDEB
:1065F00010EE103ACDF8233094F80C338DF8273094
:1066000041F0B4FF242201A940F0CCFF0BB0BDEC57
:10661000028B30BDE02E654230B587B014460D4682
:1066200018220021684698F021F9A3238DF8003044
:1066300095238DF8013049238DF8023071F000F96F
:10664000A3680393E36804936368CDF80710059388
:10665000CDF803008DF80B5041F088FF18226946F1
:1066600040F0A0FF07B030BD10B58EB0044602A8C0
:1066700007F044F802A9204601F00EFB002845D09F
:1066800001F048FD694601F09FF91F22002106A88C
:1066900098F0ECF8A3238DF8183095238DF8193075
:1066A0004A238DF81A3071F0CBF8DDED037A9FEDB7
:1066B0001B7A049BCDF82330F8EEE77A059BCDF8E2
:1066C000273067EE877ACDF81B0017EE903ADDEDA4
:1066D000007ACDF82B30F1EE677A17EE903ACDF8CC
:1066E0001F10204601A9CDF82F3000F083FC78B1AF
:1066F000DDED017AF1EE677A17EE903ACDF833309E
:1067000041F034FF1F2206A940F04CFF0EB010BD2F
:1067100041F02CFFDFED027AEEE700BF0AD7233C01
:106720005241C07F10B594B04FF07E5303A903933C
:106730000023044606930593049300F061FA17F0D2
:106740005FF890F813330C2202FB030004F5577135
:1067500000F5C4701AF070FC3322002107A88DEDFB
:10676000000ACDED010A8DED021A98F07FF8A323FF
:106770008DF81C3095238DF81D30CC238DF81E30FC
:1067800071F05EF8D4F81433CDF82730D4F818330C
:10679000CDF82B30D4F81C33CDF82F30009BCDF83A
:1067A0003330019BCDF83730029BCDF83B30039B53
:1067B000CDF83F30049BCDF84330059BCDF84730F2
:1067C000069BCDF82310CDF84B30CDF81F0041F0DB
:1067D000CDFE332207A940F0E5FE14B010BD000045
:1067E0000023036043608360C3600361436183618E
:1067F000C36103627047000090F8C432B02202FB0C
:10680000030390F8082393F8A13012B1012B28BF9D
:1068100001231846704700002DE9F04F04468BB065
:106820004FF0000A0D461EF09FFE84F814A204F5F6
:1068300006704FF07E576FF037FF4FF47A73A4F86D
:10684000623284F86852C4F84872C4F84C72C4F8D2
:10685000507204F51B70002506F050FF04F52B79EB
:106860000323C4F8803204F53476C4F89452C4F893
:106870009852C4F89C52C4F8A052C4F8A452C4F868
:10688000A8524846FFF7ACFF04F5487B3046FFF7B7
:10689000A7FFC4F81453C4F81853C4F81C5358463F
:1068A000FFF79EFFC4F84453C4F84853C4F84C5350
:1068B000C4F85053C4F85453C4F85853C4F85C5344
:1068C000C4F86053C4F86453C4F86853C4F86C53F4
:1068D000C4F87053C4F88C53C4F89053C4F894535C
:1068E000C4F8A853C4F8A453C4F8A053C4F8B053D0
:1068F000C4F8B453C4F8B853C4F8CC53C4F8C8535C
:10690000C4F8C453C4F89C73C4F8C07304F575701C
:1069100006F0F4FE04F57A7006F0F0FE04F58063EC
:10692000C4F8FC531D6004F5816304F583601D60A9
:106930005D609D6006F0E2FE04F22C4304F26448C0
:106940001D605D609D60684BC4F83C3404F50D73B8
:10695000C4F8403404F50E73C4F8443404F50F73DE
:10696000C4F8483404F51073C4F84C3404F24523D9
:10697000C4F8503404F51173C4F8543404F58B632F
:1069800040461D605D609D60FFF72AFF04F5916041
:10699000FFF726FF04F5976304F23C421D605D603B
:1069A0009D6004F2C44304F2A4501D605D609D60CC
:1069B00004F59A631D605D609D6004F2DC431D6018
:1069C0005D609D6004F2EC431D605D609D6004F2BB
:1069D000FC431D605D609D6004F5A463C2F8D47043
:1069E000C2F8D8701D605D609D6004F22C531D607C
:1069F0005D609D6004F5A9631F605D6004F26C53E7
:106A00001D605D609D6004F5AF631D605D609D600D
:106A100004F5B2631D605D609D6006F06FFE04F2D8
:106A2000B45324221D605D6004F2BC5351461D60C6
:106A30005D6004F2C45340461D605D6097F016FF30
:106A400004F2E450C8F82070C8F81070C8F800705C
:106A5000FFF7C6FE04F5C16304F5C7601D605D6005
:106A60009D6004F214631D605D609D6004F5C46365
:106A70001D605D609D6004F22C631D605D609D6023
:106A800006F03CFE194B1A491C60204637F0DAFD2F
:106A900051462422584697F0E9FEC4F84073C4F8E2
:106AA0003073C4F8207304F5257207CA04F52873FF
:106AB00083E80700484694EDAA1AD4EDA90A94ED9C
:106AC000A80A18F0B3FB3546494668466E4618F0EA
:106AD000CFFA0FCE0FC50FCE0FC533682B602046FF
:106AE0000BB0BDE8F08F00BF508C0B082087002052
:106AF0000C8B0B0810B5044688B001F095FB94F997
:106B00003232012B02D1274804F03EFD022B0AD17C
:106B1000032384F8323204A9012304F111008DF813
:106B2000103038F09DFB94F8323284F8903204F241
:106B30003C4001F02FFB94F93132642B30D16523B6
:106B400004A904F231208DF8103038F0C7FB04A9F5
:106B5000204636F079FE18B304238DF81830002350
:106B6000CDE9013303930F230593694604A836F05A
:106B7000EBFF059B28B108AA02EB8302009942F8BB
:106B8000581C0133112B0593EFD968F021FE9DEDC0
:106B9000031ADDED020A9DED010A652168F0D6FDBC
:106BA00008B010BDF8890B0870B500F5257600F522
:106BB00028758CB00446314628461AF0DDF9E0B954
:106BC00096E8070085E8070004F52B7194EDAA1AF2
:106BD000D4EDA90A94EDA80A0191084618F026FB05
:106BE00002AD019902A818F043FA0FCD04F53474F0
:106BF0000FC40FCD0FC42B6823600CB070BD000014
:106C00000B4600F54871184619F0DAB984B000F562
:106C1000487004B018F06CB913B540F2411200F599
:106C20000671044601A813F029FF04F23C4001F06C
:106C3000C1FC20461EF0F0FE01A813F041FF02B097
:106C400010BD0000F8B50B68C0F804324B68C0F8FE
:106C500008328B68C0F80C3201F10C0607460C466E
:106C600000F548750FCE0FC50FCE0FC533682B60EA
:106C700004F1300207CA07F5457383E8070004F101
:106C80003C0207CA07F5517383E8070004F1480284
:106C900007CA07F5547383E80700543494E80700E3
:106CA00007F5577383E80700384601F0D1FB3846F3
:106CB000BDE8F84001F0B4BB13B5044600F23C4017
:106CC000019003F06DF804F5BB610198009102F0AA
:106CD000C5FB0099204602B0BDE81040FFF7B2BFE7
:106CE0004A78064BC2F340121A754A78C2F38012F2
:106CF0005A750A78C2F300129A757047B58700205A
:106D000013B540F2F522044600F5067101A813F010
:106D1000B5FE002104F23C4001F0BEFE94F8603262
:106D200023B120461FF080F884F8600201A813F018
:106D3000C7FE02B010BD000038B590F80C33054610
:106D40000C462BB1032B0BD095F86832DB070CD423
:106D500005F5C7630FCB84E80F0095F8480603E0FC
:106D60001EF0B0FE0028EFD038BD0020FCE7000088
:106D700000F23C4090ED350A7047000000F23C40C4
:106D800090ED360A7047000010B490F80C230C46C2
:106D90002AB1032A0AD000205DF8044B704700F5A1
:106DA000B26007C884E807000120F5E75DF8044BEE
:106DB0001EF070BE90F88403431E5842584170473D
:106DC00038B590F80C330D468BB900F23C4001F019
:106DD00063FC044610B90024204638BD01F0B0FB26
:106DE000D5ED007A27EE800A85ED000AF4E7D0EDB4
:106DF000E07AC1ED007A90F87C43002CEBD090ED66
:106E0000DE7ADFED086AB4EEE67AF1EE10FAF7EE1C
:106E1000006AB8BFB0EE667A67EE877AC1ED007A95
:106E2000DAE700BF0000003490F80C33032B01D1E7
:106E30001EF0A0BD0020704710B490F80C43032C46
:106E400003D15DF8044B1EF0A1BD00205DF8044B9A
:106E50007047000090F80C23032A01D11EF0DCBE1D
:106E600000F23C4002F07AB830B590F80C3385B0AF
:106E700004460D468BB1032B18D004F525701AF08B
:106E8000B5F8284601A98DED010ACDED020A8DED78
:106E9000031A19F04BFC012006E000F23C4001F01F
:106EA000A5FB0028E9D1002005B030BD90F8603284
:106EB000002BF8D01EF098FEDFE700007FB590F8B9
:106EC0000C2332B1032A4FF0000309D0039304933B
:106ED0000CE000F23C4007B05DF804EB01F060BC50
:106EE00003A90393049305931EF03AFD9DED030A55
:106EF000DDED040A07B05DF804FB000007B590F86B
:106F00000C3333B100F57F7003B05DF804EB19F07A
:106F1000B9BD00F23C4001F043FC68468DED000A2B
:106F2000CDED010A19F0AEFD03B05DF804FB0000E1
:106F300090F80C03003818BF0120704708B590F88E
:106F40000C23032A05D0BDE8084000F23C4001F0C4
:106F500011BC1EF005FD012008BD000010B590F821
:106F60000C230C461AB1032A07D0002010BDBDE83F
:106F7000104000F23C4001F0A1BB1EF017FD0120C3
:106F800084ED000AF2E7000030B590F80C3385B0CC
:106F900005460C4623B1032B09D0002005B030BDB7
:106FA00000F23C4005B0BDE8304002F087BA002353
:106FB00002A9029303931EF0BBFC0028EDD001A9A7
:106FC00028461EF0C1FC0028E7D0029B2360039BEB
:106FD0006360019BA360E1E790F80C231AB1032AD8
:106FE00005D00020704700F23C4002F09BBA1EF032
:106FF0009FBC000090F80C231AB1032A05D0002092
:10700000704700F23C4002F07FBA1EF09DBC0000C9
:1070100090F932323BB990F8683213F0010F14BF87
:10702000032000207047032070470000F7B5044696
:10703000FFF7EEFF0546002862D0032839D194F807
:1070400060326BB394F86832D8072BD501A920467B
:107050001FF014F8BDF80430002B18BF002594F879
:10706000146206F0FD06012E4AD10023032D019380
:1070700007D101A920461FF00DF820461EF0E4FDBF
:10708000064604F23C4002F0CBFA08B994F8090332
:107090009DF80430D90703D55A0701D59F0632D48D
:1070A00000252DE020461EF0B3FB002808BF002578
:1070B000D5E70025D3E713F0020F2EE094F9443210
:1070C00023B99DF80430DB092FD0E9E7002EF8D072
:1070D0000FF0BEFFFFF790FB022807D99DF805309F
:1070E0009806DDD59DF80430D906D9D5FB6A93F80A
:1070F0009C30002BE5D118E0DA0601D41B0718D527
:10710000284603B0F0BD0028FAD094F80923B4F95A
:107110004C36002ACFD013F0010FF1D1154B1F6868
:10712000FB6A93F89C30002BC8D19DF804309C0773
:10713000E2D407F0CDFB07F0C9FA0028B0D10FF078
:1071400087FFFFF759FB0228AAD90FF081FF90F8BB
:10715000C432B02202FB030090ED2F7AF0EE007AE9
:10716000B4EEE77AF1EE10FA9AD59DF80530DB0916
:10717000C6D195E7782600202DE9F04790F86032D7
:1071800092B00446002B00F0948020461FF0C6F811
:107190002046FFF74BFF03287BD104F548780027F2
:1071A000414620460097019702971EF0F3FC69467E
:1071B00020461EF0E5FC009BC4F80432019BC4F895
:1071C0000832029BC4F80C32204601F041F92046F7
:1071D00001F026F916F014FB054620461EF09AFB36
:1071E0000028A8BFC6B203AA4FF0FF312046BCBF9B
:1071F00095F8129395F813630397A8BFB1460497C7
:1072000005971EF0E1FB03A819F0F0FE4FF00C0A01
:107210000AFB095084EDD10AC4EDD20A84EDD31AD9
:1072200004F5517100F5117019F0F0FE04F557776F
:107230000AFB065584EDC50AC4EDC60A84EDC71ADB
:107240003A464FF0FF31204605F5C4751EF0D0FBDD
:1072500095E8070006AE86E807003946304619F083
:107260003BFF04F52B72414609A817F091FE314609
:1072700009A817F00FFE09A9204684EDD40AC4ED31
:10728000D50A84EDD61A1EF005FF09A92046FFF79E
:1072900027FD94F84E36002B3AD109A806F02EFAB5
:1072A00009A920461EF01AFC90B3012384F84E363B
:1072B0002EE0D0F864321BB970F0BAFAC4F8640258
:1072C000154B1B68D86A03685B68984788B170F0F3
:1072D000AFFAD4F86432C01AB4F86232984204D9D2
:1072E00020461EF0A1FD84F8600294F860327BB164
:1072F0004BE770F09DFAD4F86432C01A41F287333C
:107300009842E4D841F032F940F072FF0028DED113
:1073100012B0BDE8F08700BF7826002090F80C334B
:1073200023B1032B4FF0000007D0704790F93222B1
:10733000032A04D10A70012070470870FBE7184641
:107340007047000073B50D460DF107010446FFF7C5
:10735000E5FF064628B19DF807302BB1032B09D075
:107360000026304602B070BD04F5C7630FCB85E838
:107370000F00F6E7294620461EF0A4FB94F8606251
:10738000EFE700007FB50E460DF103010446FFF75D
:10739000C5FF054618B90025284604B070BD9DF804
:1073A000033083B1032B16D004F5257019F01EFEAF
:1073B00001A930468DED010ACDED020A8DED031ACB
:1073C00019F0B4F9E8E7314604F23C4001F00EF957
:1073D0000028E9D1DFE794F86032002BDBD031469A
:1073E00020461EF001FCDFE737B50D460DF1070121
:1073F0000446FFF793FF28B19DF8073023B1032B14
:107400000FD0002003B030BD04F5BB631B682B60B8
:1074100004F2DC5304F5BC641B686B602368AB604A
:10742000F0E7204629461EF0ABFB94F86002E9E73E
:1074300010B50446FFF7ECFD18B1032807D0002073
:1074400010BD04F23C40BDE8104001F0F9B894F8DA
:107450006032002BF3D020461EF0DAF90028EED07F
:1074600094F8143203F0FD03012BE9D194F80C03D6
:10747000C31E58425841E3E710B50446FFF7C8FD64
:1074800080B1032810D194F8600250B170F0D0F9A7
:10749000D4F86432C01A44F62063984294BF0020A6
:1074A000012010BD0120FCE70020FAE708B50246E4
:1074B000FFF7AEFD032804D110461EF0EBFD0120BE
:1074C00008BD0020FCE7000030B585B004460191FE
:1074D000FEF72CFE0199054610B9002005B030BD1D
:1074E0000191FEF7CBFB01990028F6D02846FEF764
:1074F000C1FC0028F1D0B4F84C365907EED494F80A
:107500000933002BEAD00B4A1268D26A92F89C50D9
:107510006DB103A92046FFF7C9FF30B19DF80E30C9
:107520009A07DBD5C3F38000D8E72846D6E718468C
:10753000D4E700BF782600202DE9F04190F80C3305
:107540008CB00027032B06460C4615460097019782
:10755000029719D11EF0DEF96A4680464FF0FF31DE
:1075600030461EF045FAB8F1FF3FA760676027601C
:107570000DD116F045F92B4690F81313224615F05D
:10758000B3F90CB0BDE8F0814FF0FF38EBE716F02F
:1075900037F92B4622465FFA88F115F0A5F995EDEB
:1075A000000A684619F05EFD03A920468DED051A14
:1075B0008DED030ACDED040A19F08EFD06F52B7250
:1075C00006F5487103A817F0E3FC214603A817F05D
:1075D00061FC84ED021A84ED000AC4ED010A95ED08
:1075E000007ADFED037AA7EE271A84ED021AC8E7C6
:1075F0000AE81C411FB5DFED0B7A20EE270A0C4686
:107600001946094BCDE90042BDEEC00A18688DED60
:10761000020A064B9DF81820C06A13F00FFC04B054
:1076200010BD00BFE02E6542782600200C8A0B08B2
:107630002DE9F0472DED028B92B0002504460F4650
:107640004FF07E5A00F5487106A89046CDF818A074
:1076500009950895079518F0B3FC07F039F907F07C
:1076600035F881462046FFF7D3FC032803D094F871
:107670000C33032B4FD19FED558ADFED558A002641
:107680002379F2B2934247D90AAA71B22046CDF8C3
:1076900028A00D950C950B951EF086FA0AA906A850
:1076A00019F0B6F8B4EEC80AF1EE10FA0DDD494A49
:1076B000CDF800803B4648492046FFF79BFF00205D
:1076C00012B0BDEC028BBDE8F0870AA906A80395AD
:1076D0000495059519F086F803A90EA88DED0E0AFC
:1076E000CDED0F0A8DED101ACDED111A18F0EEFD4B
:1076F000B9F1000F0DD09DED050AB0EEC00AB4EE51
:10770000E80AF1EE10FA04DD344ACDF800803B4679
:10771000D1E70136B4E7002394F8686216F001005F
:1077200001D0012BCCD104F2E4510AA8CDF828A055
:107730000D950C950B9518F043FC0AA906A819F0B5
:1077400067F8DFED227AB4EEE70AF1EE10FA05DD14
:10775000204ACDF800803B462149ADE72046FFF79F
:1077600057FC03282DD120461EF062FA94F86832A7
:10777000DB0728D438BB0AA906A80395049505950C
:1077800019F030F803A90EA88DED0E0ACDED0F0A01
:107790008DED101ACDED111A18F098FDB9F1000F0A
:1077A00011D09DED050ADFED0A7AB0EEC00AB4EE05
:1077B000E70AF1EE10FA06DD084ACDF800803B46F4
:1077C000CAE70020D2E701207AE700BFC2B8323E04
:1077D000C2B8B23E388A0B08438A0B0822DF0B0876
:1077E000488A0B082DE9F74314460546884601935D
:1077F000FFF71EFE019A074638B92448244B00685B
:107800002146C06A13F01AFB019A019221462846CC
:10781000FFF70EFF064630B32846FFF7F9FB95F851
:107820000C33019A83420DD007F052F806F04EFF58
:10783000019A38B1174B154800682146C06A13F009
:10784000FDFA10E02846FFF7E3FB18B103280FD03C
:10785000114BF0E713464146224605F23C4000F04A
:1078600003FF00B107B90026304603B0BDE8F0833E
:1078700095F86092B9F1000F01D1084BDBE7134690
:107880004146224628461DF0D3FFEAE7782600202D
:107890004C8A0B08588A0B08888A0B08778A0B08D1
:1078A00090F80C33032B01D11EF00ABC0020704766
:1078B00037B5054600F5067140F6033201A813F00E
:1078C000DDF82846FFF7A4FB044640B103280AD0A0
:1078D000002401A813F0F4F8204603B030BD284678
:1078E0001EF0B4F8F5E728461EF0B0F80446F0E7BD
:1078F00008B50246FFF78CFB10B1032806D008BD7F
:10790000BDE8084002F23C4000F064BEBDE808401B
:1079100010461EF0CBBB00000B4610B411462BB135
:10792000032B09D000205DF8044B70475DF8044B31
:1079300000F23C4000F064BE5DF8044B1EF0CEB88F
:1079400013B50446FFF764FB0A4601462046019240
:10795000FFF7E2FF70B9084B019A1B68DB6A93F8E6
:107960009C0038B194F80C13204602B0BDE81040DA
:10797000FFF7D2BF02B010BD7826002037B504460D
:107980000D4640F2B25200F5067101A813F076F8E8
:10799000294620461EF0C0F894F80C33032B054608
:1079A00010D148B104F583612046FFF7C9FF84F880
:1079B0002804204600F0A4FD01A813F081F8284611
:1079C00003B030BD0025F7E770B590F87C32DB07D7
:1079D00086B004460D460CD402F096FF437C242268
:1079E00002FB0300D0ED0B7AF1EE677AC5ED007A69
:1079F0003BE002A805F082FE01A92046FFF7FAFA53
:107A0000E8B90FF025FB94F94432022B0646E3D186
:107A1000FEF7F2FE0228DFD996F8C4029FED147A31
:107A2000B02303FB0066D4F87032D6F8B0209B1A5E
:107A300007EE903AF8EEE77A67EE877AD6E702A982
:107A40002046FFF77DFF0028DBD0D4F87022039B8F
:107A5000DFED076A9DED017A9B1A07EE903AF8EE8A
:107A6000E77AA7EEE67A85ED007A06B070BD00BF32
:107A70000AD7233CF0B50C4687B000F506710646E0
:107A800040F6863201A812F0F9FFA36853B9E36803
:107A900043B9636833B9002701A813F011F83846D9
:107AA00007B0F0BD204605F031FF0028F3D094E880
:107AB0000F0002AD85E80F000021284605F0E8FE22
:107AC00007460028E7D096F87C32DB0704D440F064
:107AD0004DFD192140F0E2FA95E80F0006F51B7CF8
:107AE0008CE80F0096F87C3243F0010386F87C3274
:107AF000304600F005FD4AF039FB46214AF030FFE0
:107B00004AF034FB45214AF02BFF054BA2681B6865
:107B1000DB6A1A61E2685A6162689A61BCE700BF79
:107B20007826002038B5144B1B68DD6A2B680446A4
:107B30005B6828469847F0B12B690BB96A69D2B1E6
:107B4000C4F874326B69C4F87832A969002204F56C
:107B50001B7005F0D9FD94F87C3223F0030343F049
:107B6000030384F87C324AF001FBBDE83840034A45
:107B7000062143F04BBC38BD782600209C8A0B08B8
:107B800010B588B004460593FFF742FA0328059B19
:107B90004FF000000AD10690079006A802900B98BB
:107BA00001900A98009020461EF028F808B010BDF9
:107BB00038B50446FEF7BAFA0546D0B194F80C334E
:107BC000032B03D095F84E41204638BD20461DF0CA
:107BD0006DFFFF280446F5D001462846FEF74AF916
:107BE0000028EFD021462846FEF748F80028E9D0C3
:107BF000EAE70446E8E7000008B590F80C33032BE9
:107C000005D015F0FDFD90F91203C0B208BD1DF0BE
:107C100081FE431CF9D1F4E708B590F80C3383B129
:107C2000032B03D1BDE808401DF06CBE3EF068FE9A
:107C300040F6ED424FF480113EF01AFE4FF0FF3057
:107C400008BD1846FCE7000090F80C33032B01D167
:107C50001EF0B0BC7047000090F80C33032B01D12C
:107C60001DF034BD704700001DF0BABD10B50446CC
:107C700020F06CFD2046FEF7F1FB2046BDE81040E9
:107C8000FEF7F2BC90F80C330BB1032B01D11EF0C0
:107C90000DBD00207047000030B500F57573044637
:107CA0000D460FCB85E80F0094F8E40330BD0000CB
:107CB0007FB5054668460E4605F020FD95F87C32F6
:107CC000DB0703D40024204604B070BD6946284673
:107CD000FFF7E2FF04460028F4D0694605F51B7063
:107CE00005F024FF86ED000AC6ED010AEBE700006F
:107CF000D0F880330B6090F87C037047D0F888335D
:107D00000B6090F88503704730B500F56773044643
:107D10000D460FCB85E80F0094F8AC0330BD000092
:107D200030B500F5836304460D460FCB85E80F00A0
:107D300094F8280430BD000010B500F22C42034630
:107D40000C4607CA84E8070093F8380410BD000009
:107D50002DE9F0432DED028B8BB005460E461746FC
:107D6000FFF726FF014680462846FFF7ADFB044695
:107D7000002848D0FEF7DAF94146FEF7BDF886ED57
:107D8000000A95F93032002B3ADD0FF061F9FEF769
:107D900033FD012834D90FF05BF990F8C432D5EDEA
:107DA000DE7ADFED5D8A96ED000AB02202FB030069
:107DB00095F93032D0ED2F0A07EE103AF4EEE87A5A
:107DC000B8EEC77AF1EE10FAB7EE008AB8BFF0EE5F
:107DD000487A37EE201A20EE270A70EEC70A40F2E2
:107DE000B63016F015FAD5EDDE7AF4EEE87AF1EE5B
:107DF00010FAB8BFF0EE487A80EE277A86ED007A66
:107E000001233B7003E095F8083333B938702046FE
:107E10000BB0BDEC028BBDE8F08395F80C334FF04E
:107E20000009CDF80490CDF80890CDF80C9043B13E
:107E3000032B10D0CDF81090CDF81490CDF81890F9
:107E40007CB902233B703246414605F23C4001F0CA
:107E5000ABFB0446DBE701A928461DF01BFE0446E8
:107E6000E8E795F80C33002BEBD004A92846FFF780
:107E700063FF04460028E4D001A904A819F0DCF847
:107E800007A8CDED080A8DED091A8DED070A19F046
:107E9000E7FC04A8B0EE408A19F0E2FC95F9303214
:107EA000002B30DD07EE903AF8EEE77A4FF47F7062
:107EB00070EE670A37EE801AF5EEC00AF1EE10FA9E
:107EC00048BFDFED160AF4EE410AF1EE10FAB0EE0B
:107ED000480AC8BFB0EE601A16F09AF9B0EE408AB0
:107EE000D5EDDE7A9FED0C7AF4EEC77AF1EE10FA5A
:107EF000B7EE007AB8BFF0EE477A88EE277A032310
:107F000086ED007A7DE7B5EEC08AF1EE10FA48BF43
:107F10009FED028AE4E700BF00000034000000008B
:107F200010B50446FFF768FE84F80D032046FFF7FE
:107F300063FE84F80E032046FFF75EFE84F80F030D
:107F40002046FFF769FE04F55A7184F810032046B5
:107F5000FEF71AFF84F8740300F0F2FA04F5617278
:107F600084EDDE0A04F560712046FFF7F1FE04F5AA
:107F7000627184F87C032046FEF722FF04F56371EA
:107F800084F885032046FEF74FFF04F5677184F8F7
:107F900098032046FEF768FF04F56C7184F8AC0383
:107FA0002046FFF721FA04F5707184F8BC032046DF
:107FB000FFF7E8F904F5757184F8D0032046FEF761
:107FC000BBFE04F57A7184F8E4032046FFF7BAF9A2
:107FD00084F8F8032046FEF771FF04F5806384ED12
:107FE000FF0A2046C3ED000AFEF788FF04F20443AF
:107FF00083ED000A04F2144204F581612046FFF784
:108000009BFA04F583612046FFF79AFC04F22C41A9
:1080100084F828042046FEF791FF84F8380410BD48
:1080200037B50D46044600F0FFF81DB915F0E8FB22
:1080300014F08AFB4FF4BE7204F5067101A812F029
:108040001DFD94F869322BB92046FFF76BFD012323
:1080500084F86932224B1D68A86A03689B699847B7
:108060002046FEF7A1FD2046FEF726FE204600F042
:1080700079FA2046FFF780F8286B30B10368D4ED19
:10808000D20ADB6894EDD10A9847D4F8100208B1FF
:1080900071F030FF204600F07DF82046FEF7C6FF65
:1080A00094F8903284F80C0383420ED084F8900246
:1080B00098B10C4D0C4B032808BF1D464AF056F8EA
:1080C0000A4A2B46062143F0A1F92046FFF728FF74
:1080D00001A812F0F5FC03B030BD054DEEE700BF7E
:1080E0007826002076420B08438A0B08B48A0B08D6
:1080F000488A0B08D0EDDE7A9FED057AF4EEC77A58
:10810000F1EE10FAB7EE000AA8BFB0EE670A7047AA
:1081100000000034014B1868704700BF2087002022
:108120004FF0FF307047000001207047704700009B
:108130000020704700207047704700007047000023
:1081400000207047002070470020704700207047D3
:1081500000207047002070470020704701207047C2
:108160000368D3F894301847002070470020704708
:1081700000207047002070470020704700207047A3
:108180000020704700207047002070470020704793
:10819000704700007047000008B515F031FB90F8FB
:1081A000130308BD08B515F02BFB90F8120308BDAA
:1081B00030B52DED028B9FED1A1ADFED1A0A91ED05
:1081C000000A87B005462D200C468DED011ACDED35
:1081D000000A16F01DF89DED011ADDED000AF0EE23
:1081E000408A2E2094ED010A16F012F89DED011A36
:1081F000DDED000AB0EE408A2F2094ED020A16F061
:1082000007F803A905F52570CDED038A8DED048AE5
:108210008DED050A37F046F907B0BDEC028B30BD95
:10822000C2B8323EC2B832BE10B504466FF000FB91
:10823000D4F8F4321BB1C21AB2F57A7F12D30A4ACB
:108240001268D26A92F89C2002B15BB9C4F8F402B9
:1082500094F8314215F0D4FA80F80D4306F038FB5B
:1082600080F8254010BD00BF782600202DE9F0439E
:108270002DED028B91ED007AD1ED037A87B08DED73
:10828000047AB0EEC77AB5EEC07AF1EE10FADDE905
:108290001087DDF84C90CDED057A0C4615461E464C
:1082A00006DCF0EEE77AF5EEC07AF1EE10FA02DDC8
:1082B00004A818F065FC6B20B7EE001AFFEE000A68
:1082C0009DED050A15F0A4FF6C2089ED000AB7EEBC
:1082D000001AFFEE000A9DED040A15F099FF04A8AC
:1082E00088ED000A18F0A8FBB7EE008A002852D0EB
:1082F0000023C9F8003088ED008AD4ED067A67EED5
:10830000A77AF4EEC87AF1EE10FA4ADB0023336064
:1083100085ED008ADFED3F0A96ED000A7C20B7EE7E
:10832000001A15F075FF86ED000A95ED000A7D2014
:10833000B7EE001AFFEE000A15F06AFF85ED000A9D
:10834000D4ED067A129BDFED346AF1EE677AC3ED65
:10835000007A96ED007AF0EEC77AF4EEE67AF1EE66
:1083600010FA2BD503AB02AA01A9204616F0BEFFD6
:108370009DED018AB0EE480A93F05CFE85ED000A9F
:10838000B0EE480A93F0ACFF87ED000A07B0BDECF1
:10839000028BBDE8F08304A818F03AFB0028A7D1AF
:1083A000ABE738EE670A15F063FE86ED000A94ED40
:1083B000087AC7EE007AC5ED007AABE794ED076A5C
:1083C000C6EE077AC7ED007A96ED007AB0EEC77A6E
:1083D000B4EEE67AF1EE10FAC4D495ED007ADFED52
:1083E0000F6AB0EEC76AB4EE666AF1EE10FAB9DC55
:1083F000B4EE477AF1EE10FAB4D6B0EEE77AB4EE06
:10840000667AF1EE10FAADDCF4EE677AF1EE10FA6E
:10841000BCD7A7E70000000000000034FFFF7F7F0B
:108420001FB500F51773039300F51673029300F55B
:108430001573019300F51473009300F5127200F5A3
:10844000137300F54871FFF711FF05B05DF804FBE9
:108450009FED156A90ED817ADFED146AD0ED837A95
:1084600027EE067A67EE867A27EE267A67EEA67AF8
:10847000BDEEC77AFDEEE77A80ED7E7A90ED827AE6
:1084800027EE067A17EE903A27EE267A002BB8BF31
:1084900003F50C43BDEEC77AB8BFA03380ED7F7AF9
:1084A000C0F80032704700BFE02E65420000C842AD
:1084B000D0ED946AD1ED010AD0ED977A91ED007A72
:1084C00020EEA70A66EEA00AA7EE260A84B0E7EE21
:1084D000670A04B070470000D0ED946AD1ED010A3C
:1084E000D0ED977A91ED007A27EEE00A66EEA00AC9
:1084F000A7EE260A84B0E7EE270A04B07047000012
:108500001FB50E4B1B680446B3B1684605F0F6F87C
:1085100069462046FFF704FC20B16A460021204648
:10852000FEF77AF894F87C32DB0705D504F51B7268
:1085300001212046FEF770F804B010BDE08900204C
:1085400008B502F0E1F9BDE8084001F06FBD000098
:1085500010B580F8F81204466FF06AF9C4F8FC020E
:1085600010BD000010B590F8F832044653B16FF01A
:108570005FF9D4F8FC32C01AB0F57A7F84BF0023CB
:1085800084F8F83294F8003353B16FF051F9D4F80D
:108590000433C01AB0F57A7F84BF002384F8003317
:1085A00010BD000000F5AA700B4607C883E807005D
:1085B000012070470023C0F89C30C0F89830C0F804
:1085C0009430C0F8A830C0F8A430C0F8A030C0F88B
:1085D000AC30704770470000024B0B604FF07C538B
:1085E00013607047000048427047000008B50B4612
:1085F00000F12801184617F0E3FC012008BD000037
:1086000010B500F5B4700C460FC884E80F00204682
:1086100005F064F830B1FFF77DFD00F51B700FC861
:1086200084E80F00204605F059F880F00100C0B240
:1086300010BD000010B5044605F0CAFB204610BD71
:1086400010B5D0F8603104465BB16FF0F1F8D4F8A2
:108650006031C01A41F28833984294BF0020012053
:1086600010BD0120FCE7000013B5009303680192E0
:10867000D3F890309847DDE90021044628B9044832
:10868000044B0068C06A12F0D9FB204602B010BD4E
:10869000782600204C8A0B0813B504460191FDF79B
:1086A00045FD2368019A1B6D014608B190F84E11F3
:1086B000204602B0BDE810401847000030B585B034
:1086C000002301930293039303680D46DB6D01A918
:1086D0009847044620B1039B2B60204605B030BD6F
:1086E00002F012F9417C01F0DDFD04460028F4D0CF
:1086F00002F00AF901F03CFDB1EE400A85ED000AF6
:10870000EBE7000090ED007ADFED0F7AB0EEC77A6C
:10871000B4EEE77AF1EE10FA14D590ED017AB0EEEE
:10872000C77AB4EEE77AF1EE10FA0BD590ED027A43
:10873000B0EEC77AB4EEE77AF1EE10FA4CBF012042
:1087400000207047002070470000003410B5FDF78E
:10875000EDFC044658B190F84E11FDF78FFA30B198
:1087600094F84E112046BDE81040FDF783BB002071
:1087700010BD000038B50D460EF06AFC0446FEF749
:108780003BF8022881BF94F8C402B02303FB0040E9
:10879000D43089BF07C8002085E80700012038BD14
:1087A0002DE9F0432DED028B8FB003680025DB6CC3
:1087B0000395049505950695029502A904469847E8
:1087C000064638B1FFF7BCFEDDED027A27EE800ADF
:1087D0008DED020A0EF03CFCFEF70EF80746002E67
:1087E00050D0DDED027AD4ED646A94ED657A2368A9
:1087F0000B9527EE877A67EEA67A8DED097ACDED97
:108800000A7A0C950D959B6C0BA9204609AD9847EB
:108810000BA9284618F06AF8012F8DED030ACDED5B
:10882000040A40F2B3800EF013FC90F8C432DFED7E
:108830005B7AB02505FB030090ED308A28EE278A8D
:10884000B0EE480A93F0F6FBF0EE408AB0EE480A2C
:1088500093F046FDCDED0B8A8DED0C0A0EF0F8FB82
:1088600090F8C43205FB030090ED2F0A0BA818F016
:108870005DF809AD8DED050ACDED060A05A896BB9C
:1088800003C885E00128CED89DED020AB5EEC00AE6
:10889000F1EE10FA7FDD07AED4F89421D4F89031D0
:1088A00007923046089318F06BF823680B950C95E7
:1088B0000D959B6C0BA920469847DDED077A9DED41
:1088C0000B7A77EE877A9DED0C7ACDED077ADDEDA8
:1088D000087A77EE877A09ABCDED087A96E803003F
:1088E00083E8030049E0236993ED000AB7EE008AAC
:1088F00038EE408A18F01AF804F5BC798DED090AB3
:108900004846B0EE480ACDED0A0A18F00FF80BA958
:108910002846CDED0C0A8DED0B0A17F0E7FF04F5A4
:10892000C47603AFC4ED5F0A314684ED5E0A384673
:1089300017F0ECFF04F5C0788DED090A4046B0EE63
:10894000480ACDED0A0A17F0F1FF0BA928468DED74
:108950000B0ACDED0C0A17F0C9FF97E8030084ED70
:10896000600AC4ED610A86E803004946404617F0F4
:10897000BDFF8DED090ACDED0A0A9DED090ADDED79
:108980000A0A0FB0BDEC028BBDE8F083DDE90301FC
:1089900085E80300F1E709950A95EEE735FA8E3C84
:1089A00010B590F84213044605F0ACFB7C23C0B22E
:1089B00003FB0044D4F8A00010BD0000044B026F7C
:1089C0001B68DB6A5A60426F9A60826FDA60704798
:1089D00078260020F0B58FB0044614F011FF002374
:1089E00002930393049390F8121301AB02AA054675
:1089F00013F020FF04F19407D8B39DED010AB5EE02
:108A0000C00AF1EE10FA34DD02A818F03BFB04F1C5
:108A1000B00684ED2C0AC4ED2D0A84ED2E1A3946D9
:108A2000304618F03FFB04F17C01304618F0EEFAB6
:108A300004F1880105A88DED050ACDED060A8DED3E
:108A4000071A18F0E3FA08A88DED080A9DED010A4F
:108A5000CDED090A8DED0A1A18F004FB0BA904F1FB
:108A600028008DED0B0ACDED0C0A8DED0D1A16F0D8
:108A7000E9FC95F812030C2303FB0050394600F57E
:108A8000117018F0C3FA84ED2C0AC4ED2D0A84EDA0
:108A90002E1A0FB0F0BD00002DE9F047824B0025E3
:108AA0001F682DED028BC0F89C50C0F89850C0F89C
:108AB0009450C0F88450C0F88050C567C0F89050FA
:108AC000C0F88C50C0F88850C0F8B850C0F8B45006
:108AD000C0F8B0500446F86A03688AB05B680E4676
:108AE000984704F12809002854D06EF0A1FE42F204
:108AF0000F7398424ED8FB6A9FED6C8A93ED010A82
:108B000084ED1C0AD3ED020AC4ED1D0A93ED031A8D
:108B1000484684ED1E1A16F089FB49F027FBD4ED78
:108B20001E7A67EE887A054617EE900AF3F7ECFC9A
:108B3000D4ED1D7A67EE887ACDE9040117EE900A2C
:108B4000F3F7E2FCD4ED1C7A67EE887ACDE90201F6
:108B500017EE900AF3F7D8FC554ACDE9000106213B
:108B6000284642F053FC94ED1E8AB0EE480A93F07A
:108B700061FA84ED650AB0EE480A93F0B1FB84ED2A
:108B8000640A6EF055FEC4F864010AB0BDEC028BB5
:108B9000BDE8F087A6B194ED1C0AB4EE400AF1EEF0
:108BA00010FA0DD6D4ED1D0AF4EE600AF1EE10FABB
:108BB00006D694ED1E1AB4EE411AF1EE10FA52D711
:108BC00014F01EFE90F813334FF00C0A0AFB030357
:108BD00003F5C473074693E8070007AE86E807006D
:108BE0004FF01508B2EE028AF2EE068A304618F00F
:108BF00037FEB4EEC80AF1EE10FA38D508F1FF38A6
:108C000018F0FF083CD1304618F02AFEF1EE047A45
:108C1000B4EEE70AF1EE10FA43DD9DED090ADDED51
:108C2000087A9DED078A20EE000AA7EEA70A93F0C6
:108C30006DFDF0EE400AB0EE480A93F01DFCDDED4C
:108C4000090A84ED1D0A9DED080AF1EE600AB1EEF5
:108C5000400A93F011FC84ED1C0A9FED161AD4ED26
:108C60001D0A94ED1C0A484616F0E0FA7BE73046F0
:108C700018F0F6FDB4EEE80AF1EE10FABEDCC2E739
:108C8000384613F099FC384613F05EFD97F813331D
:108C90000AFB037303F5C47393E8070086E8070033
:108CA000A4E725676567D8E778260020E02E6542AF
:108CB000CC8B0B08000000000021FFF7EDBE000088
:108CC00037B5044608461546019118F0C9FDB7EEC0
:108CD000007AC7EE007AB4F8D03001980133A4F8D6
:108CE000D03094ED337A37EE277A84ED337AB0EED4
:108CF000007AF4EEC77AF1EE10FA06D5B6EE007AF5
:108D0000F4EEC77AF1EE10FA0DDC9FED0E7AF4EE78
:108D1000C77AF1EE10FA13D59FED0B7AF4EEC77A0D
:108D2000F1EE10FA0CDDB0EE670A18F09BF90120A5
:108D300085ED000AC5ED010A85ED021A03B030BDCC
:108D40000020FBE700247449BD37863570B52DED52
:108D5000028B00F1280600F134058AB0294604464A
:108D6000304618F0FBF9B6EE008A20EE088A284655
:108D7000B0EE480A18F076F907A93046CDED080A9A
:108D80008DED091A8DED070A18F056F930468DED74
:108D9000010AB0EE480ACDED020A8DED031A18F073
:108DA00061F907A928468DED070ACDED080A8DED7A
:108DB000091A18F041F904A901A88DED040ACDEDB6
:108DC000050A8DED061A18F0DDF9324601A9204694
:108DD0008DED070ACDED080A8DED091AFFF770FF3A
:108DE00058B96EF025FD0121C4F860012046FFF757
:108DF00053FE0AB0BDEC028B70BD2A4604A9204682
:108E0000FFF75EFF0028ECD004F1400207A92046DE
:108E1000FFF756FF0028E4D0EBE7000030B52DED5A
:108E2000028B0D4683B091F842130446284605F0A4
:108E300069F9C1B27C2000FB0151903104F1280096
:108E400016F084F868468DED000ACDED010A17F0A2
:108E500019FEDFED1C7AB4EEE70AF1EE10FA05D543
:108E60009FED190A03B0BDEC028B30BD684617F0C8
:108E700087FE684617F0E0FD0028F1D1284694ED02
:108E8000428A05F0B3FAF0EE400AB0EE480A15F057
:108E9000BBF880B9284605F0A9FA84ED420AB0EE85
:108EA000408A93F0C7F884ED430AB0EE480A93F085
:108EB00017FA84ED440A04F58671684617F08AFDB6
:108EC000D0E700BF00000034000000009FED0C7AE6
:108ED000B4EEC70AF1EE10FA0BD4DFED0A7AB4EE65
:108EE000E70AF1EE10FA07DCC0EE077AB0EE670A87
:108EF0007047F7EE007AF9E7F2EE047AF6E700BF82
:108F0000F3665F3F58A00B4108B51C3017F0BAFD5F
:108F1000F1EE007AB4EEE70AF1EE10FA9DBFF1EE41
:108F2000027A37EEC00ADFED047A9FED040A98BF9B
:108F300020EE270A08BD00BFCDCC4C3ECDCCCC3DA9
:108F400008B5836993F9000038B10EF081F8FDF798
:108F500053FC012894BF0020012008BDF8B52DED79
:108F6000028B054605F0B4FC05F0B0FB0446B8B32F
:108F7000FFF7D0F890F8093393B32846FFF7E0FFE6
:108F8000064668B30EF064F890F8C432B02707FBC9
:108F9000030090ED2F7AF0EE087AB4EEE77AF1EE66
:108FA00010FA1DD495ED1E8A0EF052F890F8C432D6
:108FB000DFED1E7A07FB030090ED300A98EE270ADA
:108FC00015F0A6F8DFED1A7AB0EEC00AB4EEE70AA3
:108FD000F1EE10FA08DC6EF02BFC3446C5F85001B7
:108FE000BDEC028B2046F8BD05F5AA7018F038FCE0
:108FF000B0EE408A0EF02CF890F8C4329FED0D7A56
:1090000007FB0303D3ED2F7A67EE877AB4EEE78A86
:10901000F1EE10FADFD56EF00BFCD5F85041001BD5
:10902000B0F5FA6F8CBF00240124D9E7E02E654229
:1090300000003442CDCC4C3F10B50A4B1B68DB6AB4
:1090400093F89C3004465BB96EF0F2FBD4F86431BF
:10905000C01A44F61F6398428CBF0020012010BD47
:109060000020FCE778260020F8B52DED068B04469D
:109070000DF0EEFF054605F02BFC064608F014F94E
:10908000002840F0AA802046FFF768FF002800F083
:10909000A7803046FFF784FCD4F8DC30984200F01B
:1090A00018813046FFF77CFCD4F8DC30DFED8E7A97
:1090B000C31A08EE903AF8EE688A304668EEA78A3E
:1090C000FFF76EFC94F8BC30C4F8DC00F3B930460E
:1090D00005F00EFBD0B104F1280796F8422339467B
:1090E000304605F087F9D4ED1D0AB0EE401A384637
:1090F00094ED1C0A16F09AF80023C4F89030C4F8D6
:109100008C30C4F88830012384F8BC3020463146C6
:10911000FFF784FE95F8C40205EB0015B0EE408A17
:109120002B6FC4F8E03004F1B000D4ED129A18F0BF
:1091300097FB6368DFED6D7A93ED007AB4EEE77A22
:10914000F1EE10FA68EE299AB0EE40AA01D5C3ED0F
:10915000007A2046B0EE4A0AFFF7B8FE636820EEB8
:10916000299A93ED000A29EE009AFFF7CDFE29EE29
:10917000009A204684ED249AFFF75EFF38B1D4EDC3
:10918000247AB2EE007A67EE877AC4ED247AF0EEA4
:10919000007AF4EEE78AF1EE10FA10D5DFED547A9A
:1091A000B4EEE7AAF1EE10FA09D5DFED527A69EED6
:1091B000A79AD4ED2A7AE9EEA87AC4ED2A7A9FED2F
:1091C0004E0A94ED367ADFED4D7AB0EEC88A28EE7D
:1091D000008AA7EE278A84ED368ABDEC068BF8BD9F
:1091E000FEF798FF90F80933002B72D02046FFF766
:1091F000A7FE00286DD095F8C42205EB0213196F65
:10920000D4F8E0308B4264D0B02606FB025292EDD7
:109210002F7AF0EE087AB4EEE77AF1EE10FA58DB26
:10922000CB1AC4F8E01008EE903A95F8C4329FEDDE
:10923000341A94ED1E0ADFED337A06FB0353D3EDA7
:10924000309A69EE819AF8EE688A39EEC00A68EEC3
:10925000A78A14F0C9FFB0EE409A93F041F894F851
:10926000BC30B0EE408AF3B1F3EE047AF4EEE78A54
:10927000F1EE10FA17DC95F8C40206FB005595EDE7
:109280002F7AF2EE027AB4EEE77AF1EE10FAFFF6F8
:109290004AAFDFED1D7AB0EEC99AB4EEE79AF1EE6F
:1092A00010FAFFF640AF9FED198AD4ED1D0A94ED38
:1092B0001C0AB0EE691A04F1280015F0B7FF01236B
:1092C00084ED248A84ED238A84ED228A84F8BC30DC
:1092D00029E7BDEC068B04F188009FED0D0ABDE87F
:1092E000F84017F013BF00BFBD378635CDCC4C3DDD
:1092F000C2B8B23E0AD7233CCDCC4C3ECDCC4C3F7D
:1093000035FA8E3C6F12833A1904863F0000000044
:10931000EC51783F30B50C2303FB010101F1C00390
:10932000144693E807008BB004AD85E8070094E885
:10933000070083E807002846FFF7E4F907AB58B1B8
:1093400094E8070083E807009DED070ADDED080AB1
:109350009DED091A0BB030BD95E80700F2E700005B
:10936000F0B52DED028BD0F818318B60D0F81C31A0
:10937000CB6085B004460D4601F0C6FA06460DF0F6
:1093800067FEA36993F90030022B07464BD1FDF726
:1093900033FA022847D997F8C432B02202FB03738C
:1093A000D3F8B0100022284604F0AEF9D4ED4A0AF2
:1093B00094ED490A284604F0D3FC94F82C3163B3A9
:1093C0006EF036FA9FED228A97F8C4128DED018A6D
:1093D00001AA064638460CF0BFFED4F820019FEDE6
:1093E0001D0A361A07EE906AF8EE677A4FF4876026
:1093F00027EE800AB6EE001AF0EE480A14F008FFD5
:10940000DDED017A30EE270A04F1F0008DED010A5E
:1094100017F08CFA284604F0A3FC94F82C0105B050
:10942000BDEC028BF0BD707C242303FB006696ED3F
:109430000B8AFEF76FFED0ED9C7A9FED077AF8EE6F
:10944000E77AE8EE077AFDEEE77A17EE901AA9E7D9
:10945000000000006F12833A0000C842F8B5036FA5
:109460000B60436F4B60836F8B6000F14C050E46C1
:10947000074601F10C040FCD0FC40FCD0FC42B68AC
:10948000236007F1B00207CA06F1300383E8070042
:1094900007F1940207CA06F13C0383E8070007F1CD
:1094A0001C0207CA06F1480383E8070006F16001C1
:1094B0003846FFF755FF86F87000F8BD30B589B023
:1094C000044668460D4604F019F969462046FFF740
:1094D00097F818B90024204609B030BD04A804F05C
:1094E0000DF9204604A9FFF73BFF04460028F1D000
:1094F00004A9684604F08CFB85ED000AC5ED010A5D
:1095000085ED021AE7E700001FB500230C4601A90C
:10951000019302930393FFF7D1FF08B1039B2360EC
:1095200004B010BD30B585B001AD00230C4629460E
:10953000019302930393FFF7C1FF034618B195E827
:10954000030084E80300184605B030BDF8B50646B0
:109550000F461546FCF7EAFD044690B13946FCF784
:109560008DFB70B120463946FCF784FC044640B1BF
:10957000FCF7DCFD3946FCF7BFFC85ED000A204610
:10958000F8BDFEF7C7FD90F8083343B13046FFF74A
:10959000D7FC044618B1D6F84C312B60EFE7D6F86B
:1095A0004C312B600024EAE770B52DED048B164694
:1095B000FFF7CCFF054670B3FEF7ACFD90F93042E3
:1095C0004CB30DF045FDFDF717F9012823D9E4B29E
:1095D00007EE904AB8EE678A0DF03AFD90F8C43273
:1095E00096ED009AB02202FB0300D0ED2F8AFEF721
:1095F000A7FF38EE281A78EEC80A40F2614029EE3B
:10960000000A14F005FEB0EE408AFEF799FFC8EE9E
:10961000007AC6ED007ABDEC048B284670BD0000D0
:1096200008B505F055F9BDE8084005F04FB8000051
:1096300010B5044617F0C2FD50B904F10C0017F044
:10964000BDFD28B904F11800BDE8104017F0B6BD03
:10965000012010BD38B500F1280504462846FFF763
:10966000E7FF28B120460121BDE83840FFF714BAD2
:10967000D4ED107AB7EE007AF4EEC77AF1EE10FA74
:1096800006D5BFEE007AF4EEC77AF1EE10FA12DCDE
:109690002046FFF75BFB2846FFF7CAFF0028E1D111
:1096A000D4ED107AB2EE047AF0EEE77AF4EEC77AEF
:1096B000F1EE10FAD6DC38BD10B5044618F0D0F83B
:1096C0002046BDE8104017F035BD00002DE9F04FF1
:1096D0002DED048B9FEDC48A95B00446F0EE408AD0
:1096E0008DED028A8DED038A8DED048AFFF7BCFCB7
:1096F00014F086F80023054695F87921012AA8BFC1
:10970000012293423FD20021284612F0C1FE0123DC
:109710000028F1D008AB0BAA002128468DED0B8A5A
:109720008DED0C8A8DED0D8A13F0DEF89DED080AA3
:10973000B5EEC00AF1EE10FA23DD0BA817F0A2FC7B
:1097400011A904F128008DED110ACDED120A8DED5D
:10975000131A15F09FFB0EA88DED0E0AB0EE680AE5
:10976000CDED0F0A8DED101A17F07CFC11A904F154
:10977000E4008DED110ACDED120A8DED131A17F0EC
:1097800091FC0123B8E795F813130C2303FB015157
:1097900004F1280B01F5C471584615F07BFB84EDEC
:1097A000070A94ED3F0AC4ED080A70EE288A84ED9A
:1097B000091AC4ED3F8A0DF04BFC0646FEF7AAFCE1
:1097C00090F8093300932046FFF7BAFB80B130468A
:1097D000FDF712F802280BD996F8C4226169B0236C
:1097E00003FB026391F9001093F8D20088425FDA1C
:1097F00094ED3F7ADFED7D7AB4EEE77AF1EE10FA80
:109800005DD4D4ED538AFEF7A1FF38B1FCF78EFC8E
:1098100090F84E11FCF770FBF0EE408A236C626BFF
:10982000A16A1393B0EE680A11A81292119117F071
:1098300019FC04F5AA7102A88DED020ACDED030A08
:109840008DED041A17F02EFC6DF0F2FF0023074691
:1098500084F814312046FFF773FB002865D096F892
:10986000C422B02302FB033232445268C4F81821E8
:1098700096F8C42202FB033333449B68C4F81C31BE
:109880006DF0D6FF0123C4F8200184ED498A84EDF0
:109890004A8A84F82C31D4F80031002B58D102AB1D
:1098A00093E80700C4F80071F03484E8070006E08C
:1098B00006EB0212176FD4F80021BA4204D115B09A
:1098C000BDEC048BBDE8F08FD43393E8070094F827
:1098D00014310DF1080C8CE807001BB904F1F003FA
:1098E00083E807000123604684F8143104F5AA7167
:1098F00017F0A2FB11A904F14C008DED110ACDED7A
:10990000120A8DED131A15F0F3FAB5EEC00AF1EE56
:1099100010FA8DED110AD8BF9FED330ACDED120A72
:109920008DED131A84ED530A94E794ED3F7AD4ED4C
:10993000497ADDED026AE6EE877ADDED036AC4ED71
:10994000497AD4ED4A7AE7EE267AC4ED4A7AA2E75C
:10995000D4ED3F7A224B8DED058AF5EEC07AF1EE1B
:1099600010FA8DED068A0793A9D99FED1E7A94F817
:10997000143167EE877AB7EE007AC7EE279A1BB9E3
:10998000009B002B00F0AA80E36804F1F00102A81C
:10999000D3ED008A17F050FB69EEA88A8DED110A0D
:1099A00011A8B0EE680ACDED120A8DED131A17F06A
:1099B00059FB0EA905A88DED0E0ACDED0F0A8DED10
:1099C000101A17F06FFB05A8FFF776FE05A817F031
:1099D0000FFCD8B16DF02CFFC4F860016FE700BF39
:1099E000000080BF0AE81C4100000000CDCC4C3EC6
:1099F000CDCC4C3FCDCC4C3D920A06BF920A063FDF
:109A0000C2B8B23E728A0E3C5B82183901230193C0
:109A10000023CDE90833CDE90A33CDE90C335FEDFE
:109A20000E8A4FF0FF3A04F1E40895F87921012AF3
:109A30001046A8BF0120834257D20123002AFAD042
:109A400095F835130029F6D0B0EE690A404617F0B4
:109A50005DFB019B0DF12C09002B41D042460021FA
:109A60002046FFF757FC8DED0B0ACDED0C0A8DED6E
:109A70000D1A4846FEF746FE70BB4846FFF71CFE2F
:109A8000484617F0B5FB38BB05A9484617F07AFBE6
:109A9000484605A98DED080ACDED090A8DED0A1A93
:109AA00017F05CFB08A8B0EE409A17F0D9FEBAF1A7
:109AB000000F06D1F4EEC08AF1EE10FAD8BFB0EE76
:109AC000680AB5EEC09AF1EE10FAF7EE008A58BFB8
:109AD000F0EE408A4FF0000A0123A6E7009B96E7CC
:109AE00098E8070089E80700C3E7BAF1000F7FF4A0
:109AF00071AF002384F804312046FFF72FFA38B104
:109B00002046FFF71DFA002840F025818DED0A8AD6
:109B100095F8123395F878219A4240F233812B441C
:109B200093F83433002B00F02D8195F8133395F81A
:109B300079219A4240F226812B4493F83533002B49
:109B400000F0208108A9584615F0D2F98DED080AD9
:109B5000CDED090A8DED0A1A08A817F02FFB002891
:109B600040F0178108A817F043FB002840F011814E
:109B70005FED627A94ED357A68EEA78A5FED647ADC
:109B8000E7EE278A04F1B000C4ED358A17F068FECD
:109B9000A3685FED687A93ED007AB4EEE77AF1EEB0
:109BA00010FAF0EE408A00F1F8802046B0EE680A24
:109BB000FFF78CF908A817F055FAA3688DED110A84
:109BC000CDED120A8DED131A93ED000A11A817F0CE
:109BD00049FA204684ED1F0AC4ED200A84ED211ABB
:109BE000FFF72AFA28B1B2EE000A04F17C0017F060
:109BF0008DFA009BB3B33046FCF7FEFD012831D946
:109C000096F8C402B02303FB006696ED2F7AF0EEBF
:109C1000087AB4EEE77AF1EE10FA23D595F813033B
:109C20000C2303FB005595ED627AF1EE0C7AB4EE4D
:109C3000E77AF1EE10FA15DBD4ED1D7A1FED927A7A
:109C4000F4EEC77AF1EE10FA0CDD1FED947AF4EE23
:109C5000C77AF1EE10FA05D5B6EE000A04F17C00E1
:109C600017F054FA5FED9A7AF4EEE78AF1EE10FA03
:109C700022D51FED9C0A08A817F0F4F90EA88DED67
:109C80000E0A94ED3F0ACDED0F0A8DED101A17F074
:109C9000E9F911A904F1A0008DED110ACDED120A28
:109CA0008DED131A17F0FEF9D4ED2B7A94ED3F7A6F
:109CB00077EE877AC4ED2B7A94ED2B7AF1EE047A65
:109CC000B4EEE77AF1EE10FA3BDB13F099FD5FEDAD
:109CD000B27A94ED2B1A94ED280A21EE271A40F25D
:109CE000C530F1EE410A8DED011ACDED000A14F0F8
:109CF0008FFA9DED011ADDED000A84ED280A40F28D
:109D0000C63094ED290A14F083FA9DED011ADDEDB9
:109D1000000A84ED290A40F2C73094ED2A0A14F0B3
:109D200077FA04F1A00184ED2A0A04F1940017F0F7
:109D3000B9F984ED2A8A84ED298A84ED288A84ED94
:109D40002B8A0023C4F8E430C4F8E830C4F8EC30BF
:109D500084ED3F8AA3E5E368F7EE000A93ED000A7D
:109D600014F052F900283FF4D1AE94ED1C0AB0EE85
:109D7000C00A92F0B5FADDED0A7A27EE800A8DED81
:109D80000A0AC5E68DED0A8A8DED098A8DED088AED
:109D9000E2E62046FFF75EFC1CE6C3ED007A04E72E
:109DA0002DE9F04D2DED048B9EB0044613F028FDF7
:109DB000D0EDC87A90ED618AF4EE487AF1EE10FAAF
:109DC00048BFB0EE678ADFED5C7AB4EEE78AF1EE69
:109DD00010FA0EDD0023C4F8E430C4F8E830C4F80B
:109DE000EC300023C4F8FC301EB0BDEC048BBDE8A1
:109DF000F08D2046FEF7EEFD2046FEF7A7FFB0EE01
:109E0000480A2046FFF762FC2046FFF723FCFEF7D6
:109E100081F914AD00F5347204F1280114A815F08D
:109E2000B7F80FCD04F14C060FC60FCD0FC62B6847
:109E3000336004F1740204F1780304F1700104F159
:109E40004C0015F053FA94ED1E8AB0EE480A92F0D9
:109E5000F1F884ED650AB0EE480A92F041FA204626
:109E600084ED640AFEF7AAFDFEF754F904F5B47117
:109E7000FDF756FF6DF0DCFCD4F89831C31A632B64
:109E8000B2D9C4F898013EF071FB9FED2C9A0546BB
:109E90006DF0D6FCD4ED1C7A67EE897A074617EE92
:109EA000900A0E46F2F730FBD4ED1D7A67EE897A00
:109EB000824617EE900A8B46F2F726FB94ED1E0AB7
:109EC00020EE090A41EC180B14F00CF9D4F85C01EF
:109ED00010EE108AF2F718FBCDE91201D4F8580100
:109EE000F2F712FBCDE91001D4F85401F2F70CFBA4
:109EF000CDE90E01D4F8D800F2F706FBCDE90C014C
:109F0000D4F8D400F2F700FBCDE90A014046F2F79D
:109F1000FBFA0B4B01930B4B0093CDE908018DED40
:109F2000068BCDE904ABCDE90276074B074A084919
:109F300028463DF05DFF57E7CDCC4C3EE02E654214
:109F4000318C0B083B8C0B08F88B0B08028C0B0830
:109F5000488A0B0808B52DED048BB0EE609AF0EE40
:109F6000408A00F011F9B0EE408A89EE280A92F09A
:109F7000EDFADFED0B7A20EE270A92F07FFADFEDA3
:109F8000097A38EE278ADFED087A28EE278AF7EE7D
:109F9000007A37EEC00A28EE000ABDEC048B08BD3B
:109FA00041D3423E33938843A1D81943FFF7D2BF30
:109FB00008B52DED048B9FED189AF0EEE07AF4EEE3
:109FC000C97AF1EE10FAF0EE408AB0EE608A1ED443
:109FD00000F0DAF8DFED117A9FED117A70EE277A52
:109FE0009FED100AE8EEC77A9FED0F7A27EE800A00
:109FF000C8EE007A87EE270AB4EEC90AF1EE10FA2D
:10A0000005DBBDEC048BBDE8084092F07FBBBDECE6
:10A01000048BB7EE000A08BD000000343393884378
:10A02000F4FDD43B48A18F43CDCC9C3F427CD0ED86
:10A03000257A242101FB020292ED0B0AD2ED090AD6
:10A0400030EE270AFFF7B4BF38B52DED088BDFEDF2
:10A0500021AA9FED21AA9FED21BA0546B0EE409AB4
:10A06000F0EE609AB0EE408A1524013CA4B25CB3D5
:10A07000F0EE490A2846B0EE480AFFF76BFFF0EE13
:10A08000490A70EE698A284638EE2A0AFFF762FF0D
:10A09000B0EEE87A70EE697AB4EECA7AF1EE10FAB0
:10A0A00077EEE87A10D468EEAA8A40F2631088EE60
:10A0B000A70AB0EE4B1A38EE400AF0EE4A0A14F046
:10A0C000A7F8B0EE408AD0E7B0EE480ABDEC088BA6
:10A0D00038BD00BFCDCCCC3D0AD7233C0024744909
:10A0E000002343608360C360036143618361C36194
:10A0F000002380F82030704790F82020531CDBB2FA
:10A10000062B80F8203000EB820288BF002382ED0E
:10A11000010A88BF80F82030704700004FF0FF33FD
:10A1200010B543610E4BC0F8A8300023044680F8F8
:10A13000C830A830FFF7D4FF0A4BC4F8A83004F5A4
:10A1400086706CF0B1FA084B08491C60204634F068
:10A1500079FAD4F89030C4F89430204610BD00BF8E
:10A16000588E0B08688E0B0824870020F88E0B0889
:10A1700008B5A83040F0CAFADFED027A20EE270ACF
:10A1800008BD00BF00007A4490ED3C0ADFED057A7F
:10A19000B0EEC07AB4EEE77AF1EE10FA48BF90ED77
:10A1A0003D0A70470000003473B5D0F8A43004466F
:10A1B0000E4663B16DF03CFBD4F8A430C01A42F2F5
:10A1C0000F73984203D894ED280A02B070BD114B6A
:10A1D0001D687DB195F84E112846FBF74BFE48B13E
:10A1E00095F84E1101AA2846FBF7FCFB10B19DED36
:10A1F000010AEAE7242101FB064494ED0A0ADFED97
:10A20000067AB4EEE70AF1EE10FA58BFB0EE670A2C
:10A21000DBE700BF1C87002000000C4208B561B1DD
:10A220000378022B02D906486DF0D0FA5A1C02704E
:10A2300000EB83004160012008BD0846FCE700BF39
:10A24000208D0B082DE9F84305460E469146002463
:10A2500000F13C082B78A34211DD00234A46314629
:10A26000012010F065FA242363430746002158F8C3
:10A27000030010F06DFA874204D00134EAE70020B1
:10A28000BDE8F8830120FBE7054B1B682BB1416952
:10A290004A1C02D018463DF08FBF0020704700BF17
:10A2A000E089002002290BD8242303FB010191F847
:10A2B000390030B191F83A0018B191F83B0070477D
:10A2C000002070472DE9F04704466DF0B1FAD4F84C
:10A2D000F86042F21073861B9E4288BFC4F8F800F3
:10A2E00000274FF0240942F2107A237CFDB2AB42E2
:10A2F0001CD929462046FFF7D5FF70B109FB054858
:10A3000098ED0D0AD8ED097AD4ED250A30EE270A2A
:10A310002046FFF799FE88ED0C0A564504D909FB43
:10A320000540303034F066FB0137DEE7617C2046C3
:10A33000FFF73AFF84ED3D0ABDE8F08770B50446AB
:10A3400086B06DF075FAD4F89830C31AB3F57A7FF9
:10A3500005464FD3344B94ED257A1B68DFED336A05
:10A36000DB6AD4ED247A93F89C60B0EEC76AB4EE51
:10A37000E66AF1EE10FA32D5B0EEE76AB4EEE66ABC
:10A38000F1EE10FA2BD502A803F0B8F996BBFDF751
:10A39000C1FE02A9FDF7C4FC60B3DDED037A9FEDB9
:10A3A000247AF8EEE77A67EE877AC4ED257AC4F866
:10A3B0009850FDF7AFFEFDF77BFA2046FFF782FFCE
:10A3C00047F0D4FE0546D4F89400F2F79DF8194AF8
:10A3D000CDE900010621284641F018F80AE037EEE1
:10A3E000676AF7EE005AB0EEC66AB4EEE56AF1EEBF
:10A3F00010FA01DC06B070BDB0EEE76AB4EEE66AB2
